:100000000C94305D0C94565D0C94565D0C94565DCA
:100010000C94565D0C94565D0C94565D0C94565D94
:100020000C94565D0C94565D0C9440EC0C94565D0B
:100030000C94565D0C94565D0C9451E90C94565DED
:100040000C94565D0C94565D0C94565D0C94565D64
:100050000C9453620C94565D0C94565D0C94565D52
:100060000C94565D0C9403EA0C94565D0C94CBEB07
:100070000C9423EA0C94565D0C9499EB0C94565D09
:100080000C94565D0C94565D0C94FDEB0C94565DEF
:100090000C94565D0C94565D0C94565D0C94565D14
:1000A0000C94565D0C94565D0C94565D0C94565D04
:1000B0000C94565D0C94565D0C94565D0C94CEE9F0
:1000C0000C94565D0C94565D0C94565D0C94565DE4
:1000D0000C94565D0C94565D0C94565D0C94565DD4
:1000E0000C94565D0C94565D0C9476EA0C94565D17
:1000F0000C9482EB0C94565D0C94565D0C94565DFA
:100100000C94565D0C94565D0C94565D0C94565DA3
:100110000C94565D0C94565D0C94565D0C94565D93
:100120000C94565D0C94565D0C94565D0C94565D83
:100130000C94565D0C9490E90C94565D0C94565DAD
:100140000C94565D0C94565D0C94565D0C94565D63
:100150000C94565D0C94565D0C94565D0C94565D53
:100160000C9486610C94565D0C9475610C9443EA72
:100170000C94565D0C94565D0C94565D0C94565D33
:100180000C94565D0C94565D0C94565D0C94565D23
:100190000C94565D0C94565D0C94565D0C94565D13
:1001A0000C94565D0C94565D0C9480EC0C94B5EC5C
:1001B0000C94565D0C94565D0C94565D0C94565DF3
:1001C0000C94565D0C94565D0C94565D0C94565DE3
:1001D0000C94565D0C94565D0C94565D0C9463EA39
:1001E0000C94565D0C94565D0C94565D0C94565DC3
:1001F0000C94565D0C94565D0C94565DA164766427
:10020000BA63BA63BA636C64BA63BA63BA63BA6353
:10021000BA63BA63BA63BA63BA634D64BA63BA6362
:10022000BA63BA63BA634D6443643A640964BA63F7
:10023000BA63BA63BA63F663BA63BA63BA63BA639A
:10024000BA63BA63BA63BA63BA63E6638E6FD36F95
:100250000A74A873656FDF7357747B74B272EB72A4
:1002600015734D73796F1475AF74D574FF6F2F705C
:10027000656F5C708870CB70656F6B71656F656F53
:10028000D770FD70656FA37160727972656F9F7230
:10029000656F656F656F656F796FC971EE71656FB9
:1002A0001E72656F656F656F287276732576257689
:1002B000257625765D752576CC752576CC752576E3
:1002C0005D75257625762576CC75CC75CC7525762D
:1002D0005D752576CC7525765D75CC755D755D751E
:1002E000257625765D7525762576CC755D75257622
:1002F0005D755D755D755D752576257625765D7513
:1003000025765D755D755D7525762576637C447C07
:10031000177CFE7BCD76E67BBF7B947B7E7B517B1F
:10032000CD76257BF77AC97AB17A857A727A5C7A4A
:10033000CD763C7A117AFB79CD76CF79CD76CD76B4
:10034000B6799D79CD7685795A793279CD760679E7
:10035000CD76CD76CD76CD76D878AB787B78CD76E8
:100360004E78CD76CD76CD762178F4773D863E8673
:100370003F86408641864286528653863586CFAE7A
:10038000DEAEECAEFBAE0AAF19AFB1AEC0AE1CD55F
:1003900018D5DFD414D511D5DFD40DD509D505D5A1
:1003A00001D5FDD4E3D4F9D4F6D4F2D4EED4EAD412
:1003B000310B13050A050A0B130414141717010156
:1003C000002B0B1323370B130B1300000006060141
:1003D00000002A01050105000000000109081213B0
:1003E00000000320020601040000000001090911B9
:1003F000110000031F050C0E1D050C040A0000006F
:1004000010100101001E060A3C4B060A1A220004C5
:10041000050C0C0100001A0C030C030C030C030068
:1004200003031010000104190204283302041218F7
:100430000105050C0D01000016050A2940050A11E9
:100440001C0000000202010000120208080E02084F
:100450000105000E142028010100170407030600FF
:1004600000000000090911160000030F060A060A21
:10047000000000000000010B110001030E02047EC9
:100480009C020429350000031314010000270E18F4
:10049000040904090E180000000A0A0100000D0FEB
:1004A000190307050A0F180000000A0A0100000CD2
:1004B0000104637C010441520206060C0C01000099
:1004C00009050C050900000000050D0D15150000BB
:1004D00003080307171E0307090D0005050F0F0189
:1004E0000000070B100B10000000000107070D0DA6
:1004F000000001060104637C010441520104040A66
:100500000A01000030040D0D16040D0307182828F9
:1005100038380101000407131738071307130C18A4
:10052000000C1801010022050D0F1E050D050D0020
:1005300000000F0F01000003050C0F1E050C040B3B
:1005400000101525250101001C050C1122050C05C4
:100550000C000D1A222A01010002050C1122050CC3
:10056000050C000000000001010002050C1122052D
:100570000C050C0010102020010100010F15070BC5
:10058000070B070B0F14000F140001000000000000
:10059000000000000000000000000000000000005B
:1005A000000000000000000000000000000000004B
:1005B000000000000000000000000000000000003B
:1005C000000000000000000000000000000000002B
:101CE0000000001C000000001C000000001C0000A0
:101CF00000001C000000001C000000001C00000090
:101D0000001C000000001C000000001C000000007F
:101D10001C000000001C000000001C000000001C53
:101D2000000000001C000000001C000000001C005F
:101D30000000001C00000000000000000000000087
:101D4000000000000000001C000000001C0000005B
:101D5000001C000000000000000000000000000067
:101D60000000000000000000000000000000000073
:101D70000000000000000000000000000000000063
:101D80000000000000000000000000000000000053
:101D90000000000000000071C000000071C00000E1
:101DA0000071C000000071C000000071C0000000A0
:101DB00071C000000071C000000020800000000021
:101DC0000000000000000000000000000000000013
:101DD0000000000000000000000000000000000003
:101DE00000000000000000000000000000000000F3
:101DF00000000000000000000000000000000000E3
:101E000000000000000000000000000000000000D2
:101E100000000000000000000000000000000000C2
:101E200000000000000000000000000000000000B2
:101E300000000000000000000000000000000000A2
:101E400000000000000000000000000E380000004C
:101E50000E380000000E38000000000000000000F6
:101E600000000000000000000003F00000000FFC74
:101E70000000001F3E0000003C0F0000003807007B
:101E8000000078078000007003800000700380006D
:101E90000070038000007003800000700380000069
:101EA000700780000038070000003C0F0000001F92
:101EB0003E0000000FFC00000003F00000000000E6
:101EC0000000000000000000000000000000000012
:101ED0000000000000000000000000000000000002
:101EE00000000000000000000000000000000000F2
:101EF0000000000000000000000000000000000ED4
:101F0000380000000E380000000E3800000000000D
:101F10000000000000000000000000000007F000CA
:101F200000001FFC0000001E3C000000380E0000F6
:101F300000380E000000000E00000003FE0000004C
:101F40001FFE0000003F0E000000380E0000007071
:101F50000E000000700E000000700E000000781EE1
:101F60000000003C7E0000003FEE0000000F8E00ED
:101F70000000000000000000000000000000000061
:101F80000000000000000000000000000000000051
:101F90000000000000000000000000000000000041
:101FA0000000000000000000000000000000000031
:101FB00000000007C01C00000FE01800001EF030F9
:101FC00000003838300000383860000038386000D1
:101FD000003838C000003838C000001EF180000012
:101FE0000FE180000007C300000000071F00000091
:101FF000063F8000000C71C000000CE0E0000018FB
:10200000E0E0000018E0E0000030E0E0000030E038
:10201000E0000060F1E00000607BC00000C03F8095
:102020000001C01F000000000000000000000000D0
:1020300000000000000000000000000000000000A0
:102040000000000000000000000000000000000090
:102050000000000000000000000000000000000080
:102060000000000000000001F000000003FC000080
:102070000007BC0000000E0E0000000E0E00000065
:102080000E0E0000000F0E000000071C00000007ED
:10209000F800000003F000000003E00000000FE083
:1020A0000000001E70E000003C78E00000783CE09A
:1020B0000000701FE00000700FC000007007C0003B
:1020C000007807800000380FC000003E3FE00000AD
:1020D0000FFCE0000007F0400000000000000000DE
:1020E00000000000000000000000000000000000F0
:1020F00000000000000000000000000000000000E0
:1021000000000000000000000000000000000000CF
:1021100000000000000000000000000E3800000079
:102120000E380000000E3800000000000000000023
:102130000000000000000000003807000000380721
:1021400000000038070000003807000000380700D2
:1021500000003807000000380700000038070000C2
:1021600000380700000038070000003807000000B2
:102170003807000000380F0000003C1F0000001F5F
:102180007F0000000FF700000007C70000000000FC
:10219000000000000000000000000000000000003F
:1021A000000000000000000000000000000000002F
:1021B000000000000000000000000000000000001F
:1021C000000000000000000000000000000000010E
:1021D00080000000018000000003000000000700F4
:1021E00000000006000000000E000000000C0000CF
:1021F00000001C000000001C000000001C0000008B
:102200000038000000003800000000380000000026
:1022100038000000003800000000380000000038DE
:1022200000000000380000000038000000001C0022
:102230000000001C000000001C000000000C00005A
:1022400000000E0000000006000000000700000073
:102250000003000000000180000000018000000079
:10226000000000000000000000000000000000006E
:10227000000000000000000000000000000000005E
:1022800000000030000000003000000000180000D6
:1022900000001C000000000C000000000E00000008
:1022A000000600000000070000000007000000001A
:1022B000070000000003800000000380000000030E
:1022C0008000000003800000000380000000038005
:1022D0000000000380000000038000000003800075
:1022E00000000700000000070000000007000000D9
:1022F0000006000000000E000000000C00000000BE
:102300001C00000000180000000030000000003039
:1023100000000000000000000000000000000000BD
:1023200000000000000000000000000000000000AD
:102330000000000000000006000000000600000091
:1023400000060000000076E00000007FE0000000D2
:102350000F000000000F000000001D8000000019A9
:10236000C00000000080000000000000000000002D
:10237000000000000000000000000000000000005D
:10238000000000000000000000000000000000004D
:10239000000000000000000000000000000000003D
:1023A000000000000000000000000000000000002D
:1023B000000000000000000000000000000000001D
:1023C000000000000000000000000000000000000D
:1023D00000000000000000000000000000000000FD
:1023E00000000000000000000000000000000000ED
:1023F00000000000000000000000000000000000DD
:10240000E000000000E000000000E000000000E04C
:1024100000000000E000000000E00000003FFF803E
:1024200000003FFF80000000E000000000E000002E
:102430000000E000000000E000000000E0000000FC
:1024400000E000000000E0000000000000000000CC
:10245000000000000000000000000000000000007C
:10246000000000000000000000000000000000006C
:10247000000000000000000000000000000000005C
:10248000000000000000000000000000000000004C
:10249000000000000000000000000000000000003C
:1024A000000000000000000000000000000000002C
:1024B000000000000000000000000000000000001C
:1024C000000000000000000000000000000000000C
:1024D00000000000000000000000000000000000FC
:1024E00000000000000000000000000000000000EC
:1024F00000000000000000000000000000000000DC
:102500000000003C000000003C000000003C000017
:1025100000000C000000000C00000000180000008B
:102520000038000000001000000000000000000063
:10253000000000000000000000000000000000009B
:10254000000000000000000000000000000000008B
:10255000000000000000000000000000000000007B
:10256000000000000000000000000000000000006B
:10257000000000000000000000000000000000005B
:10258000000000000000000000000000000000004B
:102590000000000000000000007FC00000007FC0BD
:1025A000000000000000000000000000000000002B
:1025B000000000000000000000000000000000001B
:1025C000000000000000000000000000000000000B
:1025D00000000000000000000000000000000000FB
:1025E00000000000000000000000000000000000EB
:1025F00000000000000000000000000000000000DB
:1026000000000000000000000000000000000000CA
:1026100000000000000000000000000000000000BA
:1026200000000000000000000000000000000000AA
:10263000000000000000000000000000000000009A
:10264000000000000000000000000000000000008A
:10265000000000000000000000000000000000007A
:1026600000000000000000000000001C000000004E
:102670001C000000001C0000000000000000000022
:10268000000000000000000000000000000000004A
:10269000000000000000000000000000000000003A
:1026A000000000000000000000000000000000002A
:1026B0000000000000000000000000038000000097
:1026C00003000000000300000000030000000007FA
:1026D00000000000060000000006000000000E00E0
:1026E0000000000C000000000C000000000C0000C6
:1026F00000001C000000001800000000180000008E
:102700000038000000003000000000300000000031
:102710003000000000700000000060000000006059
:1027200000000000E000000000C000000000000009
:102730000000000000000000000000000000000099
:102740000000000000000000000000000000000089
:102750000000000000000000000000000000000079
:102760000000000000000000000000000000000366
:10277000E00000000FF80000001E3C0000001C1CE0
:10278000000000380E000000380E00000070070046
:1027900000007007000000700700000070070000D4
:1027A00000700700000070070000007007000000C4
:1027B0007007000000700700000070070000007044
:1027C00007000000380E000000380E0000001C1C3E
:1027D0000000001E3C0000000FF800000003E000B5
:1027E00000000000000000000000000000000000E9
:1027F00000000000000000000000000000000000D9
:1028000000000000000000000000000000000000C8
:1028100000000000000000000000000000000000B8
:102820000000000030000000007000000000F00018
:10283000000003F00000001FF00000000E70000018
:102840000000700000000070000000007000000038
:102850000070000000007000000000700000000028
:1028600070000000007000000000700000000070A8
:102870000000000070000000007000000000700008
:1028800000000070000000007000000000700000F8
:1028900000007000000000000000000000000000C8
:1028A0000000000000000000000000000000000028
:1028B0000000000000000000000000000000000018
:1028C0000000000000000000000000000000000008
:1028D0000000000000000003F00000000FFC0000FA
:1028E000001F3E0000003C0E000000380700000002
:1028F000380700000030070000000007000000005B
:1029000007000000000E000000001E000000003C58
:10291000000000007800000000F000000001E0006E
:10292000000003C000000007800000000F0000004E
:10293000001E000000003C00000000380000000005
:102940007FFF0000007FFF0000000000000000008B
:102950000000000000000000000000000000000077
:102960000000000000000000000000000000000067
:102970000000000000000000000000000000000057
:10298000000000000000000000000007E000000060
:102990001FF80000003E3C000000381E00000078D8
:1029A0000E000000300E000000000E000000001EAF
:1029B000000000003C00000001F800000001F800E9
:1029C0000000003C000000000E000000000F0000AE
:1029D00000000700000000070000003007000000B2
:1029E0007007000000780F000000380E0000003E65
:1029F0003C0000001FF800000007E000000000009D
:102A000000000000000000000000000000000000C6
:102A100000000000000000000000000000000000B6
:102A200000000000000000000000000000000000A6
:102A30000000000000000000000000000000000096
:102A40001C000000001C000000003C000000007C96
:102A500000000000FC00000000DC00000001DC00C1
:102A60000000039C000000031C000000071C000085
:102A7000000E1C0000001C1C0000001C1C000000BC
:102A8000381C000000701C0000007FFF8000007FE9
:102A9000FF800000001C000000001C000000001C63
:102AA000000000001C000000001C000000001C00D2
:102AB0000000000000000000000000000000000016
:102AC0000000000000000000000000000000000006
:102AD00000000000000000000000000000000000F6
:102AE00000000000000000000000000000000000E6
:102AF0000000001FFE0000001FFE00000038000064
:102B0000000038000000003800000000380000001D
:102B100000380000000038000000003FF000000016
:102B20003FFC0000003C3E000000300E00000000B2
:102B30000F00000000070000000007000000000771
:102B400000000000070000007007000000700E0089
:102B50000000381E0000003E3C0000001FF800008E
:102B60000007E0000000000000000000000000007E
:102B70000000000000000000000000000000000055
:102B80000000000000000000000000000000000045
:102B90000000000000000000000000000000000035
:102BA0000000000000000003F00000000FFC000027
:102BB000001F3E0000001C0E000000380E00000048
:102BC00038000000003000000000700000000073BA
:102BD000F000000077FC0000007E1E000000780E70
:102BE000000000700F000000700700000070070078
:102BF00000007007000000700700000038070000A8
:102C000000380E0000001C0E0000001F3C000000F9
:102C10000FF800000003F0000000000000000000BA
:102C200000000000000000000000000000000000A4
:102C30000000000000000000000000000000000094
:102C40000000000000000000000000000000000084
:102C500000000000000000000000003FFF800000B6
:102C60003FFF80000000038000000007000000001C
:102C7000070000000007000000000E000000000E2A
:102C8000000000001C000000001C000000003C00D0
:102C90000000003800000000380000000070000054
:102CA00000007000000000F000000000E0000000E4
:102CB00000E000000001C000000001C000000003AF
:102CC000C00000000380000000078000000000003A
:102CD00000000000000000000000000000000000F4
:102CE00000000000000000000000000000000000E4
:102CF00000000000000000000000000000000000D4
:102D000000000000000000000000000000000003C0
:102D1000E00000000FF80000001E3C0000003C1E18
:102D2000000000380E000000380E000000380E00D1
:102D300000003C1E0000001C1C0000000F7800007A
:102D40000007F000000007F00000001F7C000000FA
:102D50003C1E000000380E000000700700000070EC
:102D60000700000070070000007007000000380E28
:102D70000000003E3E0000001FFC00000007F000C5
:102D80000000000000000000000000000000000043
:102D90000000000000000000000000000000000033
:102DA0000000000000000000000000000000000023
:102DB0000000000000000000000000000000000013
:102DC00000000007E00000000FF80000001E7C007B
:102DD0000000381C000000380E000000700E0000DB
:102DE000007007000000700700000070070000007E
:102DF0007007000000380F0000003C3F0000001F7B
:102E0000F700000007E700000000070000000007CF
:102E1000000000000E000000300E000000380E0020
:102E20000000381C0000001E7C0000000FF80000AD
:102E30000007E000000000000000000000000000AB
:102E40000000000000000000000000000000000082
:102E50000000000000000000000000000000000072
:102E60000000000000000000000000000000000062
:102E70000000000000000000000000000000000052
:102E80000000000000000000000000000000000042
:102E900000000000001C000000001C000000001CDE
:102EA0000000000000000000000000000000000022
:102EB0000000000000000000000000000000000012
:102EC0000000000000000000000000000000000002
:102ED00000000000000000000000001C00000000D6
:102EE0001C000000001C00000000000000000000AA
:102EF00000000000000000000000000000000000D2
:102F000000000000000000000000000000000000C1
:102F100000000000000000000000000000000000B1
:102F200000000000000000000000000000000000A1
:102F30000000000000000000000000000000000091
:102F40000000000000000000001C000000001C0049
:102F50000000001C00000000000000000000000055
:102F60000000000000000000000000000000000061
:102F70000000000000000000000000000000000051
:102F80000000000000000000000000000000001C25
:102F9000000000001C000000001C000000000C00ED
:102FA0000000000C000000000C00000000180000F1
:102FB0000000100000000000000000000000000001
:102FC0000000000000000000000000000000000001
:102FD00000000000000000000000000000000000F1
:102FE00000000000000000000000000000000000E1
:102FF00000000000008000000007800000001F802B
:103000000000007E00000003F80000000FC0000078
:10301000003F000000003C000000003E00000000F7
:103020001F8000000003F000000000FC0000000012
:103030003F800000000F80000000018000000000C1
:103040000000000000000000000000000000000080
:103050000000000000000000000000000000000070
:103060000000000000000000000000000000000060
:103070000000000000000000000000000000000050
:103080000000000000000000000000000000000040
:103090000000000000000000000000000000000030
:1030A0000000000000000000000000000000000020
:1030B000003FFF8000003FFF800000000000000094
:1030C0000000000000000000000000000000000000
:1030D000000000003FFF8000003FFF800000000074
:1030E00000000000000000000000000000000000E0
:1030F00000000000000000000000000000000000D0
:1031000000000000000000000000000000000000BF
:1031100000000000000000000000000000000000AF
:10312000000000000000000000000000000000009F
:10313000000000000000000000000000000000008F
:10314000000000000000000000000000000000007F
:10315000000000000000000000000020000000004F
:103160003C000000003F000000000FC00000000312
:10317000F8000000007E000000001F800000000733
:10318000800000000F800000003F00000001F800F8
:10319000000007E00000003F800000003E0000004B
:1031A00000300000000000000000000000000000EF
:1031B000000000000000000000000000000000000F
:1031C00000000000000000000000000000000000FF
:1031D00000000000000000000000000000000000EF
:1031E00000000000000000000000000000000000DF
:1031F000000000000000000000000003F0000000DC
:103200000FFC0000001E3E0000003C0E00000038D5
:1032100007000000700700000070070000000007B2
:10322000000000000F000000001E000000003C0035
:103230000000007800000000F000000000E0000046
:103240000001C000000001C000000001C00000003B
:1032500001C00000000000000000000000000001AC
:10326000C000000001C000000001C000000000001C
:10327000000000000000000000000000000000004E
:10328000000000000000000000000000000000003E
:10329000000000000000000000000000000000002E
:1032A000000000000000000000000000000000001E
:1032B00007FC0000001FFF0000007E0FC00001F0AF
:1032C00001E00003C000700007800038000703E73A
:1032D0001C000E0FFF0C001C1E3E0C001C3C1E0EA2
:1032E0000018380E060038700E060030700E06000A
:1032F00030E01C060030E01C060030E01C0E003000
:10330000E01C0C0030E0381C0038E038180018F0E1
:103310007838001879FDF0001C3FBFC0000E1F1F59
:1033200000000E00000000078000000003E0000025
:103330000000FE078000003FFF80000007FC000047
:10334000000000000000000000000000000000007D
:10335000000000000000000000000000000000006D
:10336000000000007000000000F800000000F800FD
:10337000000001F800000001DC000000019C0000DA
:1033800000038E000000038E000000030E0000000A
:10339000070700000007070000000E038000000E72
:1033A000038000000E03C000001FFFC000001FFFCD
:1033B000C000003C01E000003800E000003800F0F0
:1033C0000000700070000070007000007000780055
:1033D00000E00038000000000000000000000000D5
:1033E00000000000000000000000000000000000DD
:1033F00000000000000000000000000000000000CD
:1034000000000000000000000000000000000000BC
:10341000000000000000001FFE0000001FFF8000F1
:10342000001C07C000001C01C000001C00E00000E0
:103430001C00E000001C00E000001C00E000001C7C
:1034400001C000001C03C000001FFF0000001FFFA0
:103450008000001C03C000001C00E000001C007085
:1034600000001C007000001C007000001C007000B8
:10347000001C007000001C00E000001C03E00000C5
:103480001FFFC000001FFE00000000000000000041
:10349000000000000000000000000000000000002C
:1034A000000000000000000000000000000000001C
:1034B000000000000000000000000000000000000C
:1034C000000000000000000000000000FE000000FE
:1034D00003FF80000007C7E000000E00E000001CB2
:1034E0000070000038007800003800380000380014
:1034F000000000700000000070000000007000007C
:10350000000070000000007000000000700000006B
:103510000070000000003800000000380038000093
:1035200038007000001C007000000E00F000000762
:10353000C7E0000003FF80000000FE000000000064
:10354000000000000000000000000000000000007B
:10355000000000000000000000000000000000006B
:10356000000000000000000000000000000000005B
:103570000000000000000000000000000000001F2C
:10358000FE0000001FFF8000001C07E000001C0080
:10359000F000001C007000001C003800001C003807
:1035A00000001C003C00001C001C00001C001C0053
:1035B000001C001C00001C001C00001C001C000063
:1035C0001C001C00001C001C00001C003C00001C17
:1035D000003800001C003800001C007000001C00B7
:1035E000F000001C07E000001FFF8000001FFE002D
:1035F00000000000000000000000000000000000CB
:1036000000000000000000000000000000000000BA
:1036100000000000000000000000000000000000AA
:10362000000000000000000000000000000000009A
:103630000000001FFFF000001FFFF000001C000052
:1036400000001C000000001C000000001C00000026
:10365000001C000000001C000000001C0000000016
:103660001C000000001FFFE000001FFFE000001C26
:10367000000000001C000000001C000000001C00F6
:103680000000001C000000001C000000001C0000E6
:1036900000001C000000001C000000001FFFF000E4
:1036A000001FFFF00000000000000000000000000C
:1036B000000000000000000000000000000000000A
:1036C00000000000000000000000000000000000FA
:1036D00000000000000000000000000000000000EA
:1036E000000000000000001FFFE000001FFFE000DE
:1036F000001C000000001C000000001C0000000076
:103700001C000000001C000000001C000000001C49
:10371000000000001C000000001FFF8000001FFFD1
:103720008000001C000000001C000000001C0000C5
:1037300000001C000000001C000000001C00000035
:10374000001C000000001C000000001C0000000025
:103750001C000000001C0000000000000000000031
:103760000000000000000000000000000000000059
:103770000000000000000000000000000000000049
:103780000000000000000000000000000000000039
:10379000000000000000000000000000FF0000002A
:1037A00003FFC0000007C3E000000F00F000001C92
:1037B000007800003C003800003800380000380075
:1037C00000000070000000007000000000700000A9
:1037D00000007007FC00007007FC000070001C0077
:1037E0000070001C000038001C000038001C0000A5
:1037F0003C001C00001C003C00000F007C00000787
:10380000C3FC000003FFDC000000FF0C0000000010
:1038100000000000000000000000000000000000A8
:103820000000000000000000000000000000000098
:103830000000000000000000000000000000000088
:103840000000000000000000000000000000001C5C
:10385000003800001C003800001C003800001C006C
:103860003800001C003800001C003800001C003824
:1038700000001C003800001C003800001C0038004C
:10388000001FFFF800001FFFF800001C00380000B8
:103890001C003800001C003800001C003800001C10
:1038A000003800001C003800001C003800001C001C
:1038B0003800001C003800001C003800001C0038D4
:1038C00000000000000000000000000000000000F8
:1038D00000000000000000000000000000000000E8
:1038E00000000000000000000000000000000000D8
:1038F00000000000000000000000000000000000C8
:103900000000001C000000001C000000001C000063
:1039100000001C000000001C000000001C00000053
:10392000001C000000001C000000001C0000000043
:103930001C000000001C000000001C000000001C17
:10394000000000001C000000001C000000001C0023
:103950000000001C000000001C000000001C000013
:1039600000001C000000001C000000001C00000003
:10397000001C00000000000000000000000000002B
:103980000000000000000000000000000000000037
:103990000000000000000000000000000000000027
:1039A0000000000000000000000000000000000017
:1039B00000000000000000001C000000001C0000CF
:1039C00000001C000000001C000000001C000000A3
:1039D000001C000000001C000000001C0000000093
:1039E0001C000000001C000000001C000000001C67
:1039F000000000001C000000001C000000001C0073
:103A00000000001C000000701C000000701C000082
:103A100000701C00000078380000003C78000000B6
:103A20001FF000000007C0000000000000000000C0
:103A30000000000000000000000000000000000086
:103A40000000000000000000000000000000000076
:103A50000000000000000000000000000000000066
:103A600000000000000000000000001C00780000C2
:103A70001C00F000001C01E000001C03C000001C42
:103A8000078000001C0F0000001C1E0000001C3CF2
:103A90000000001C780000001CF00000001DF00079
:103AA00000001FF80000001FBC0000001F1E0000E7
:103AB000001E0E0000001C0F0000001C078000000C
:103AC0001C03C000001C01C000001C01E000001C21
:103AD00000F000001C007800001C007800000000CE
:103AE00000000000000000000000000000000000D6
:103AF00000000000000000000000000000000000C6
:103B000000000000000000000000000000000000B5
:103B10000000000000000000000000000000001C89
:103B2000000000001C000000001C000000001C0041
:103B30000000001C000000001C000000001C000031
:103B400000001C000000001C000000001C00000021
:103B5000001C000000001C000000001C0000000011
:103B60001C000000001C000000001C000000001CE5
:103B7000000000001C000000001C000000001C00F1
:103B80000000001FFF8000001FFF8000001FFF805B
:103B90000000000000000000000000000000000025
:103BA0000000000000000000000000000000000015
:103BB0000000000000000000000000000000000005
:103BC00000000000000000000000000000000000F5
:103BD0000000001F000F80001F000F80001F801FCB
:103BE00080001F801F80001F801F80001DC03B8041
:103BF000001DC03B80001DC03B80001CC0738000C6
:103C00001CE07380001CE07380001C606380001C5B
:103C100070E380001C70E380001C30C380001C39FE
:103C2000C380001C39C380001C198380001C1F83C3
:103C300080001C1F8380001C0F0380001C0F03806A
:103C4000001C0F03800000000000000000000000C6
:103C50000000000000000000000000000000000064
:103C60000000000000000000000000000000000054
:103C70000000000000000000000000000000000044
:103C8000000000000000001E003800001E00380088
:103C9000001F003800001F803800001F803800001F
:103CA0001FC03800001DC03800001CE03800001C98
:103CB000F03800001C703800001C383800001C3C34
:103CC0003800001C1C3800001C0E3800001C0F3887
:103CD00000001C073800001C03B800001C03F8009B
:103CE000001C01F800001C00F800001C00F8000097
:103CF0001C007800001C007800000000000000009C
:103D000000000000000000000000000000000000B3
:103D100000000000000000000000000000000000A3
:103D20000000000000000000000000000000000093
:103D3000000000000000000000000000FF00000084
:103D400003FFC0000007C3E000000F00F000001EEA
:103D5000003800003C003C000038001C0000380027
:103D60001C000070000E000070000E000070000EBD
:103D7000000070000E000070000E000070000E00C9
:103D80000070000E000038001C000038001C00000D
:103D90003C003C00001C003800000F00F000000751
:103DA000C3E0000003FFC0000000FF0000000000AF
:103DB0000000000000000000000000000000000003
:103DC00000000000000000000000000000000000F3
:103DD00000000000000000000000000000000000E3
:103DE0000000000000000000000000000000001FB4
:103DF000FF0000001FFFC000001C03E000001C00CB
:103E0000E000001C007000001C007000001C00702E
:103E100000001C007000001C007000001C00E0008E
:103E2000001C01E000001FFFC000001FFF00000099
:103E30001C000000001C000000001C000000001C12
:103E4000000000001C000000001C000000001C001E
:103E50000000001C000000001C000000001C00000E
:103E60000000000000000000000000000000000052
:103E70000000000000000000000000000000000042
:103E80000000000000000000000000000000000032
:103E90000000000000000000000000000000000022
:103EA000000000007E00000003FFC0000007C3E028
:103EB00000000F00F000001E007800003C003C00F5
:103EC0000038001C000038001C000070000E0000CC
:103ED00070000E000070000E000070000E000070F8
:103EE000000E000070000E000070000E0000380090
:103EF0001C000038011C00003C03BC00001E03F83D
:103F000000000F01F0000007C3F8000003FFFC00F1
:103F100000007F1E000000000C00000000000000F8
:103F20000000000000000000000000000000000091
:103F30000000000000000000000000000000000081
:103F40000000000000000000000000000000000071
:103F5000000000000000001FFF8000001FFFE000C5
:103F6000001C01F000001C007000001C0038000064
:103F70001C003800001C003800001C003800001C29
:103F8000003800001C007000001C01F000001FFF42
:103F9000C000001FFF8000001C03C000001C01C007
:103FA00000001C00E000001C00E000001C0070008D
:103FB000001C007000001C007800001C003800008D
:103FC0001C003800001C003C000000000000000045
:103FD00000000000000000000000000000000000E1
:103FE00000000000000000000000000000000000D1
:103FF00000000000000000000000000000000000C1
:10400000000000000000000000000001FC000000B3
:1040100007FF0000001F0F8000001C03C0000038D5
:1040200001C000003801C000003800C000003C00A2
:104030000000003E000000001FE00000000FFE0036
:10404000000003FF800000007FC000000007C000E8
:10405000000001E000000000E000003000E000008F
:104060003800E000003800E000001C01C000001F24
:104070008F80000007FF00000001FC00000000002E
:104080000000000000000000000000000000000030
:104090000000000000000000000000000000000020
:1040A0000000000000000000000000000000000010
:1040B0000000000000000000000000000000007F81
:1040C000FFE000007FFFE0000000700000000070D3
:1040D0000000000070000000007000000000700090
:1040E0000000007000000000700000000070000080
:1040F0000000700000000070000000007000000070
:10410000007000000000700000000070000000005F
:1041100070000000007000000000700000000070DF
:10412000000000007000000000700000000070003F
:10413000000000000000000000000000000000007F
:10414000000000000000000000000000000000006F
:10415000000000000000000000000000000000005F
:10416000000000000000000000000000000000004F
:104170000000001C003800001C003800001C003843
:1041800000001C003800001C003800001C00380033
:10419000001C003800001C003800001C0038000023
:1041A0001C003800001C003800001C003800001CF7
:1041B000003800001C003800001C003800001C0003
:1041C0003800001C003800001E007800000E00704F
:1041D00000000F00F0000007C3E0000003FFC00074
:1041E0000000FF00000000000000000000000000D0
:1041F00000000000000000000000000000000000BF
:1042000000000000000000000000000000000000AE
:10421000000000000000000000000000000000009E
:1042200000000000000000F000380000700078007E
:1042300000700070000038007000003800E00000DE
:104240003800E000001C00E000001C01C000001E5F
:1042500001C000000E038000000E03800000070371
:104260008000000707000000070700000003870028
:104270000000038E000000018E00000001DC000041
:104280000001DC00000000FC00000000F80000005D
:104290000078000000007000000000000000000036
:1042A000000000000000000000000000000000000E
:1042B00000000000000000000000000000000000FE
:1042C00000000000000000000000000000000000EE
:1042D00000000000000000000000007007801C00CB
:1042E00070078038007007C03800700FC038003881
:1042F0000EC03800380CC07000380CE07000381C5C
:10430000E070001C1C6070001C1870E0001C38700D
:10431000E0000C3870E0000E3830C0000E3039C0BC
:10432000000E7039C000067019C0000760198000C7
:1043300007E01F800007E01F800003E00F800003FC
:10434000C00F000003C00F000001C0070000000004
:10435000000000000000000000000000000000005D
:10436000000000000000000000000000000000004D
:10437000000000000000000000000000000000003D
:1043800000000000000000000000000000000078B5
:1043900000F000003C00E000001C01C000000E0323
:1043A000C000000F078000000787000000038F0097
:1043B000000003DE00000001FC00000000F8000027
:1043C000000078000000007800000000FC00000001
:1043D00001FC00000003CE000000038F0000000776
:1043E000070000000F038000001E03C000001C0136
:1043F000E000003C00E000007800F0000070007871
:1044000000000000000000000000000000000000AC
:10441000000000000000000000000000000000009C
:10442000000000000000000000000000000000008C
:10443000000000000000000000000000000000007C
:10444000000000F0007800007800F000003800E084
:1044500000003C01E000001E03C000000E038000CD
:10446000000F078000000787000000038E00000097
:1044700003DE00000001FC00000000F80000000066
:10448000F8000000007000000000700000000070E4
:1044900000000000700000000070000000007000CC
:1044A00000000070000000007000000000700000BC
:1044B000000070000000000000000000000000008C
:1044C00000000000000000000000000000000000EC
:1044D00000000000000000000000000000000000DC
:1044E00000000000000000000000000000000000CC
:1044F000000000000000001FFFE000001FFFE000C0
:10450000000001E000000001C00000000380000086
:104510000007800000000F000000001E00000000E7
:104520001C000000003C000000007800000000F0CB
:1045300000000001E000000001E000000003C000F6
:10454000000007800000000F000000001F000000B6
:10455000001E000000003C000000007C0000000085
:104560007FFFE000007FFFE000000000000000008F
:10457000000000000000000000000000000000003B
:104580000000000000000000000000000000E70044
:10459000000000E700000000E7000000000000004D
:1045A0000000000000000000000000007E0000008D
:1045B00003FFC0000007C3E000000F00F000001E72
:1045C000007800003C003C000038001C000038006F
:1045D0001C000070000E000070000E000070000E45
:1045E000000070000E000070000E000070000E0051
:1045F0000070000E000038001C000038001C000095
:104600003C003C00001E007800000F00F000000796
:10461000C3E0000003FFC00000007E0000000000B7
:10462000000000000000000000000000000000008A
:10463000000000000000000000000000000000007A
:10464000000000000000038E000000038E00000048
:10465000038E0000000000000000000000000000C9
:104660007000000000F800000000F800000001FCED
:1046700000000001DC000000019C000000038E002F
:104680000000038E00000003070000000707000081
:104690000007070000000E038000000E03800000EA
:1046A0000E03C000001FFFC000001FFFE000003825
:1046B00000E000003800E000003800F0000070006A
:1046C0007000007000780000F000380000E0003852
:1046D00000000000000000000000000000000000DA
:1046E00000000000000000000000000000000000CA
:1046F000000000000000E700000000E700000000EC
:10470000E7000000000000000000000000000000C2
:104710000000001C003800001C003800001C00389D
:1047200000001C003800001C003800001C0038008D
:10473000001C003800001C003800001C003800007D
:104740001C003800001C003800001C003800001C51
:10475000003800001C003800001C003800001C005D
:104760003800001C003800001E007800000E0070A9
:1047700000000F00F0000007C3E0000003FFC000CE
:104780000000FF000000000000000000000000002A
:104790000000000000000000000000000000000019
:1047A0000000000000000000000000000000000009
:1047B00000000000000000000000000000000000F9
:1047C0000000000000000003F00000000FFC0000EB
:1047D000001F3C0000001C0E000000380E0000000E
:1047E000380E000000381C000000381C00000038A3
:1047F0003800000038700000003870000000387089
:10480000000000387C000000383E000000380F0037
:10481000000038078000003803C000003801C000E5
:10482000003801C0000039C1C0000039E780000035
:1048300038FF000000383E000000000000000000CB
:104840000000000000000000000000000000000068
:104850000000000000000000000000000000000058
:104860000000000000000000000000000000000048
:104870000000000000000000000000000000000038
:104880000000000000000000000000000000000028
:104890000000000000000000000000000000000018
:1048A0000000000000000000000000000000000008
:1048B00000000000000000000000000000000000F8
:1048C00000000000000000000000000000000000E8
:1048D00000000000000000000000000000000000D8
:1048E00000000000000000000000000000000000C8
:1048F00000000000000000000000000000FFFFC0FA
:104900000000FFFFC00000000000000000000000E9
:104910000000000000000000000000000000000097
:10492000000000000000000000000000000000384F
:10493000000000001C000000000C000000000E0041
:104940000000000000000000000000000000000067
:104950000000000000000000000000000000000057
:104960000000000000000000000000000000000047
:104970000000000000000000000000000000000037
:104980000000000000000000000000000000000027
:104990000000000000000000000000000000000017
:1049A0000000000000000000000000000000000007
:1049B00000000000000000000000000000000000F7
:1049C00000000000000000000000000000000000E7
:1049D00000000000000000000000000000000000D7
:1049E00000000000000000000000000000000000C7
:1049F00000000000000000000000000000000000B7
:104A00000007F00000001FFC0000001E3C0000003A
:104A1000380E000000380E000000000E00000003F9
:104A2000FE0000001FFE0000003F0E000000380ED8
:104A3000000000700E000000700E000000700E00FC
:104A40000000781E0000003C7E0000003FEE0000E9
:104A5000000F8E00000000000000000000000000B9
:104A60000000000000000000000000000000000046
:104A70000000000000000000000000000000000036
:104A80000000000000000000000000000000000026
:104A900000000000000000380000000038000000A6
:104AA000003800000000380000000038000000005E
:104AB000380000000039F00000003BFC0000003F1F
:104AC0003C0000003C0E000000380E0000003807DB
:104AD0000000003807000000380700000038070019
:104AE0000000380700000038070000003807000009
:104AF00000380E0000003C0E0000003F3C000000AB
:104B00003FF800000039F000000000000000000045
:104B10000000000000000000000000000000000095
:104B20000000000000000000000000000000000085
:104B30000000000000000000000000000000000075
:104B40000000000000000000000000000000000065
:104B50000000000000000000000000000000000055
:104B600000000000000000000003F00000000FFC47
:104B70000000001F3C0000003C0E000000380E004A
:104B800000007000000000700000000070000000D5
:104B900000700000000070000000007000000000C5
:104BA0007000000000380E0000003C0E0000001FE6
:104BB0003E0000000FFC00000003F00000000000B9
:104BC00000000000000000000000000000000000E5
:104BD00000000000000000000000000000000000D5
:104BE00000000000000000000000000000000000C5
:104BF00000000000000000000000000000000000B5
:104C00000700000000070000000007000000000788
:104C10000000000007000000000700000003E7009C
:104C200000000FFF0000001E3F0000003C0F0000CE
:104C30000038070000007007000000700700000047
:104C4000700700000070070000007007000000708F
:104C50000700000070070000003807000000381F40
:104C60000000001E3F0000000FF700000007E700F3
:104C70000000000000000000000000000000000034
:104C80000000000000000000000000000000000024
:104C90000000000000000000000000000000000014
:104CA0000000000000000000000000000000000004
:104CB00000000000000000000000000000000000F4
:104CC00000000000000000000000000000000000E4
:104CD0000003F00000000FFC0000001E3E0000007A
:104CE0003C0E000000380700000070070000007054
:104CF000070000007FFF0000007FFF000000700041
:104D00000000007000000000700000000038070084
:104D100000003C0F0000001F3E0000000FFC0000E0
:104D20000003F00000000000000000000000000090
:104D30000000000000000000000000000000000073
:104D40000000000000000000000000000000000063
:104D50000000000000000000000000000000000053
:104D60000000000000000007C00000000FE000008D
:104D7000001E000000001C000000001C00000000DD
:104D80001C000000007FC00000007FC00000001C6D
:104D9000000000001C000000001C000000001C00BF
:104DA0000000001C000000001C000000001C0000AF
:104DB00000001C000000001C000000001C0000009F
:104DC000001C000000001C000000001C000000008F
:104DD0001C000000001C000000000000000000009B
:104DE00000000000000000000000000000000000C3
:104DF00000000000000000000000000000000000B3
:104E000000000000000000000000000000000000A2
:104E10000000000000000000000000000000000092
:104E20000000000000000000000000000000000082
:104E300000000000000000000003E70000000FFF7A
:104E40000000001E3F0000003C0F0000003807007B
:104E500000007007000000700700000070070000ED
:104E600000700700000070070000007007000000DD
:104E700070070000003807000000381F0000001E07
:104E80003F0000000FF700000007E70000000007E8
:104E90000000003807000000380E0000001E3E0031
:104EA00000000FFC00000007F00000000000000000
:104EB00000000000000000000000000000000000F2
:104EC00000000000000000000000000000000038AA
:104ED000000000003800000000380000000038002A
:104EE0000000003800000000380000000038F80022
:104EF00000003BFC0000003F1E0000003E0F0000D1
:104F000000380700000038070000003807000000E4
:104F1000380700000038070000003807000000389C
:104F200007000000380700000038070000003807BD
:104F300000000038070000003807000000380700B4
:104F40000000000000000000000000000000000061
:104F50000000000000000000000000000000000051
:104F60000000000000000000000000000000000041
:104F70000000000000000000000000000000000031
:104F80000000003800000000380000000038000079
:104F90000000000000000000000000000000000011
:104FA0000038000000003800000000380000000059
:104FB0003800000000380000000038000000003811
:104FC0000000000038000000003800000000380039
:104FD0000000003800000000380000000038000029
:104FE0000000380000000038000000003800000019
:104FF0000038000000000000000000000000000079
:1050000000000000000000000000000000000000A0
:105010000000000000000000000000000000000090
:105020000000000000000000000000000000000080
:105030000000000000000038000000003800000000
:105040000038000000000000000000000000000028
:1050500000000000003800000000380000000038A8
:105060000000000038000000003800000000380098
:105070000000003800000000380000000038000088
:105080000000380000000038000000003800000078
:105090000038000000003800000000380000000068
:1050A0003800000000380000000038000000003820
:1050B0000000000038000000007800000000F00050
:1050C000000000E000000000000000000000000000
:1050D00000000000000000000000000000000000D0
:1050E0000000000000000000000000380000000088
:1050F00038000000003800000000380000000038D0
:10510000000000003800000000381E000000383C9D
:10511000000000387800000038F000000039E0009E
:1051200000003BC00000003F800000003FC00000C6
:10513000003FC00000003CE000000038F00000002C
:1051400038700000003878000000383C000000385B
:105150001C000000381E000000380E000000000097
:10516000000000000000000000000000000000003F
:10517000000000000000000000000000000000002F
:10518000000000000000000000000000000000001F
:1051900000000000000000000000000000000038D7
:1051A0000000000038000000003800000000380057
:1051B0000000003800000000380000000038000047
:1051C0000000380000000038000000003800000037
:1051D0000038000000003800000000380000000027
:1051E00038000000003800000000380000000038DF
:1051F0000000000038000000003800000000380007
:1052000000000038000000003800000000380000F6
:10521000000000000000000000000000000000008E
:10522000000000000000000000000000000000007E
:10523000000000000000000000000000000000006E
:10524000000000000000000000000000000000005E
:10525000000000000000000000000000000000004E
:10526000000000000000000000000000000000003E
:105270000038F07C00003BFCFF00003F3FCF000007
:105280003C0F078000380E038000380E0380003882
:105290000E038000380E038000380E038000380EA5
:1052A000038000380E038000380E038000380E03A0
:1052B0008000380E038000380E038000380E038013
:1052C00000380E0380000000000000000000000015
:1052D00000000000000000000000000000000000CE
:1052E00000000000000000000000000000000000BE
:1052F00000000000000000000000000000000000AE
:10530000000000000000000000000000000000009D
:10531000000000000000000000000000000000008D
:10532000000000000038F80000003BFC0000003FD7
:105330001E0000003E0F0000003807000000380784
:1053400000000038070000003807000000380700A0
:105350000000380700000038070000003807000090
:105360000038070000003807000000380700000080
:1053700038070000003807000000000000000000AF
:10538000000000000000000000000000000000001D
:10539000000000000000000000000000000000000D
:1053A00000000000000000000000000000000000FD
:1053B00000000000000000000000000000000000ED
:1053C00000000000000000000000000000000000DD
:1053D00000000000000000000003F00000000FFCCF
:1053E0000000001F3E0000003C0F000000380700D6
:1053F00000007807800000700380000070038000C8
:1054000000700380000070038000007003800000C3
:10541000700780000038070000003C0F0000001FEC
:105420003E0000000FFC00000003F0000000000040
:10543000000000000000000000000000000000006C
:10544000000000000000000000000000000000005C
:10545000000000000000000000000000000000004C
:10546000000000000000000000000000000000003C
:10547000000000000000000000000000000000002C
:105480000000000000000000000000000039F000F3
:1054900000003BFC0000003F3C0000003C0E000010
:1054A00000380E0000003807000000380700000038
:1054B00038070000003807000000380700000038F7
:1054C000070000003807000000380E0000003C0E06
:1054D0000000003F3C0000003FF800000039F000F1
:1054E0000000380000000038000000003800000014
:1054F0000038000000003800000000380000000004
:10550000000000000000000000000000000000009B
:10551000000000000000000000000000000000008B
:10552000000000000000000000000000000000007B
:10553000000000000000000000000000000000006B
:105540000003E70000000FFF0000001E3F00000006
:105550003C0F0000003807000000700700000070DA
:1055600007000000700700000070070000007007CF
:1055700000000070070000007007000000380700FE
:105580000000381F0000001E3F0000000FF7000061
:105590000007E7000000000700000000070000000F
:1055A00000070000000007000000000700000000E6
:1055B00007000000000000000000000000000000E4
:1055C00000000000000000000000000000000000DB
:1055D00000000000000000000000000000000000CB
:1055E00000000000000000000000000000000000BB
:1055F000000000000039E00000003BE00000003F38
:10560000000000003C0000000038000000003800EE
:1056100000000038000000003800000000380000E2
:1056200000003800000000380000000038000000D2
:1056300000380000000038000000003800000000C2
:1056400038000000003800000000000000000000EA
:10565000000000000000000000000000000000004A
:10566000000000000000000000000000000000003A
:10567000000000000000000000000000000000002A
:10568000000000000000000000000000000000001A
:10569000000000000000000000000000000000000A
:1056A0000000000000000000000FE00000001FF8F4
:1056B0000000003C7C000000701C000000701C001A
:1056C000000070000000007E000000003FE00000CD
:1056D000000FF800000001FC000000001E000000A8
:1056E000000E000000700E000000781E0000003C5C
:1056F0003C0000001FF80000000FE0000000000068
:105700000000000000000000000000000000000099
:105710000000000000000000000000000000000089
:105720000000000000000000000000000000000079
:105730000000000000000000000000000000000069
:105740000000000000000000001C000000001C0021
:105750000000001C000000001C000000007F800012
:1057600000007F800000001C000000001C00000002
:10577000001C000000001C000000001C00000000D5
:105780001C000000001C000000001C000000001CA9
:10579000000000001C000000001C000000001C00B5
:1057A0000000001E000000000F80000000078000C5
:1057B00000000000000000000000000000000000E9
:1057C00000000000000000000000000000000000D9
:1057D00000000000000000000000000000000000C9
:1057E00000000000000000000000000000000000B9
:1057F00000000000000000000000000000000000A9
:105800000000000000000000000000000000000098
:1058100000380700000038070000003807000000CB
:105820003807000000380700000038070000003883
:1058300007000000380700000038070000003807A4
:1058400000000038070000003807000000380F0093
:1058500000003C1F0000001F7F0000000FF7000049
:105860000007C7000000000000000000000000006A
:105870000000000000000000000000000000000028
:105880000000000000000000000000000000000018
:105890000000000000000000000000000000000008
:1058A00000000000000000000000000000000000F8
:1058B00000000000000000000000000000000000E8
:1058C0000000000000700E000000700E000000706C
:1058D0000E000000381C000000381C000000381CBE
:1058E0000000001C380000001C380000000C3000D4
:1058F00000000E700000000E700000000660000046
:105900000007E000000007E000000003C000000006
:1059100003C0000000018000000000000000000043
:105920000000000000000000000000000000000077
:105930000000000000000000000000000000000067
:105940000000000000000000000000000000000057
:105950000000000000000000000000000000000047
:105960000000000000000000000000000000000037
:10597000000000000000000000F0380E0000703849
:105980001C0000707C1C0000707C1C0000707C1CE3
:105990000000386C38000038EE38000038EE38006F
:1059A0000018C63000001DC77000001DC770000041
:1059B0000DC37000000F83E000000F83E000000FB4
:1059C00083E000000701C000000701C000000000E4
:1059D00000000000000000000000000000000000C7
:1059E00000000000000000000000000000000000B7
:1059F00000000000000000000000000000000000A7
:105A00000000000000000000000000000000000096
:105A10000000000000000000000000000000000086
:105A200000000000000000000000000000781E00E0
:105A30000000381C0000003C3C0000001E78000004
:105A4000000E700000000FE000000007E000000002
:105A500003C000000003C000000007E000000007D2
:105A6000E00000000E700000001E780000001C38EE
:105A7000000000381C000000781E000000700E00BE
:105A80000000000000000000000000000000000016
:105A90000000000000000000000000000000000006
:105AA00000000000000000000000000000000000F6
:105AB00000000000000000000000000000000000E6
:105AC00000000000000000000000000000000000D6
:105AD00000000000000000000000000000000000C6
:105AE000007007000000700E000000380E0000007B
:105AF000381E000000381C0000001C1C0000001CA8
:105B0000380000000C380000000E380000000E7055
:105B10000000000770000000076000000003E000C4
:105B2000000003E000000003C000000001C000000E
:105B30000001C000000001800000000380000000A0
:105B400007000000003F000000003E000000003C95
:105B50000000000000000000000000000000000045
:105B60000000000000000000000000000000000035
:105B70000000000000000000000000000000000025
:105B80000000000000000000000000000000000015
:105B900000000000007FFE0000007FFE000000000B
:105BA0001E000000003C000000007800000000F033
:105BB00000000000E000000001E000000003C00061
:105BC000000007800000000F000000000E00000031
:105BD000001C0000000038000000007800000000F9
:105BE0007FFF0000007FFF000000000000000000B9
:105BF00000000000000000000000000000000000A5
:105C00000000000000000000000000000000000094
:105C10000000000000000000000000000000000084
:105C2000000000000000000000000003C0000000B1
:105C300007C00000000F000000000E000000000E72
:105C4000000000000E000000000E000000000E002A
:105C50000000000E000000000E000000000E00001A
:105C600000001C000000003C00000000700000006C
:105C70000078000000001C000000001C0000000074
:105C80000E000000000E000000000E000000000EDC
:105C9000000000000E000000000E000000000E00DA
:105CA0000000000E000000000E00000000070000D1
:105CB000000007C000000003C0000000000000005A
:105CC00000000000000000000000000000000000D4
:105CD0000000000000000000000000000000001CA8
:105CE000000000001C000000001C000000001C0060
:105CF0000000001C000000001C000000001C000050
:105D000000001C000000001C000000001C0000003F
:105D1000001C000000001C000000001C000000002F
:105D20001C000000001C000000001C000000001C03
:105D3000000000001C000000001C000000001C000F
:105D40000000001C000000001C000000001C0000FF
:105D500000001C000000001C000000001C000000EF
:105D6000001C000000001C000000001C00000000DF
:105D70000000000000000000000000000000000023
:105D80000000000000000000000000000000000013
:105D900000000078000000007C000000001E0000F1
:105DA00000000E000000000E000000000E000000C9
:105DB000000E000000000E000000000E00000000B9
:105DC0000E000000000E00000000070000000007A9
:105DD0008000000001C000000003C00000000700B8
:105DE00000000007000000000E000000000E000090
:105DF00000000E000000000E000000000E00000079
:105E0000000E000000000E000000000E0000000068
:105E10000E000000001C000000007C000000007864
:105E20000000000000000000000000000000000072
:105E30000000000000000000000000000000000062
:105E4000000000000000001F008000007FE18000D3
:105E5000007FFF80000061FF800000403E000000E6
:105E60000000000000000000000000000000000032
:105E70000000000000000000000000000000000022
:105E80000000000000000000000000000000000012
:105E90000000000000000000000000000000000002
:105EA00000000000000000000000000000000000F2
:105EB00000000000000000000000000000000000E2
:105EC00000000000000000000000000000000000D2
:105ED000000000000000000009090909090909097A
:105EE0000909090909090909090909090909090922
:105EF000090909090909090909090B12111D1512D6
:105F00000B0B0C13090B09091112121112111112AA
:105F10001111090913131312211716171816141843
:105F200018091116121C1818151817151418161E12
:105F300016161418171813120B11111012120B1237
:105F400012070910071B121211120B100A12101758
:105F50001010110B090B12000100000005000000D9
:105F60002200000024000000E0FFFFFF000000000E
:105F70000000000000000000000000000000000021
:105F80000000000000000000000000000000000011
:105F90000000000000000000000000000000000001
:105FA00000000000000000000000000000000000F1
:106DF0000000000030000000300000003000000003
:106E000030000000300000003000000030000000C2
:106E100030000000300000003000000030000000B2
:106E20003000000030000000000000000000000002
:106E300000000000300000003000000000000000F2
:106E40000000000000000000000000000000000042
:106E50000000000000000000000000000000000032
:106E600000000000630000006300000063000000F9
:106E700063000000630000006300000000000000E9
:106E80000000000000000000000000000000000002
:106E900000000000000000000000000000000000F2
:106EA00000000000000000000000000000000000E2
:106EB00000000000000000000000000000000000D2
:106EC00000000000000000000000000000000000C2
:106ED000000000000CC000000CC00000000000001A
:106EE00000000000000000000FC000001FE00000D4
:106EF000387000003030000070380000601800006A
:106F00006018000060180000703800003030000089
:106F1000387000001FE000000FC0000000000000FB
:106F20000000000000000000000000000000000061
:106F30000000000000000000000000000000000051
:106F4000000000000CC000000CC0000000000000A9
:106F500000000000000000000FC000003FE0000043
:106F600038700000303000000030000007F00000F2
:106F70003FF000003830000070300000603000004A
:106F8000707000003FF000001F30000000000000A3
:106F900000000000000000000000000000000000F1
:106FA00000000000000000000000000000000000E1
:106FB000000000000F0180001F81000038C30000A6
:106FC00030C2000030C6000030C4000038CC0000E1
:106FD0001F8800000F1800000031E000003330006F
:106FE000006618000046180000C618000086180049
:106FF000018738000103F0000301E00000000000F9
:107000000000000000000000000000000000000080
:107010000000000000000000000000000000000070
:107020000000000007C000000FE000001C7000001E
:10703000183000001C7000001C7000000EE0000002
:10704000078000000F8000001F80000039C600008C
:1070500070EE0000607E0000603C0000701C0000CC
:10706000383E00001FFE00000FC4000000000000BA
:107070000000000000000000000000000000000010
:107080000000000000000000000000000000000000
:10709000000000000C6000000C6000000000000018
:1070A0000000000000000000303000003030000020
:1070B0003030000030300000303000003030000050
:1070C0003030000030300000303000003830000038
:1070D000387000001FF000000F30000000000000BA
:1070E00000000000000000000000000000000000A0
:1070F0000000000000000000000000000000000090
:1071000000000000060000000C0000000C00000061
:1071100018000000180000003000000030000000DF
:1071200030000000700000006000000060000000FF
:1071300060000000600000006000000070000000BF
:107140003000000030000000300000001800000097
:10715000180000000C0000000C00000000000000FF
:10716000000000000000000000000000000000001F
:1071700000000000200000003000000018000000A7
:10718000180000000C0000000C0000000E000000C1
:1071900006000000060000000600000006000000D7
:1071A00006000000060000000600000006000000C7
:1071B000060000000E0000000C0000000C000000A3
:1071C000180000001800000030000000000000005F
:1071D00000000000000000000000000000000000AF
:1071E000000000000C0000000C0000006D8000009A
:1071F0007F8000001C0000001E0000003300000023
:10720000000000000000000000000000000000007E
:10721000000000000000000000000000000000006E
:10722000000000000000000000000000000000005E
:10723000000000000000000000000000000000004E
:10724000000000000000000000000000000000003E
:10725000000000000000000000000000000000002E
:107260000300000003000000030000000300000012
:10727000030000007FF800007FF80000030000001A
:1072800003000000030000000300000003000000F2
:1072900000000000000000000000000000000000EE
:1072A00000000000000000000000000000000000DE
:1072B00000000000000000000000000000000000CE
:1072C00000000000000000000000000000000000BE
:1072D00000000000000000000000000000000000AE
:1072E000000000000000000000000000000000009E
:1072F000000000000000000000000000000000008E
:107300000000000018000000180000000800000045
:107310001800000010000000000000000000000045
:10732000000000000000000000000000000000005D
:10733000000000000000000000000000000000004D
:10734000000000000000000000000000000000003D
:10735000000000000000000000000000000000002D
:107360007F0000007F00000000000000000000001F
:10737000000000000000000000000000000000000D
:1073800000000000000000000000000000000000FD
:1073900000000000000000000000000000000000ED
:1073A00000000000000000000000000000000000DD
:1073B00000000000000000000000000000000000CD
:1073C00000000000000000000000000000000000BD
:1073D00000000000000000000000000000000000AD
:1073E000000000003000000030000000000000003D
:1073F000000000000000000000000000000000008D
:10740000000000000000000000000000000000007C
:107410000000000006000000060000000C00000054
:107420000C0000000C000000080000001800000024
:1074300018000000180000003000000030000000BC
:10744000300000002000000060000000600000002C
:1074500040000000C0000000C0000000000000006C
:10746000000000000000000000000000000000001C
:10747000000000000000000000000000000000000C
:10748000000000000F8000001FC0000038E0000076
:10749000307000007030000070300000603000007C
:1074A000603000006030000060300000603000009C
:1074B000603000007030000070300000307000005C
:1074C00038E000001FC000000F8000000000000036
:1074D00000000000000000000000000000000000AC
:1074E000000000000000000000000000000000009C
:1074F0000000000001800000018000000380000007
:107500001F8000001D80000001800000018000003D
:107510000180000001800000018000000180000067
:107520000180000001800000018000000180000057
:1075300001800000018000000180000000000000C8
:10754000000000000000000000000000000000003B
:10755000000000000000000000000000000000002B
:107560000000000007C000001FF0000038300000DD
:10757000303800003018000000180000003800000B
:10758000003000000070000000E0000001C00000BA
:10759000038000000F0000001E0000003C000000FF
:1075A000380000007FF800007FF8000000000000B5
:1075B00000000000000000000000000000000000CB
:1075C00000000000000000000000000000000000BB
:1075D000000000000F8000001FE000003870000075
:1075E00070700000003000000070000000600000BB
:1075F00003C0000003E0000000F000000070000085
:1076000000300000003000006030000070300000EA
:10761000306000003FE000000F800000000000002C
:10762000000000000000000000000000000000005A
:10763000000000000000000000000000000000004A
:10764000000000000060000000E0000001E0000019
:1076500001E0000003E0000006600000066000009A
:107660000C6000001860000018600000306000002E
:10767000606000007FF800007FF8000000600000FC
:1076800000600000006000000060000000000000DA
:1076900000000000000000000000000000000000EA
:1076A00000000000000000000000000000000000DA
:1076B000000000001FF800001FF00000180000008C
:1076C0001800000018000000380000003B80000097
:1076D0003FE0000038700000003800000018000093
:1076E00000180000001800003018000030380000BA
:1076F000387000001FE0000007C00000000000001C
:107700000000000000000000000000000000000079
:107710000000000000000000000000000000000069
:107720000000000007C000001FE00000187000000B
:10773000303800003000000070000000638000005E
:107740006FE00000787000007030000060380000CA
:107750006018000070180000303800003030000061
:10776000387000001FE0000007C0000000000000AB
:107770000000000000000000000000000000000009
:1077800000000000000000000000000000000000F9
:10779000000000007FF800007FF8000000380000C3
:1077A00000300000007000000060000000E00000F9
:1077B00000E0000000C0000001C0000001800000E7
:1077C0000380000003000000030000000700000029
:1077D000060000000E0000000C0000000000000089
:1077E0000000000000000000000000000000000099
:1077F0000000000000000000000000000000000089
:10780000000000000F8000001FE000003870000042
:107810003070000030300000307000003860000030
:107820001FC000000F8000001FE000003870000043
:107830007038000060180000601800007038000008
:10784000387000001FE000000FC0000000000000C2
:107850000000000000000000000000000000000028
:107860000000000000000000000000000000000018
:10787000000000000F8000001FE0000038700000D2
:1078800030300000703000006038000060180000E8
:107890007018000070380000387800001FF80000F1
:1078A00007180000003800000030000070300000B1
:1078B000386000001FE000000F80000000000000A2
:1078C00000000000000000000000000000000000B8
:1078D00000000000000000000000000000000000A8
:1078E0000000000000000000000000000000000098
:1078F0000000000000000000300000003000000028
:107900000000000000000000000000000000000077
:107910000000000000000000000000000000000067
:1079200000000000300000003000000000000000F7
:107930000000000000000000000000000000000047
:107940000000000000000000000000000000000037
:107950000000000000000000000000000000000027
:1079600000000000000000003000000030000000B7
:107970000000000000000000000000000000000007
:1079800000000000000000000000000000000000F7
:107990000000000030000000300000001000000077
:1079A00010000000200000000000000000000000A7
:1079B00000000000000000000000000000000000C7
:1079C00000000000000000000000000000000000B7
:1079D000000000000038000000F8000007E0000090
:1079E0001F0000007C000000700000007C00000010
:1079F0000F80000003E00000007800000018000085
:107A00000000000000000000000000000000000076
:107A10000000000000000000000000000000000066
:107A20000000000000000000000000000000000056
:107A30000000000000000000000000000000000046
:107A400000000000000000007FF800007FF8000048
:107A50000000000000000000000000007FF80000AF
:107A60007FF800000000000000000000000000009F
:107A70000000000000000000000000000000000006
:107A800000000000000000000000000000000000F6
:107A900000000000000000000000000000000000E6
:107AA00000000000000000000000000000000000D6
:107AB00000000000700000007C0000001F8000003B
:107AC00003E0000000F800000038000000F80000AB
:107AD00007C000001F0000007800000060000000E8
:107AE0000000000000000000000000000000000096
:107AF0000000000000000000000000000000000086
:107B00000000000000000000000000000000000075
:107B10000000000007C000001FE0000038700000F7
:107B20003038000070180000001800000038000015
:107B30000070000000E0000001C0000001800000B3
:107B400003800000030000000300000000000000AC
:107B5000000000000300000003000000000000001F
:107B60000000000000000000000000000000000015
:107B70000000000000000000000000000000000005
:107B800000000000003F800001FFE000038078005B
:107B90000F001C000C000E001C3CC60038FFC70084
:107BA00030C3C70031818300738183007301830078
:107BB00063018700630307006303060073070E0079
:107BC000738F1C0031FFF80038F3E0001C00000048
:107BD0000E0000000780000003FFE000000000002E
:107BE0000000000000000000000000000000000095
:107BF0000000000001C0000003C0000003C000003E
:107C00000360000006600000067000000E300000F7
:107C10000C3000000C3800001C180000181C00007C
:107C20003FFC00003FFC0000300E0000700600002A
:107C30006007000060070000E00380000000000013
:107C40000000000000000000000000000000000034
:107C50000000000000000000000000000000000024
:107C6000000000003FE000003FF80000301C000072
:107C7000300C0000300C0000300C0000300C000014
:107C8000301800003FF000003FFC0000300E000004
:107C9000300600003006000030060000300600000C
:107CA000300E00003FFC00003FF00000000000002C
:107CB00000000000000000000000000000000000C4
:107CC00000000000000000000000000000000000B4
:107CD0000000000003F000000FFC00001C0E00007C
:107CE0003807000030030000300000007000000082
:107CF0006000000060000000600000006000000004
:107D0000700000003003000030030000380700005E
:107D10001C0E00000FFC000003F00000000000003B
:107D20000000000000000000000000000000000053
:107D30000000000000000000000000000000000043
:107D4000000000003FF000003FFC0000300E00008B
:107D50003007000030030000300380003003800053
:107D6000300180003001800030018000300180004F
:107D70003003800030038000300300003007000033
:107D8000300E00003FFC00003FF00000000000004B
:107D900000000000000000000000000000000000E3
:107DA00000000000000000000000000000000000D3
:107DB000000000003FFE00003FFE00003000000019
:107DC00030000000300000003000000030000000F3
:107DD000300000003FFE00003FFC000030000000CB
:107DE00030000000300000003000000030000000D3
:107DF000300000003FFE00003FFF000000000000D8
:107E00000000000000000000000000000000000072
:107E10000000000000000000000000000000000062
:107E2000000000003FFC00003FFC000030000000AC
:107E30003000000030000000300000003000000082
:107E4000300000003FF800003FF800003000000064
:107E50003000000030000000300000003000000062
:107E60003000000030000000300000000000000082
:107E70000000000000000000000000000000000002
:107E800000000000000000000000000000000000F2
:107E90000000000001F8000007FE00001E070000BF
:107EA000180380003801800030018000700000005D
:107EB0006000000060000000601FC000601FC00084
:107EC0007000C0003000C0003800C0001801C000C1
:107ED0001E07C00007FEC00001F8C000000000003F
:107EE0000000000000000000000000000000000092
:107EF0000000000000000000000000000000000082
:107F000000000000300300003003000030030000D8
:107F10003003000030030000300300003003000095
:107F2000300300003FFF00003FFF0000300300006F
:107F30003003000030030000300300003003000075
:107F40003003000030030000300300000000000098
:107F50000000000000000000000000000000000021
:107F60000000000000000000000000000000000011
:107F70000000000030000000300000003000000071
:107F80003000000030000000300000003000000031
:107F90003000000030000000300000003000000021
:107FA0003000000030000000300000003000000011
:107FB0003000000030000000300000000000000031
:107FC00000000000000000000000000000000000B1
:107FD00000000000000000000000000000000000A1
:107FE0000000000000600000006000000060000071
:107FF0000060000000600000006000000060000001
:1080000000600000006000000060000000600000F0
:1080100000600000006000006060000070E0000090
:1080200070C000003FC000001F0000000000000002
:108030000000000000000000000000000000000040
:108040000000000000000000000000000000000030
:108050000000000030070000300E0000301C00005F
:10806000303800003070000030E0000031C0000007
:10807000338000003FC000003FC000003CE0000033
:10808000387000003038000030380000301C00002C
:10809000300E0000300F000030070000000000002C
:1080A00000000000000000000000000000000000D0
:1080B00000000000000000000000000000000000C0
:1080C0000000000030000000300000003000000020
:1080D00030000000300000003000000030000000E0
:1080E00030000000300000003000000030000000D0
:1080F00030000000300000003000000030000000C0
:10810000300000003FF800003FF8000000000000D1
:10811000000000000000000000000000000000005F
:10812000000000000000000000000000000000004F
:10813000000000003C01E0003C01E0003C01E000E8
:108140003E03E00036036000360360003306600043
:108150003306600033066000318C6000318C6000B3
:10816000318C600030D8600030D8600030F860009A
:1081700030706000307060003070600000000000FF
:1081800000000000000000000000000000000000EF
:1081900000000000000000000000000000000000DF
:1081A00000000000380300003C0300003C03000016
:1081B0003E0300003E03000037030000338300004D
:1081C0003183000031C3000030E300003063000061
:1081D00030730000303B0000301F0000301F0000F3
:1081E000300F0000300F00003007000000000000DA
:1081F000000000000000000000000000000000007F
:10820000000000000000000000000000000000006E
:108210000000000003F8000007FC00001E0F000033
:108220001803000038038000300180007001C00096
:108230006000C0006000C0006000C0006000C000BE
:108240007001C00030018000380380001803000076
:108250001E0F000007FC000003F8000000000000F3
:10826000000000000000000000000000000000000E
:1082700000000000000000000000000000000000FE
:10828000000000003FF000003FFC0000300E000046
:108290003006000030060000300600003006000006
:1082A000300E0000301C00003FF800003FE00000EE
:1082B00030000000300000003000000030000000FE
:1082C000300000003000000030000000000000001E
:1082D000000000000000000000000000000000009E
:1082E000000000000000000000000000000000008E
:1082F0000000000003F8000007FC00001E0F000053
:108300001803000038038000300180007001C000B5
:108310006000C0006000C0006000C0006000C000DD
:108320007001C0003001C000381B8000181F8000A1
:108330001E0F000007FF800003F9C000000080004E
:10834000000000000000000000000000000000002D
:10835000000000000000000000000000000000001D
:10836000000000003FFC00003FFE0000300700005E
:108370003003000030030000300300003003000031
:10838000300700003FFE00003FF80000301C0000F6
:10839000300E0000300600003006000030070000FC
:1083A00030030000300300003003800000000000B4
:1083B00000000000000000000000000000000000BD
:1083C00000000000000000000000000000000000AD
:1083D0000000000007E000000FF80000181C00007B
:1083E000380E0000300E0000380000003C00000095
:1083F0001FC000000FF8000003FC0000003E00005A
:10840000000E0000300600003006000038060000B4
:108410001C0C00000FFC000007F000000000000032
:10842000000000000000000000000000000000004C
:10843000000000000000000000000000000000003C
:10844000000000007FFE00007FFE000001800000B1
:108450000180000001800000018000000180000018
:108460000180000001800000018000000180000008
:1084700001800000018000000180000001800000F8
:108480000180000001800000018000000000000069
:1084900000000000000000000000000000000000DC
:1084A00000000000000000000000000000000000CC
:1084B0000000000030030000300300003003000023
:1084C00030030000300300003003000030030000E0
:1084D00030030000300300003003000030030000D0
:1084E00030030000380700003807000018060000BD
:1084F0001C0E00000FFC000003F000000000000054
:10850000000000000000000000000000000000006B
:10851000000000000000000000000000000000005B
:1085200000000000E003000060070000700700008A
:1085300070060000300E0000380C0000180C00001F
:10854000181C00001C1800000C1800000E30000061
:1085500006300000067000000760000003600000A5
:1085600003E0000001C0000001C0000000000000A6
:1085700000000000000000000000000000000000FB
:1085800000000000000000000000000000000000EB
:1085900000000000E0380600603C0E00603C0E0069
:1085A000707C0C00306C0C0030661C0030661C00C7
:1085B00038C6180018C3180018C3180018C33000B4
:1085C0001D8330000D81B0000D81B0000F01E0006F
:1085D0000701E0000700E0000700E00000000000E5
:1085E000000000000000000000000000000000008B
:1085F000000000000000000000000000000000007B
:108600000000000070070000380E0000181C000079
:108610001C1800000E3800000770000003E0000086
:1086200003C0000001C0000003C0000003E0000020
:10863000077000000E3800001C180000181C000015
:10864000380E000070060000E00700000000000087
:10865000000000000000000000000000000000001A
:10866000000000000000000000000000000000000A
:1086700000000000E007000070060000300E00005F
:10868000381C00001C1800000C3800000E700000A0
:108690000760000003E0000003C00000018000004C
:1086A00001800000018000000180000001800000C6
:1086B0000180000001800000018000000000000037
:1086C00000000000000000000000000000000000AA
:1086D000000000000000000000000000000000009A
:1086E000000000003FFE00003FFE0000000E000002
:1086F000001C000000380000007000000060000056
:1087000000E0000001C0000003800000070000003E
:10871000060000000E0000001C00000038000000F1
:10872000700000007FFE00007FFE000000000000DF
:108730000000000000000000000000000000000039
:1087400000000000031800000318000000000000F3
:108750000000000003F8000007FC00001E0F0000EE
:108760001803000038038000300180007001C00051
:108770006000C0006000C0006000C0006000C00079
:108780007001C00030018000380380001803000031
:108790001E0F000007FC000003F8000000000000AE
:1087A00000000000000000000000000000000000C9
:1087B000000000000000000006300000063000004D
:1087C0000000000001C0000001C0000003E0000044
:1087D0000360000007700000063000000630000053
:1087E0000E3800000C1800000C1C00001C0C0000CF
:1087F0001FFC00003FFE00003006000030070000B4
:108800007007000060038000E003800000000000AB
:108810000000000000000000000000000000000058
:1088200000000000033000000330000000000000E2
:10883000000000003003000030030000300300009F
:10884000300300003003000030030000300300005C
:10885000300300003003000030030000300300004C
:108860003003000038070000380700001806000039
:108870001C0E00000FFC000003F0000000000000D0
:1088800000000000000000000000000000000000E8
:1088900000000000000000000000000000000000D8
:1088A0000000000007C000001FE00000187000007A
:1088B00038300000307000003060000030E0000010
:1088C00030C0000030C0000030E000003070000018
:1088D000303C0000300E0000300E0000300600007A
:1088E000330E000031FC000030F8000000000000F2
:1088F0000000000000000000000000000000000078
:108900000000000000000000000000000000000067
:108910000000000000000000000000000000000057
:108920000000000000000000000000000000000047
:108930000000000000000000000000000000000037
:108940000000000000000000000000000000000027
:108950000000000000000000000000000000000017
:1089600000000000FFFC0000FFFC00000000000011
:1089700000000000000000000000000000000000F7
:108980000000000070000000380000001800000027
:1089900000000000000000000000000000000000D7
:1089A00000000000000000000000000000000000C7
:1089B00000000000000000000000000000000000B7
:1089C00000000000000000000000000000000000A7
:1089D0000000000000000000000000000000000097
:1089E0000000000000000000000000000000000087
:1089F0000000000000000000000000000000000077
:108A000000000000000000000FC000003FE0000078
:108A100038700000303000000030000007F0000027
:108A20003FF000003830000070300000603000007F
:108A3000707000003FF000001F30000000000000D8
:108A40000000000000000000000000000000000026
:108A50000000000000000000000000000000000016
:108A60000000000030000000300000003000000076
:108A7000300000003000000033C000003FF0000074
:108A80003C3000003838000030180000301800007A
:108A90003018000030180000301800003038000096
:108AA000383000003FF0000033C00000000000003C
:108AB00000000000000000000000000000000000B6
:108AC00000000000000000000000000000000000A6
:108AD0000000000000000000000000000000000096
:108AE000000000000000000007C000001FE00000C0
:108AF000387000003030000070000000600000009E
:108B000060000000600000007000000030300000D5
:108B1000387000001FE0000007C0000000000000E7
:108B20000000000000000000000000000000000045
:108B30000000000000000000000000000000000035
:108B40000000000000300000003000000030000095
:108B500000300000003000000FB000001FF00000E7
:108B600038700000303000007030000060300000CD
:108B70006030000060300000703000007030000095
:108B8000387000001FF000000F30000000000000EF
:108B900000000000000000000000000000000000D5
:108BA00000000000000000000000000000000000C5
:108BB00000000000000000000000000000000000B5
:108BC00000000000000000000FC000001FE00000D7
:108BD0003870000030300000701800007FF800008E
:108BE0007FF80000600000007000000030380000D6
:108BF000383000001FE0000007C000000000000047
:108C00000000000000000000000000000000000064
:108C10000000000000000000000000000000000054
:108C200000000000070000000F0000001C00000012
:108C300018000000180000007F0000007F00000006
:108C400018000000180000001800000018000000C4
:108C500018000000180000001800000018000000B4
:108C600018000000180000001800000000000000BC
:108C700000000000000000000000000000000000F4
:108C800000000000000000000000000000000000E4
:108C900000000000000000000000000000000000D4
:108CA00000000000000000000FB000001FF00000F6
:108CB000387000003030000070300000603000007C
:108CC0006030000060300000703000007030000044
:108CD000387000001FF000000F300000003000006E
:108CE00030300000387000001FE00000000000007D
:108CF0000000000000000000000000000000000074
:108D000000000000300000003000000030000000D3
:108D1000300000003000000033C000003FF00000D1
:108D20003C7000003830000030300000303000006F
:108D300030300000303000003030000030300000B3
:108D40003030000030300000303000000000000003
:108D50000000000000000000000000000000000013
:108D60000000000000000000000000000000000003
:108D70000000000030000000300000000000000093
:108D80000000000000000000300000003000000083
:108D90003000000030000000300000003000000013
:108DA0003000000030000000300000003000000003
:108DB0003000000030000000300000000000000023
:108DC00000000000000000000000000000000000A3
:108DD0000000000000000000000000000000000093
:108DE0000000000030000000300000000000000023
:108DF0000000000000000000300000003000000013
:108E000030000000300000003000000030000000A2
:108E10003000000030000000300000003000000092
:108E20003000000030000000300000003000000082
:108E30003000000030000000F000000000000000E2
:108E40000000000000000000000000000000000022
:108E50000000000030000000300000003000000082
:108E600030000000300000003070000030E00000F2
:108E700031C0000033800000370000003F000000D8
:108E80003F0000003980000031C0000030C0000009
:108E900030E00000307000003030000000000000C2
:108EA00000000000000000000000000000000000C2
:108EB00000000000000000000000000000000000B2
:108EC0000000000030000000300000003000000012
:108ED00030000000300000003000000030000000D2
:108EE00030000000300000003000000030000000C2
:108EF00030000000300000003000000030000000B2
:108F000030000000300000003000000000000000D1
:108F10000000000000000000000000000000000051
:108F20000000000000000000000000000000000041
:108F30000000000000000000000000000000000031
:108F4000000000000000000033C3C0003FEFE0005D
:108F50003C78600038307000303070003030700085
:108F600030307000303070003030700030307000C1
:108F70003030700030307000303070000000000081
:108F800000000000000000000000000000000000E1
:108F900000000000000000000000000000000000D1
:108FA00000000000000000000000000000000000C1
:108FB000000000000000000033C000003FF000008F
:108FC0003C700000383000003030000030300000CD
:108FD0003030000030300000303000003030000011
:108FE0003030000030300000303000000000000061
:108FF0000000000000000000000000000000000071
:109000000000000000000000000000000000000060
:109010000000000000000000000000000000000050
:1090200000000000000000000FC000001FE0000072
:109030003870000030300000703800006018000008
:109040006018000060180000703800003030000028
:10905000387000001FE000000FC00000000000009A
:109060000000000000000000000000000000000000
:1090700000000000000000000000000000000000F0
:1090800000000000000000000000000000000000E0
:10909000000000000000000033C000003FF00000AE
:1090A0003C30000038380000301800003018000054
:1090B0003018000030180000301800003038000070
:1090C000383000003FF0000033C0000030000000E6
:1090D0003000000030000000300000000000000000
:1090E0000000000000000000000000000000000080
:1090F0000000000000000000000000000000000070
:1091000000000000000000000FB000001FF0000091
:109110003870000030300000703000006030000017
:1091200060300000603000007030000070300000DF
:10913000387000001FF000000F3000000030000009
:10914000003000000030000000300000000000008F
:10915000000000000000000000000000000000000F
:1091600000000000000000000000000000000000FF
:109170000000000000000000338000003F000000FD
:10918000380000003800000030000000300000000F
:10919000300000003000000030000000300000000F
:1091A000300000003000000030000000000000002F
:1091B00000000000000000000000000000000000AF
:1091C000000000000000000000000000000000009F
:1091D000000000000000000000000000000000008F
:1091E00000000000000000001F8000003FC00000E1
:1091F00070E0000060600000700000003E000000B1
:109200001FC0000001E0000000600000606000007E
:1092100070E000003FC000001F8000000000000060
:10922000000000000000000000000000000000003E
:10923000000000000000000000000000000000002E
:109240000000000000000000000000001800000006
:1092500018000000180000007E0000007E000000E2
:10926000180000001800000018000000180000009E
:10927000180000001800000018000000180000008E
:10928000180000001E0000000E000000000000009A
:1092900000000000000000000000000000000000CE
:1092A00000000000000000000000000000000000BE
:1092B00000000000000000000000000000000000AE
:1092C00000000000000000003030000030300000DE
:1092D000303000003030000030300000303000000E
:1092E00030300000303000003030000038300000F6
:1092F000387000001FF000000F3000000000000078
:10930000000000000000000000000000000000005D
:10931000000000000000000000000000000000004D
:10932000000000000000000000000000000000003D
:1093300000000000000000006030000060700000CD
:10934000706000003060000030C0000038C00000D5
:1093500019C00000198000000D8000000F8000007F
:109360000F000000070000000600000000000000E1
:1093700000000000000000000000000000000000ED
:1093800000000000000000000000000000000000DD
:1093900000000000000000000000000000000000CD
:1093A0000000000000000000E0C1C00060E180009B
:1093B00061E1800071E1800071E3800033330000DF
:1093C00033330000333300001F1E00001E1E000058
:1093D0001E1E00000E1C00000C0C0000000000000F
:1093E000000000000000000000000000000000007D
:1093F000000000000000000000000000000000006D
:10940000000000000000000000000000000000005C
:1094100000000000000000007070000030E000005C
:1094200038C000001D8000000F8000000F00000009
:10943000070000000F0000001D80000019C00000A0
:1094400038E0000070600000607000000000000064
:10945000000000000000000000000000000000000C
:1094600000000000000000000000000000000000FC
:1094700000000000000000000000000000000000EC
:109480000000000000000000E070000060600000CC
:1094900060E0000070E0000030C0000031C000005B
:1094A00039800000198000001B8000000F000000C0
:1094B0000F0000000E000000060000000600000083
:1094C0000C0000001C0000007800000000000000FC
:1094D000000000000000000000000000000000008C
:1094E000000000000000000000000000000000007C
:1094F00000000000000000007FF000007FF000008E
:1095000000E0000001C0000001C000000380000076
:10951000070000000E0000001C00000038000000E2
:10952000300000007FF000007FF00000000000002D
:10953000000000000000000000000000000000002B
:10954000000000000000000000000000000000001B
:10955000000000000F0000000E0000001C000000D2
:10956000180000001800000018000000180000009B
:109570001800000018000000380000007000000013
:10958000E00000003000000018000000180000009B
:10959000180000001800000018000000180000006B
:1095A000180000001C0000000E0000000000000079
:1095B00000000000000000000000000000000000AB
:1095C000000000003000000030000000300000000B
:1095D00030000000300000003000000030000000CB
:1095E00030000000300000003000000030000000BB
:1095F00030000000300000003000000030000000AB
:10960000300000003000000030000000300000009A
:1096100030000000300000003000000000000000BA
:10962000000000000000000000000000000000003A
:10963000000000007000000078000000180000002A
:1096400018000000180000001800000018000000BA
:10965000180000001C0000000C00000007000000C3
:10966000070000000C0000001C00000018000000B3
:10967000180000001800000018000000180000008A
:109680001800000018000000780000000000000032
:1096900000000000000000000000000000000000CA
:1096A000000000003E0800007FF8000041F00000CC
:1096B00000000000000000000000000000000000AA
:1096C000000000000000000000000000000000009A
:1096D000000000000000000000000000000000008A
:1096E000000000000000000000000000000000007A
:1096F000000000000000000000000000070707074E
:1097000007070707070707070707070707070707E9
:109710000707070707070707070707070707090ED0
:109720000E17110E08090A0E070907070E0E0E0D77
:109730000E0E0E0E0E0E07060E0E0E0E1912111242
:1097400012110F1412070D110E151213101312110E
:1097500010121118111210131212100E080E0E0D05
:109760000E0E090E0E06070D06150E0E0E0E090C36
:10977000080E0D120D0D0D0807090E000100000066
:10978000040000001A0000001C000000240000007B
:1097900000000000000000000000000000000000C9
:1097A00000000000000000000000000000000000B9
:1097B00000000000000000000000000000000000A9
:1097C0000000000000000000000000000000000099
:10A0800000300000300000300000300000300000E0
:10A0900030000030000030000030000030000030A0
:10A0A0000000000000000000000000300000000080
:10A0B00000000000000000000000000000000000A0
:10A0C0000000000000006C00006C00006C00006CE0
:10A0D00000006C0000000000000000000000000014
:10A0E0000000000000000000000000000000000070
:10A0F0000000000000000000000000000000000060
:10A1000000000000000000000000001980000000B6
:10A11000000000000000000F00003FC00030C00041
:10A12000606000606000606000606000606000303F
:10A13000C0003FC0000F0000000000000000000051
:10A14000000000000000000000000000000000000F
:10A150001980000000000000000000001F00003B0C
:10A16000800060C00000C0001FC00038C00060C098
:10A170000060C00060C0003FC0001EC000000000C2
:10A1800000000000000000000000000000000000CF
:10A1900000000000001C08003E1000631000632057
:10A1A000006320007640003E4000009E00009200C8
:10A1B000013300013300023300023300041E000C9F
:10A1C0001E00000000000000000000000000000071
:10A1D000000000000000000000000700000F8000E9
:10A1E00018C00018C00019C0000F80000F00001F29
:10A1F000000033300061B00060F00060E00070608B
:10A20000003FF0001F1000000000000000000000F0
:10A21000000000000000000000000000000000330B
:10A22000000000000000000000000060C00060C0EE
:10A230000060C00060C00060C00060C00060C0007E
:10A2400060C00061C0003FC0001EC00000000000F0
:10A2500000000000000000000000000000000000FE
:10A26000000000000C00001800001000003000008A
:10A27000300000200000600000600000600000600E
:10A28000000060000060000060000020000030005E
:10A29000003000001000001800000C00000000005A
:10A2A00000000000000000000060000020000030FE
:10A2B00000001000001800001800000C00000C0046
:10A2C000000C00000C00000C00000C00000C000052
:10A2D0001800001800001800003000002000006086
:10A2E0000000000000000000000000000000180056
:10A2F000001000007E00003800003C000024000038
:10A30000000000000000000000000000000000004D
:10A31000000000000000000000000000000000003D
:10A32000000000000000000000000000000000002D
:10A330000000000000000000000000000600000611
:10A3400000000600000600007FC0000600000600B6
:10A3500000060000060000060000000000000000EB
:10A3600000000000000000000000000000000000ED
:10A3700000000000000000000000000000000000DD
:10A3800000000000000000000000000000000000CD
:10A3900000000000000000000000000000000000BD
:10A3A000000030000010000010000020000000003D
:10A3B000000000000000000000000000000000009D
:10A3C000000000000000000000000000000000008D
:10A3D00000000000000000007C0000000000000001
:10A3E000000000000000000000000000000000006D
:10A3F000000000000000000000000000000000005D
:10A40000000000000000000000000000000000004C
:10A41000000000000000000000000000000000003C
:10A4200000000000000000000000000030000000FC
:10A43000000000000000000000000000000000001C
:10A4400000000000000000080000080000180000E4
:10A450001800001000001000003000002000002054
:10A460000000200000600000400000400000C0002C
:10A4700000C000000000000000000000000000001C
:10A480000000000000000000000000000E00003F7F
:10A49000800031800060C00060C00060C00060C00B
:10A4A0000060C00060C00060C00060C00060C0000C
:10A4B0003180003F80000E0000000000000000001E
:10A4C000000000000000000000000000000000008C
:10A4D000000300000300000700001F00000300004D
:10A4E000030000030000030000030000030000035A
:10A4F0000000030000030000030000030000000050
:10A50000000000000000000000000000000000004B
:10A510000000000000000F80001FC00030E000308D
:10A52000600000600000600000C00001C000038007
:10A53000000700000E00001800003000007000004E
:10A540007FE00000000000000000000000000000AC
:10A5500000000000000000000000001F00003F801D
:10A560000060C00020C00000C000018000070000A3
:10A5700003800000C00000C00000C00060C0006197
:10A5800080003F80001F000000000000000000006D
:10A5900000000000000000000000000000000000BB
:10A5A0000180000180000380000780000580000D0D
:10A5B00080001980001180003180006180007FE000
:10A5C0000001800001800001800001800000000087
:10A5D000000000000000000000000000000000007B
:10A5E00000000000003F800070000060000060007C
:10A5F000006000007F000073800041800000C00008
:10A6000000C00000C00040C0006180007F00001E4C
:10A61000000000000000000000000000000000003A
:10A62000000000000000000000000F00001F80007C
:10A6300030C0002000006000006F00007B800060E0
:10A64000C00060C00060C00060C00060C000318019
:10A65000001F80000F00000000000000000000004C
:10A660000000000000000000000000000000007F6B
:10A67000C00000C00000C000018000018000010097
:10A6800000030000030000060000060000060000B2
:10A690000C00000C00000800001800000000000082
:10A6A00000000000000000000000000000000000AA
:10A6B000000000000F00001F800030C00030C0000C
:10A6C00030C0001980001F00000F000039800060BA
:10A6D000C00060C00060C00060C0003F80001F007C
:10A6E000000000000000000000000000000000006A
:10A6F0000000000000000000001E00003F000031CC
:10A70000800060C00060C00060C00060C00031C058
:10A71000001EC00000C00000C0006080002180005A
:10A720003F00001E000000000000000000000000CC
:10A730000000000000000000000000000000000019
:10A7400000000000000000000000300000000000D9
:10A7500000000000000000000000000000000000F9
:10A7600000000000000000003000000000000000B9
:10A7700000000000000000000000000000000000D9
:10A780000000000000000000000000000000003099
:10A7900000000000000000000000000000000000B9
:10A7A0000000000000000000000000000030000079
:10A7B0001000001000002000000000000000000059
:10A7C0000000000000000000000000000000000089
:10A7D0000000600003C0000F00003C00007000009B
:10A7E0007800001E000007C00000E000000000002C
:10A7F0000000000000000000000000000000000059
:10A800000000000000000000000000000000000048
:10A810000000000000000000007FC00000000000F9
:10A8200000000000000000007FC0000000000000E9
:10A830000000000000000000000000000000000018
:10A840000000000000000000000000000000000008
:10A850000000000000000000000000600000780020
:10A86000001F000003C00000E00001C0000F000056
:10A870003C0000700000000000000000000000002C
:10A8800000000000000000000000000000000000C8
:10A89000000000000000000F00001FC00030E000BA
:10A8A00060600000600000600000C00001800003E4
:10A8B0000000060000060000060000000000000086
:10A8C0000006000000000000000000000000000082
:10A8D00000000000000000000000000001FC000774
:10A8E000FF000E03801C01C038F4C031FC60330C43
:10A8F00060630C60660C60660C606608606618C079
:10A900006618C033FF8031CE001800001C0000071D
:10A91000FE0001FC0000000000000000000000003C
:10A92000000700000700000700000D80000D8000F8
:10A9300018C00018C00018C0003060003FE0003FA1
:10A94000F000603000603000601800C018000000A7
:10A9500000000000000000000000000000000000F7
:10A960000000000000003FC00031E0003030003047
:10A9700030003030003030003060003FC0003070B8
:10A980000030180030180030180030380030F00067
:10A990003FC00000000000000000000000000000B8
:10A9A000000000000000000000000007C0001FF0D1
:10A9B00000383800301800600800600000600000B7
:10A9C000600000600000600000600800301800387F
:10A9D00038001FF00007C000000000000000000069
:10A9E0000000000000000000000000000000000067
:10A9F0003FC00031F000303800301800300C00301B
:10AA00000C00300C00300C00300C00300C00300812
:10AA10000030180030380031F0003FC00000000066
:10AA20000000000000000000000000000000000026
:10AA300000000000003FF80030000030000030004F
:10AA4000003000003000003000003FF00030000017
:10AA50003000003000003000003000003000003FC7
:10AA6000F8000000000000000000000000000000EE
:10AA7000000000000000000000003FF00030000077
:10AA80003000003000003000003000003000003F97
:10AA9000E0003000003000003000003000003000E6
:10AAA0000030000030000000000000000000000046
:10AAB000000000000000000000000000000000078F
:10AAC000E0001FF000181800300C0060000060006B
:10AAD0000060000060FC00600C00600C00600C0076
:10AAE000300C00181C001FFC0007CC000000000008
:10AAF0000000000000000000000000000000000056
:10AB00000000000030180030180030180030180025
:10AB10003018003018003018003FF80030180030AE
:10AB200018003018003018003018003018003018A5
:10AB30000000000000000000000000000000000015
:10AB40000000000000000000003000003000003075
:10AB50000000300000300000300000300000300005
:10AB600000300000300000300000300000300000F5
:10AB70003000003000000000000000000000000075
:10AB80000000000000000000000000000000018044
:10AB90000001800001800001800001800001800030
:10ABA00001800001800001800001800001800061BF
:10ABB00080006180003F00001E00000000000000D7
:10ABC0000000000000000000000000000000000085
:10ABD00000000030380030700030600030C00031BC
:10ABE00080003300003700003F000039800031C092
:10ABF0000030E00030600030700030380030180065
:10AC00000000000000000000000000000000000044
:10AC100000000000000000003000003000003000A4
:10AC20000030000030000030000030000030000034
:10AC30003000003000003000003000003000003FE5
:10AC4000E0003FE000000000000000000000000005
:10AC500000000000000000000000000000380700B5
:10AC6000380F003C0F003C0F00341B00361B003631
:10AC70001B0032130033330033330031230031E340
:10AC80000031E30030C30030C300000000000000CA
:10AC900000000000000000000000000000000000B4
:10ACA00000003018003818003C18003C1800361816
:10ACB0000036180033180033980031980030D8005F
:10ACC00030D800307800307800303800301800007C
:10ACD0000000000000000000000000000000000074
:10ACE0000000000000000007E0000FF0001818004E
:10ACF000300C00600C00600600600600600600601A
:10AD00000600600600600C00300C001818000FF000
:10AD10000007E0000000000000000000000000004C
:10AD20000000000000000000000000003FE00030D4
:10AD3000F0003030003018003018003018003018A3
:10AD4000003070003FE000300000300000300000B4
:10AD50003000003000003000000000000000000063
:10AD600000000000000000000000000000000000E3
:10AD70000007E0000FF000181800300C00600C0015
:10AD80006006006006006006006006006006006065
:10AD90000C00306C001838000FFC0007EE000004B7
:10ADA00000000000000000000000000000000000A3
:10ADB0000000000000003FE00030F00030180030DC
:10ADC00018003018003018003030003FE00030E04C
:10ADD0000030700030300030300030180030180083
:10ADE000301800000000000000000000000000001B
:10ADF00000000000000000000000000F80003FC0C5
:10AE0000006060006060006000007000003F0000B3
:10AE10000FC00001E00000700040300060300060B2
:10AE200060003DE0001F8000000000000000000006
:10AE30000000000000000000000000000000000012
:10AE40007FF0000300000300000300000300000384
:10AE500000000300000300000300000300000300E3
:10AE600000030000030000030000030000000000D6
:10AE700000000000000000000000000000000000D2
:10AE800000000000003018003018003018003018A2
:10AE9000003018003018003018003018003018004A
:10AEA0003018003018003018001830001FF000076C
:10AEB000C0000000000000000000000000000000D2
:10AEC00000000000000000000000C0180060180032
:10AED00060300060300030300030600010600018DA
:10AEE000400018C00008C0000D80000D80000780E1
:10AEF0000007000003000000000000000000000048
:10AF0000000000000000000000000000000000C081
:10AF1000E06060E0C060E0C061B0C061B08031B1AD
:10AF200080311180331980331900121B001A0B0075
:10AF30001E0F000E0E000C06000C060000000000A4
:10AF40000000000000000000000000000000000001
:10AF50000000000060300030700038600018C00051
:10AF60000DC0000F80000700000700000780000DE3
:10AF7000800018C000186000306000603000E018E9
:10AF800000000000000000000000000000000000C1
:10AF90000000000000000000006018007038003061
:10AFA000300018600018E0000CC000078000078027
:10AFB0000003000003000003000003000003000082
:10AFC000030000030000000000000000000000007B
:10AFD00000000000000000000000000000003FF042
:10AFE0000000700000600000E00000C00001800070
:10AFF0000300000700000600000C00001C000038E1
:10B0000000003000007000007FF000000000000031
:10B0100000000000000000000000066000000000CA
:10B0200000000007E0000FF000181800300C00606E
:10B030000C00600600600600600600600600600606
:10B0400000600C00300C001818000FF00007E00042
:10B050000000000000000000000000000000000CE4
:10B06000C00000000000000003000007800007800F
:10B07000000C80000CC0000CC000186000186000BC
:10B080001060003FF0003FF00060180060180060A2
:10B090001800C00C000000000000000000000000CC
:10B0A0000000000006C00000000000000030180092
:10B0B00030180030180030180030180030180030F8
:10B0C0001800301800301800301800301800301800
:10B0D000001830001FF00007C00000000000000052
:10B0E0000000000000000000000000000000000060
:10B0F00000001E00003F80006180006180006180D0
:10B100000063000063000063000063800061C00012
:10B1100060600060600064600067C00063800000E1
:10B12000000000000000000000000000000000001F
:10B13000000000000000000000000000000000000F
:10B1400000000000000000000000000000000000FF
:10B1500000000000000000000000000000000000EF
:10B1600000000000000000000000FFE00000000000
:10B17000000000000000000000000000600000303F
:10B1800000001000000000000000000000000000AF
:10B1900000000000000000000000000000000000AF
:10B1A000000000000000000000000000000000009F
:10B1B000000000000000000000000000000000008F
:10B1C000000000000000000000000000001F000060
:10B1D0003B800060C00000C0001FC00038C000609D
:10B1E000C00060C00060C0003FC0001EC000000082
:10B1F000000000000000000000000000000000004F
:10B2000000000000000060000060000060000060BE
:10B2100000006F00007F800071800060C00060C08F
:10B220000060C00060C00060C0006180007F8000DE
:10B230006F0000000000000000000000000000009F
:10B2400000000000000000000000000000000000FE
:10B25000000000000000000F00003F800030C00030
:10B2600060000060000060000060000060000030CE
:10B27000C0003F80000F0000000000000000000040
:10B2800000000000000000000000000000000000BE
:10B2900000C00000C00000C00000C0001EC0003F91
:10B2A000C00030C00060C00060C00060C00060C06E
:10B2B0000060C00031C0003FC0001EC000000000A0
:10B2C000000000000000000000000000000000007E
:10B2D000000000000000000000000000000000006E
:10B2E000000F00003F800020C00060C0007FC00051
:10B2F00060000060000060400030C0003F80000F30
:10B30000000000000000000000000000000000003D
:10B31000000000000000000000001E00003E0000D1
:10B320003000003000007C000030000030000030B1
:10B33000000030000030000030000030000030001D
:10B34000003000003000000000000000000000009D
:10B3500000000000000000000000000000000000ED
:10B3600000000000000000000000001EC0003FC000
:10B370000030C00060C00060C00060C00060C0005D
:10B3800060C00031C0003FC0001EC00000C00060AF
:10B39000C0003F80001F000000000000000000000F
:10B3A000000000006000006000006000006000001D
:10B3B0006F00007F800070C00060C00060C000604F
:10B3C000C00060C00060C00060C00060C00060C01D
:10B3D000000000000000000000000000000000006D
:10B3E00000000000000000000060000000000000FD
:10B3F00000000000006000006000006000006000CD
:10B40000006000006000006000006000006000005C
:10B41000600000600000000000000000000000006C
:10B4200000000000000000000000000000006000BC
:10B43000000000000000000000006000006000004C
:10B4400060000060000060000060000060000060BC
:10B45000000060000060000060000060000060000C
:10B4600000E00000C000000000000000000000003C
:10B4700000000060000060000060000060000063E9
:10B4800080006300006600006C00007C00007C000F
:10B4900000660000660000630000618000618000BB
:10B4A000000000000000000000000000000000009C
:10B4B000000000000000000060000060000060006C
:10B4C000006000006000006000006000006000009C
:10B4D000600000600000600000600000600000602C
:10B4E00000006000000000000000000000000000FC
:10B4F000000000000000000000000000000000004C
:10B500000000000000000000006F3C007FFE0071A2
:10B51000C6006186006186006186006186006186E2
:10B520000061860061860061860000000000000066
:10B53000000000000000000000000000000000000B
:10B5400000000000000000000000000000006F008C
:10B55000007F800070C00060C00060C00060C0005C
:10B5600060C00060C00060C00060C00060C000003B
:10B5700000000000000000000000000000000000CB
:10B5800000000000000000000000000000000000BB
:10B590000000000F00003FC00030C000606000608D
:10B5A000600060600060600060600030C0003FC00C
:10B5B000000F00000000000000000000000000007C
:10B5C000000000000000000000000000000000007B
:10B5D00000000000000000006F00007F800071800C
:10B5E0000060C00060C00060C00060C00060C000BB
:10B5F0006180007F80006F000060000060000060DC
:10B6000000006000000000000000000000000000DA
:10B61000000000000000000000000000001EC0004C
:10B620003FC00030C00060C00060C00060C000606B
:10B63000C00060C00031C0003FC0001EC00000C09C
:10B640000000C00000C00000C000000000000000BA
:10B6500000000000000000000000000000000000EA
:10B6600000006E00007C00006000006000006000D0
:10B6700000600000600000600000600000600000EA
:10B68000600000000000000000000000000000005A
:10B6900000000000000000000000000000000000AA
:10B6A000000000000000001F00007F80006180009B
:10B6B0006000007C00001F800003C00000C000602C
:10B6C000C0003F80001F00000000000000000000DC
:10B6D000000000000000000000000000000000006A
:10B6E0000000001000003000003000007C0000303E
:10B6F000000030000030000030000030000030005A
:10B70000003000003000003C00001C000000000081
:10B710000000000000000000000000000000000029
:10B720000000000000000000000000000000000019
:10B730000060C00060C00060C00060C00060C00069
:10B7400060C00060C00060C00061C0003FC0001E5B
:10B75000C000000000000000000000000000000029
:10B7600000000000000000000000000000000000D9
:10B77000000000000000C0C0006180006180002166
:10B7800000003300003300001200001E00001E0005
:10B79000000C00000C000000000000000000000091
:10B7A0000000000000000000000000000000000099
:10B7B0000000000000000000000000C30C00430C6B
:10B7C00000638C0067880066980026D80034D0009B
:10B7D0003CF0001C700018700018600000000000B1
:10B7E0000000000000000000000000000000000059
:10B7F0000000000000000000000000000000000049
:10B800006180007380003300001E00001E00000CE9
:10B8100000001E00003F0000330000618000E1C016
:10B820000000000000000000000000000000000018
:10B830000000000000000000000000000000000008
:10B840000000000000C08000618000618000610095
:10B85000003300003300001200001E00001E000034
:10B860000C00000C000008000018000078000070B8
:10B8700000000000000000000000000000000000C8
:10B88000000000000000000000003FC00001C000F8
:10B890000180000300000700000E00000C000018EB
:10B8A00000003800007800007FC0000000000000A9
:10B8B0000000000000000000000000000000000088
:10B8C0000000000E00001C00001800001800001806
:10B8D0000000180000180000180000300000600090
:10B8E00000300000180000180000180000180000C8
:10B8F0001800001800001C00000E000000000000EE
:10B9000000000000000000003000003000003000A7
:10B910000030000030000030000030000030000037
:10B9200030000030000030000030000030000030F7
:10B930000000300000300000300000300000300017
:10B940000000000000000000000000000070000087
:10B9500070000018000018000018000018000018FF
:10B9600000001800000C00000600000C0000180089
:10B97000001800001800001800001800001800004F
:10B980003000007000000000000000000000000017
:10B9900000007C20007FE0000000000000000000AC
:10B9A0000000000000000000000000000000000097
:10B9B0000000000000000000000000000000000087
:10B9C000000000000000000000000005050505055E
:10B9D0000505050505050505050505050505050517
:10B9E00005050505050505050505050506070C0BF7
:10B9F000110D0B0707080B060706060B0C0C0B0CAA
:10BA00000B0B0B0B0B06060C0B0C0C140F0E0E0F76
:10BA10000E0C0F0F060A0E0C110F100E100E0D0D4E
:10BA20000F0E130E0E0D100F0F0C0B070B0B0A0B46
:10BA30000B070B0B04050A04100B0C0B0B070B0771
:10BA40000B0A0F0A0A0B0706080C0001000000038E
:10BA500000000014000000170000004F000000006C
:10BA600011241FBECFEFCDBFDFE3DEBF00E00CBF70
:10BA700018BE19BE1ABE1BBE11E2A0E0B0E2EEEC89
:10BA8000F3EF01E00BBF02C007900D92A438B1079D
:10BA9000D9F71BBE22E2A4E8B1E201C01D92AC3E80
:10BAA000B207E1F70E94B5E50C94E5F90C940000AB
:10BAB000AF92CF92EF920F93A12CCC24C394E12CA0
:10BAC00000E020E040EA56E060EC7BE08FE692E2A6
:10BAD0000E94FDEC0F91EF90CF90AF900895CF9220
:10BAE000DF92EF92FF921F93CF93DF936B017C0164
:10BAF000C0EAD6E010E11E8363E08FE692E20E9486
:10BB00002FEDB701882799278FE692E20E942FED4B
:10BB100099278F2D7E2D6D2D8FE692E20E942FEDBD
:10BB20006C2D8FE692E20E942FED60E08FE692E2AC
:10BB30000E942FED1D83DF91CF911F91FF90EF9019
:10BB4000DF90CF9008950F931F93CF93DF93C0EAB8
:10BB5000D6E010E11E8365E08FE692E20E942FEDB1
:10BB600060E08FE692E20E942FED082F60E08FE602
:10BB700092E20E942FED1D83802FDF91CF911F91C4
:10BB80000F910895CF92DF92EF92FF92CF93DF93C0
:10BB90006B017C01D42FC0E1C093A60662E08FE662
:10BBA00092E20E942FEDB701882799278FE692E253
:10BBB0000E942FED99278F2D7E2D6D2D8FE692E21D
:10BBC0000E942FED6C2D8FE692E20E942FED6D2FDB
:10BBD0008FE692E20E942FEDC093A506B4DF80FDB0
:10BBE000FDCFDF91CF91FF90EF90DF90CF90089540
:10BBF000CF93DF93C82F80E18093A606C130D9F19F
:10BC000066E08FE692E20E942FED80E18093A50628
:10BC10009ADF80FDFDCFC130D1F110928421D0E1B7
:10BC2000D093A60661E08FE692E20E942FED8FE3AB
:10BC30009FE10197F1F700C00000609184218FE639
:10BC400092E20E942FEDD093A5067DDF80FDFDCF0F
:10BC500080E18093A606C130A1F066E08FE692E213
:10BC60000E942FED80E18093A5066DDF80FDFDCF62
:10BC7000DF91CF91089564E08FE692E20E942FED6C
:10BC8000C4CF64E08FE692E20E942FEDEBCF80E814
:10BC900080938421C4CFCF9380E0AADF2FEF83EC81
:10BCA00099E0215080409040E1F700C000004BDF58
:10BCB0008093762248DF80FDFDCFC0E1C093A606C9
:10BCC00060E68FE692E20E942FEDC093A5063BDF6F
:10BCD00080FDFDCFCF9108954F925F926F927F923A
:10BCE0008F929F92AF92BF92CF92DF92EF92FF928C
:10BCF000CF93F82E80E07CDF2FEF83EC99E021508A
:10BD000080409040E1F700C000001DDF8093762264
:10BD1000FA942F2D30E0AFEFBFEF0E94BDF96B0119
:10BD20007C012FEFC21AD20AE20AF20A8D2C9E2C55
:10BD3000AF2CBB2427016624772405DF80FDFDCFCF
:10BD4000C0E1C093A60668ED8FE692E20E942FED57
:10BD5000642D8FE692E20E942FED682D8FE692E22D
:10BD60000E942FED6C2D8FE692E20E942FEDC09382
:10BD7000A506E9DE80FDFDCFCF91FF90EF90DF902B
:10BD8000CF90BF90AF909F908F907F906F905F907B
:10BD90004F9008958F929F92AF92BF92CF92DF9271
:10BDA000EF92FF92CF937C0180E022DFCCDE809384
:10BDB0007622C701A0E0B0E02CE0880F991FAA1FEF
:10BDC000BB1F2A95D1F7892E9A2EAB2EBB246D016D
:10BDD000EE24FF24B8DE80FDFDCFC0E1C093A606AF
:10BDE00060E28FE692E20E942FED6C2D8FE692E2E8
:10BDF0000E942FED682D8FE692E20E942FED60E009
:10BE00008FE692E20E942FEDC093A5069CDE80FD96
:10BE1000FDCFCF91FF90EF90DF90CF90BF90AF908C
:10BE20009F908F90089590E19093A606813061F0E5
:10BE300066E08FE692E20E942FED80E18093A506F6
:10BE400082DE80FDFDCF089564E08FE692E20E94DD
:10BE50002FEDF3CF86E38093CA01EF93FF930F9307
:10BE60002F93EBECF1E008ED21E004BF20832F914C
:10BE70000F91FF91EF9108951F93CF93DF93C82FF8
:10BE8000D62F142F8091CF0187FDFCCF8091CF0159
:10BE900081FDE0DF83E38093CA0120E2C29FC001FD
:10BEA0001124DF718D2B8093C0019093C1011092FA
:10BEB000C2011093C40185E38093CA01EF93FF93FD
:10BEC0000F932F93EBECF1E008ED21E004BF20830A
:10BED0002F910F91FF91EF91DF91CF911F910895D5
:10BEE0009091CF0197FDFCCF20E2829FC0011124E9
:10BEF0006F71862B8093C0019093C1011092C20193
:10BF000086E08093CA01EF93FF930F932F93EBEC9E
:10BF1000F1E008ED21E004BF20832F910F91FF9104
:10BF2000EF918091C4010895109260081092610809
:10BF300067E080E498E00E9441ED789408958130B4
:10BF400029F0823011F480936506089582E0809391
:10BF50006606089591E090939C229091A10995FF27
:10BF6000FCCF8093A00980919C228130E1F3089559
:10BF7000E0E6F6E088E0818384E08283E0EAF9E0AD
:10BF800083E085838381806383832FEF89EF90E053
:10BF9000215080409040E1F700C0000083818C6018
:10BFA00083838FEC8683178284818061848384817C
:10BFB00088608483089582E0809365068FE79EE31E
:10BFC0000197F1F700C0000081E080939C228091EE
:10BFD000A10985FFFCCF8FEF8093A00980919C225F
:10BFE0008130E1F382E0809366069FEF29EF30E035
:10BFF000915020403040E1F700C00000809365067A
:10C000008FE79EE30197F1F700C0000081E0809385
:10C010009C228091A10985FFFCCF8FEF8093A0091E
:10C0200080919C228130E1F382E08093660608953E
:10C0300092E090936506EFE7FEE33197F1F700C0D9
:10C04000000091E090939C229091A10995FFFCCF74
:10C0500097E99093A00990919C229130E1F391E0AF
:10C0600090939C229091A10995FFFCCF95E090932D
:10C07000A00990919C229130E1F391E090939C2251
:10C080009091A10995FFFCCF92E09093A009909127
:10C090009C229130E1F392E090936606FFEF2AEA4A
:10C0A00039E0F15020403040E1F700C000009093AB
:10C0B0006506EFEBFDE53197F1F700C0000091E078
:10C0C00090939C229091A10995FFFCCF8093A009A9
:10C0D00080919C228130E1F381E080939C228091C9
:10C0E000A10985FFFCCF6093A00980919C2281303B
:10C0F000E1F381E080939C228091A10985FFFCCF30
:10C100004093A00980919C228130E1F382E08093EA
:10C110006606FFEF23EF31E0F15020403040E1F7B9
:10C1200000C00000809365068FE79EE30197F1F75A
:10C1300000C0000081E080939C228091A10985FFCE
:10C14000FCCF8FEF8093A00980919C228130E1F396
:10C1500082E080936606089592E090936506EFE78B
:10C16000FEE33197F1F700C0000091E090939C222C
:10C170009091A10995FFFCCF98EC9093A009909124
:10C180009C229130E1F391E090939C229091A1093F
:10C1900095FFFCCF4093A00990919C229130E1F350
:10C1A00091E090939C229091A10995FFFCCF809300
:10C1B000A00980919C228130E1F381E080939C2250
:10C1C0008091A10985FFFCCF6093A00980919C22FA
:10C1D0008130E1F381E080939C228091A10985FF69
:10C1E000FCCF8DE08093A00980919C228130E1F307
:10C1F00082E0809366068FE39FE10197F1F700C02C
:10C2000000000895CF9392E090936506EFE7FEE378
:10C210003197F1F700C0000091E090939C2290913B
:10C22000A10995FFFCCF97E99093A00990919C22DA
:10C230009130E1F391E090939C229091A10995FFB8
:10C24000FCCF95E09093A00990919C229130E1F36E
:10C2500091E090939C229091A10995FFFCCF93E0EF
:10C260009093A00990919C229130E1F392E09093F9
:10C270006606FFEF23EF31E0F15020403040E1F758
:10C2800000C0000090936506EFEBFDE53197F1F7F4
:10C2900000C0000091E090939C229091A10995FF2D
:10C2A000FCCF8093A00980919C228130E1F3C2E011
:10C2B000C093660639DE1092B622C0938A22CF91CF
:10C2C0000895E0E4F8E010A211A28FEF95E186A3B3
:10C2D00097A360E080E498E00E9441ED61E080E493
:10C2E00098E00E944DED789408951F920F920FB63A
:10C2F0000F92112408B60F9218BE10929C220F9034
:10C3000008BE0F900FBE0F901F9018951F920F92AE
:10C310000FB60F92112408B60F9218BE09B60F92ED
:10C3200019BE0BB60F921BBE2F933F934F935F9393
:10C330006F937F938F939F93AF93BF93EF93FF93ED
:10C34000F3DD809185218A3010F010928521809153
:10C3500085218F5F80938521E09185218091A009BF
:10C36000F0E0E958FD4D8083809178228F3F09F4F9
:10C3700086C0E0918521F0E0E958FD4D80818F3F36
:10C3800009F445C0809185218230B9F0FF91EF9189
:10C39000BF91AF919F918F917F916F915F914F91DD
:10C3A0003F912F910F900BBE0F9009BE0F9008BECA
:10C3B0000F900FBE0F901F90189580918A228230A7
:10C3C00029F760E080E498E00E9441EDE09185214A
:10C3D000F0E0EA58FD4D80818093AB22E091852109
:10C3E000F0E0E958FD4D80818093A022E7E7F2E27A
:10C3F000119282E2E138F807D9F710928A2210925E
:10C40000852181E080938A228093B622BFCF8091DC
:10C410008521823008F4B6CFE0918521F0E0EC5818
:10C42000FD4D8081873D09F0ADCFE0918521F0E0A1
:10C43000ED58FD4D8081873D09F0A4CFE091852125
:10C44000F0E0EB58FD4D808180934322E0918521FF
:10C45000F0E0EA58FD4D808180934222E7E7F2E266
:10C46000119282E2E138F807D9F710928A221092ED
:10C47000852160E080E498E00E9441ED83CF60E098
:10C4800080E498E00E9441EDE7E7F2E281E892E281
:10C4900011928E179F07E1F710928A221092852140
:10C4A00010928A2273CF1F920F920FB60F9211240F
:10C4B00008B60F9218BE09B60F9219BE0BB60F92AE
:10C4C0001BBE2F933F934F935F936F937F938F93F5
:10C4D0009F93AF93BF93EF93FF93109260081092D6
:10C4E0006108E7E7F2E2119282E2E138F807D9F752
:10C4F00010928A221092852160E080E498E00E94E8
:10C5000041EDFF91EF91BF91AF919F918F917F91FD
:10C510006F915F914F913F912F910F900BBE0F90B4
:10C5200009BE0F9008BE0F900FBE0F901F90189578
:10C530009091CE212091BD21911103C02F3009F49B
:10C540009EC03091C621931708F43FC04091C72187
:10C550009417D8F54091CC21442309F496C0482F74
:10C5600050E0692F631B02C0440F551F6A95E2F724
:10C570006091A1217091A221462B572B4093A121BC
:10C580005093A221223009F444C02C3109F441C057
:10C590002330B9F42FEE290F243098F4282F30E0FF
:10C5A0008FEE890F02C0220F331F8A95E2F7409168
:10C5B000952150919621242B352B20939521309352
:10C5C00096219F5F9093CE2108953091C8219317B3
:10C5D000C8F24091C9219417A8F64091CC21442378
:10C5E00009F45FC0293209F468C0482F50E0692F70
:10C5F000631B02C0440F551F6A95E2F760919F21AB
:10C600007091A021462B572B40939F215093A0213E
:10C61000B9CF983030F54091992150919A21440F2B
:10C62000551F482B4093992150939A212C3109F0A2
:10C63000AFCF23EF290F2D3020F6282F30E083EFE6
:10C64000890F02C0220F331F8A95E2F740919D2186
:10C6500050919E21242B352B20939D2130939E2198
:10C66000B0CF983118F74091972150919821440FFD
:10C67000551F482B4093972150939821D7CF8093F3
:10C68000CF219F5F9093CE2108954091A121509199
:10C69000A221440F551F482B4093A1215093A22162
:10C6A00071CF40919F215091A021440F551F482BDD
:10C6B00040939F215093A02165CF903208F495CFED
:10C6C000282F30E080EE6DCF9091BD212091CE21BA
:10C6D000992311F0225001C021503091B521231728
:10C6E000B0F09091B621291790F490E0231B02C07E
:10C6F000880F991F2A95E2F720919D2130919E2164
:10C70000822B932B80939D2190939E2108953091AD
:10C71000B7212317A8F09091B821291788F490E049
:10C72000231B02C0880F991F2A95E2F720919B21B5
:10C7300030919C21822B932B80939B2190939C2161
:10C740000895E0E2F6E084818F77848380818F779B
:10C7500080830895CF93DF93EC018091AB218823F0
:10C7600089F1E091AA218E2F90E0FC013297E83206
:10C77000F10510F18091AA2188838091A8219091E0
:10C78000A92189839A838091A6219091A7218B83E7
:10C790009C838091A3218D831092A6211092A721C2
:10C7A0001092A8211092A9211092A32181E0109249
:10C7B000AB21DF91CF9108958827E250FF4F8F4F33
:10C7C0000C94B4F980E0DF91CF9108952091A621D7
:10C7D0003091A7218091A4219091A521982F88279D
:10C7E000822B8093A6219093A721C4CF2091A621CC
:10C7F0003091A7218091A6219091A721232F332743
:10C800008095909599272817390709F4C9C080E0C9
:10C81000CECF8091A6219091A72194FFF8CF80914F
:10C82000A6219091A7218F719927459709F4C2C03D
:10C830008091A6219091A7218F719927409739F770
:10C840008091A6219091A7219695879592958295A2
:10C850008F7089279F7089278093A6219093A721A5
:10C860008091A6219091A72180688093A621909322
:10C87000A72180CF8091A6219091A721892B09F033
:10C8800079CF80E094CF8091A6219091A7218D3718
:10C89000910509F06FCF80E08ACF2091A6213091D9
:10C8A000A7218091A6219091A7212695217031E0A2
:10C8B00023278170992731E083278170281709F495
:10C8C000A6CF8091A6219091A721969587958093D8
:10C8D000A6219093A7214ECF8091A8219091A921C4
:10C8E0008F7D8093A8219093A92144CF2091A621E8
:10C8F0003091A7218091A6219091A721232F332742
:10C900008095909599272817390709F080CF809155
:10C91000A6219091A72199278093A6219093A721E2
:10C920008091A4219091A5212091A6213091A72149
:10C93000982F8827822B932B8093A6219093A72151
:10C9400019CF2091A6213091A7218091A621909105
:10C95000A721232F332780959095992728173907EA
:10C96000F9F08091A8219091A9218E3E974809F075
:10C970004ECF8BE08093AA218091A6219091A72190
:10C98000892F99278093A8219093A9218091A6218E
:10C990009091A72199278093A6219093A721EACE71
:10C9A0008091A6219091A72199278093A621909309
:10C9B000A721E0CE8091A6219091A72196958795F9
:10C9C000929582958F7089279F7089278093A621E1
:10C9D0009093A7218091A6219091A7218F779927E5
:10C9E0008093A6219093A721C5CE0F931F93CF9339
:10C9F000DF93809128069091AB2191113AC0807805
:10CA0000C09194219C2FC1113BC0882309F428C1F7
:10CA1000809193218111A0C180918C2190918D21D1
:10CA20008F3F2FEF920729F1019680938C219093ED
:10CA30008D2180910420909105208F3F6FEF960704
:10CA4000C1F001968093042090930520883E924087
:10CA500080F080918A2190918B21892B51F0109246
:10CA60008A2110928B218FEF9FEF80930420909367
:10CA700005208091AB21DF91CF911F910F910895F7
:10CA800020919221222309F1882309F4F5C0809195
:10CA90008F2190919021019680938F2190939021E6
:10CAA000209193212951213108F0D1C18C3B914033
:10CAB00008F44DC18091AA211092942110929321E3
:10CAC00010928F2110929021D4CF9091912199238F
:10CAD00009F436C181116FC13091CD21832F30FF10
:10CAE000B0C2C09193219091BF219C1708F0AFC4B0
:10CAF0009091BD21993029F49091CE21943009F480
:10CB00009BC711E086958170812712DD8091BD2140
:10CB1000893029F48091CE21843009F4A4C7809112
:10CB2000CD218695817004DD8091CD21869581701F
:10CB3000809387219091AC21C0918F21D091902139
:10CB4000923109F411C5C0938821D09389211092A4
:10CB50009121C091942181E080939321CC2309F409
:10CB600088CF2091CA219091CE21921382CF8091BB
:10CB7000CB2181117ECF60910220709103204091E2
:10CB80009F215091A0219A016417750709F47DC374
:10CB9000109286218091BD21813009F43FC38D30F0
:10CBA00009F481C3873209F09FC39091862190FDDB
:10CBB000EFC291E09093AB21E091A121F091A221ED
:10CBC0008093AA21E093A821F093A921823009F44F
:10CBD000C0C49A01873039F480918E21282B20938C
:10CBE0009F213093A0212093A6213093A7218091EB
:10CBF0009521909196218093A4219093A5218091D5
:10CC0000AB218823C1F080919F219091A0216817CA
:10CC1000790709F484C42091A1213091A2212093A5
:10CC200000203093012080930220909303201092E3
:10CC30008C2110928D211092942110929F2110929C
:10CC4000A0211092932110928F2110929021809117
:10CC5000AA21843109F00DCF87E88093932109CF71
:10CC6000809193218F5F809393218091AB21DF91FD
:10CC7000CF911F910F9108951092AC218091932133
:10CC800041EE480F4B30F0F520918F2130919021EB
:10CC90002650310924303105A8F56BE775E041E1F4
:10CCA00050E08DEB91E20E94DCF9C091942110924A
:10CCB000CE218091CD2180FFFFC09091BD21973181
:10CCC000B9F09930A9F02091BF2140918F21509166
:10CCD000902130E02417350730F4220F331F24173A
:10CCE000350708F0A0C490918721992309F437C42F
:10CCF00081E08093932110928F21109290211092C5
:10CD000092212CCF2091AA21243109F4B3C026EA24
:10CD1000280F213508F4A0C02091AA2129EF280F5F
:10CD2000253008F0B9C020918F21309190212351F6
:10CD300031092630310508F0AFC066E275E0AFCFAB
:10CD4000811175C0809193218F5F80939321E09131
:10CD5000CA21F091CE2178C081E080939421809304
:10CD600092211092912110929F211092A021109255
:10CD7000A1211092A2211092952110929621109239
:10CD80009B2110929C2110929D2110929E21109225
:10CD90009721109298211092992110929A218FEF49
:10CDA0008093CE2181E090E080938F219093902119
:10CDB00010928E215ECEE091CA212E2FF091CE21CD
:10CDC0009F2FEF1709F477C240918F215091902146
:10CDD0004F5F5F4F40938F2150939021A091BD21D1
:10CDE000A13009F4F3C28091CD21382F82FF03C016
:10CDF000AA3109F412C3AF3009F453C3A73109F0C3
:10CE0000C0C06091CB216111BCC06091C12170E0B4
:10CE1000660F771F4617570708F478C5FF30A0F054
:10CE200081E18093CA2181E08093CB2157CE81E0BC
:10CE30008093912181E090E080938F2190939021C5
:10CE4000E091CA21F091CE212E2F9F2F8ECE8A3EC7
:10CE5000910508F02FCE7BCF20918F21309190212A
:10CE6000B9016C5271096932710508F06AC068E451
:10CE700075E015CF20EB280F2F3608F048CF209112
:10CE80008F21309190212A5331092C36310508F039
:10CE90003ECF6AE675E003CF21E5280F2A3208F578
:10CEA00020918F2130919021285231092C30310569
:10CEB000C0F461EC73E0F3CE82FD1ACF8091BD2106
:10CEC000883009F40DC38E3109F012CF80918F2183
:10CED00090919021CC97409708F00AC381E028DB1D
:10CEE00007CF27EE280F213160F420918F21309158
:10CEF000902124543140263A310518F468E374E057
:10CF0000CECE24EC280F203160F420918F21309177
:10CF100090212C5331092031310518F467E375E075
:10CF2000BECE27ED280F2831D0F420918F213091EB
:10CF30009021295231092831310588F465E175E0E5
:10CF4000AECE6B5E7F4F6731710508F015C18091E1
:10CF5000AA21843109F49DCF69E575E0A0CE20EDCA
:10CF6000280F2D3048F520918F21309190212551A7
:10CF700031092730310500F564E075E090CE8091ED
:10CF8000CD2180FF29C06091C12170E0660F771F1D
:10CF90004617570708F10F2F10E06E2F70E0625010
:10CFA000710906171707C4F03091CB21311114C055
:10CFB00091E09093CB2195CD28ED280F2C3078F57A
:10CFC00020918F21309190212E5531092831310542
:10CFD00030F560EB73E063CE4A3E510508F4C5CDF1
:10CFE0006F2F70E04E2F50E04150510964177507C4
:10CFF00009F420C3A23009F442C3AC3109F4B4C32C
:10D00000A93209F0E0C4F03209F446C61092942126
:10D010001092932110928F21109290212ACD5FEFD0
:10D02000580F543008F088C020918F213091902102
:10D03000235631092A31310508F07EC063EF74E0D0
:10D040002ECE32FD39C08091BD21833009F4FBC260
:10D050008C3109F439C38E3009F065C18091932178
:10D0600082508330F8F48091CE21813009F47EC65D
:10D07000833109F48BC680918F21909190219C017E
:10D080002E5731092F31310508F4A6C69C012952CB
:10D0900031092D30310508F4C5C6835591094697ED
:10D0A00008F4B8C61092942110928F21109290210A
:10D0B000C0E051CD109293212091CA219091CE21B0
:10D0C000921708F080C1109193218091BF218117A0
:10D0D000D8F481E02DDA8091BE21181758F3181B7F
:10D0E000109393212091CA219091CE21E9CF081B62
:10D0F000190B00938F21109390219091CE21809154
:10D10000CA21981708F05FC100918F2110919021DA
:10D110008091C12190E08017910708F054C180E010
:10D1200007DA8091C02190E00817190700F71092E4
:10D130008F2110929021E1CF24EF280F243068F145
:10D1400028EE280F273048F19DEF980F953008F012
:10D150003DC220918F2130919021B9016751710911
:10D160006830710530F0295031092530310508F05B
:10D170002DC261ED74E093CD5091AA21543109F094
:10D18000CDCD255031092830310508F482CEC6CDE9
:10D1900010928C2110928D2132CD20918F213091CF
:10D1A0009021B9016C5071096430710528F06C5000
:10D1B00071096730710540F643EE480F4530B0F411
:10D1C000A9014D5051094330510580F441E150E02F
:10D1D00069E474E08CEA91E20E94DCF920918F21ED
:10D1E00030919021809193219091942120938821D6
:10D1F0003093892180518F3008F48BC1205131093F
:10D200002F30310508F485C181E080938721C92F33
:10D21000992309F44CCD62EE74E041CD90918621C2
:10D220009150923008F4B4CF8093AB21E091A121CA
:10D23000F091A2218093AA21823109F0C3CCCA01C6
:10D240008F7099279A01329522952F7023273F706E
:10D250002327892B09F02068CF01880F991F880F99
:10D26000991F88279F70282B392B20939F2130935B
:10D27000A021CF018F7399278093A1219093A221A0
:10D280008093A8219093A921AECCE0918C21F091BC
:10D290008D21E03BF44008F07BCC809186218F5FAC
:10D2A0008093862177CC9091862190FD71CF91E07B
:10D2B0009093AB21BBCF8091CB21813009F084CDFD
:10D2C0008091CD21857061F4809193219091C2214C
:10D2D000891708F49BCE9091C321981708F496CE35
:10D2E0001092CB219E2F43CCE1E0E093AB2188301C
:10D2F00009F094C29A01209530953370E0918A210B
:10D30000F0918B212E173F0709F417C240FD72C11F
:10D3100040938A2150938B21109204201092052073
:10D320001092AB216CCC909193212091BE21921749
:10D33000A0F02091BF21291780F040918F215091BA
:10D3400090212091C02130E04217530730F0209106
:10D35000C12130E024173507A0F52091C221921792
:10D36000A8F02091C321291788F040918F21509176
:10D3700090212091C42130E04217530738F02091CA
:10D38000C52130E02417350708F0B3C4893109F00E
:10D3900089CE9250933008F085CE8091CE2188308E
:10D3A00009F4C7C4863009F4C4C48C3009F07ACEBD
:10D3B00080918F219091902183559109469708F093
:10D3C00071CE81E0B5D810929121C5CB4C3051057A
:10D3D00008F4D5CDFB3008F4D2CD81E08F0F8093D7
:10D3E000CA218F2F90E00B97982F88272091A12199
:10D3F0003091A221822B932B8093A1219093A22183
:10D400008091C821F80FFF5FF093C9218AE090E076
:10D4100080938F21909390215FCB60E170E06F1B30
:10D4200071098B01000F111F600F711F660F771FAD
:10D43000660F771F4617570708F4A3CD80FF40CE2D
:10D44000C09193219091BF219C1708F45ACB8091F1
:10D45000BE21C81708F44FC08091C12120918821B6
:10D460003091892190E08217930708F086C2880FD7
:10D47000991F8217930708F480C281E09091872159
:10D48000911180E0809387219091BD21993009F41A
:10D4900044C34ED89091AC21C0918F21D09190215E
:10D4A0004FCB6091CB2161116CCD4632510528F0F4
:10D4B0008BEF8F0F823008F4C1C36091C12170E0FF
:10D4C000660F771F4617570708F4EAC1F83008F4CB
:10D4D000BBCC8AE08093CA2181E08093CB21FECA35
:10D4E00080918F21909190214797089708F4F6CC6E
:10D4F00080E01ED8FDCB9091AC21923109F475C12A
:10D500001092942110928F2110929021C0E0D0E0CF
:10D5100017CB1092872180E480938E2178CE4091A2
:10D520000020509101202091A1213091A221421789
:10D53000530709F074CB40918C2150918D214A3CC6
:10D54000584008F06CCB4091A32141604093A32147
:10D5500066CBE0930020F09301209A0144CB86959E
:10D5600081700E949862C4CB809193218250873051
:10D5700008F0E9CA9E01285031092730310508F426
:10D5800059C3CE010197059708F4A1C38091BD212D
:10D590008111D9CA81E1ECEAF1E2ADEBB1E201908F
:10D5A0000D928A95E1F71092AC2180919D21909186
:10D5B0009E218093A1219093A22180919B21909103
:10D5C0009C2180939F219093A021BDCA2AEF280F10
:10D5D0002530B8F460918F2170919021FB01FC9768
:10D5E000709728F06A5171096930710550F465E04F
:10D5F00074E055CB10928A2110928B211092AB21AE
:10D60000FECA36EF380F3D3008F07EC060918F21A2
:10D61000709190216E5071096031710508F074C0ED
:10D6200064EF73E03CCB8695817091E089270E947E
:10D6300098625ECB8091CB218111DCCC91E09F0F71
:10D640009093CE2192CA2091CE21203109F06BCE49
:10D65000809193218550883008F024CD80918F21CE
:10D6600090919021AC014C5351094031510508F083
:10D6700032C31092912181E18093CE216CCA80EF58
:10D680008F0F823008F429C284EE8F0F823008F0A9
:10D69000BDCC81E08093CB2128E22093BD21F09383
:10D6A000CA21209197213091982120939F21309376
:10D6B000A0212091992130919A212093A12130938A
:10D6C000A2218093942153CA9091CE21983009F0E1
:10D6D0002ACE20918F21309190212C52310929326C
:10D6E000310508F020CE8BE18093BD211092C62138
:10D6F0009093C7219093C82180E18093C9218093A2
:10D70000CA211092912127CA3DED380F3B3008F015
:10D710005CC060918F21709190216B5071096630CF
:10D72000710508F052C0109288211092892181E081
:10D730008093872160EC74E0B2CA20939F213093DC
:10D74000A02110928A2110928B218093AA2180918E
:10D75000A1219091A2218093A8219093A9212093A7
:10D76000A6213093A7214BCAF03209F40BC2FC3139
:10D7700009F4EEC180EF8F0F823008F047CC81E0D2
:10D780008093CB2184E18093BD21F093CA21209125
:10D79000A1213091A22180919D2160E070E0782F3D
:10D7A000770FA901529542954F7045275F70452725
:10D7B000462B572B40939F215093A0212F70332746
:10D7C0002093A1213093A221D2C9543008F08DC0FA
:10D7D00060918F2170919021605371096E307105B5
:10D7E00008F083C06FEA74E05ACA8EEF8C0F87305E
:10D7F00008F086CEC0918F21D09190219E012850B3
:10D8000031092730310538F0AE014150510945301A
:10D81000510508F075CE1092BD21AFCE8F3041F486
:10D820004F3F91E0590709F001CD1092AB21E7C9B4
:10D83000803149F1823009F0FEC291111FC0209160
:10D840008C2130918D212830374008F0EEC0E091D6
:10D850000020F0910120E093A121F093A221609398
:10D860009F217093A0219091A32191609093A32177
:10D8700010928C2110928D21AB01A2C9E091A121BF
:10D88000F091A2219DC9E091A121F091A221EF3F49
:10D89000F10509F095C94E3F510509F091C9C5CF71
:10D8A000FA3008F462C980E18093BD2189E0809359
:10D8B000C62131E13093C72131E03093C8218093F4
:10D8C000C92140919F215091A021BA016627737010
:10D8D000672B09F44AC95093A1211092A221552720
:10D8E00040939F215093A02140C931EF380F3B3026
:10D8F00008F046C060918F217091902163507109AA
:10D9000065307105E8F56EE974E0C9C9F13108F4D4
:10D910002CC981E18093BD211092C6218BE08093B8
:10D92000C7218093C82186E18093C92140919F211E
:10D930005091A0216091A1217091A221FB01EE0FD5
:10D94000FF1FEE0FFF1FBA010024660F771F001C98
:10D95000660F771F001C672F702D6E2B7F2B609337
:10D96000A1217093A2214F73552780918721482BC5
:10D9700040939F215093A021F8C88091872184CDA6
:10D980005CEF580F563060F460918F2170919021B8
:10D990006E5071096B30710518F46DE874E07FC941
:10D9A000EEEFE80FE33008F078C060918F217091BE
:10D9B0009021DB0199971D9708F015C110928721DE
:10D9C0006CE774E06CC9A43009F020CBF63109F0A3
:10D9D0001DCB2091A1213091A221220F331F209332
:10D9E000A1213093A22140919F215091A02153FF6A
:10D9F0000AC021602093A1213093A221577F409338
:10DA00009F215093A021209530953770241735071A
:10DA100009F0FCCA1092A1211092A2218FE28093FA
:10DA2000BD2186E18093CA21A2C81092AB21E0916A
:10DA3000A121F091A221C4C82C2F30E02C30310557
:10DA40000CF45FC88091CA21843209F4CFC180E010
:10DA50000E949862109287219091AC21C0918F21F1
:10DA6000D09190216DC88C2F90E00C970CF457C882
:10DA700081E00E9498628091C121C0918F21D09154
:10DA8000902190E0880F991F8C179D0708F0BCC16A
:10DA9000109287219091AC2153C8253008F486C19B
:10DAA0005B3008F0B8C020918F2130919021B901EE
:10DAB000665071096530710530F066507109693042
:10DAC000710508F0A8C0209388213093892181E056
:10DAD000809387216AE574E0E2C881E08093CB21DE
:10DAE00024E12093BD21F093CA212091A1213091FE
:10DAF000A221A901529542954F7045275F70452795
:10DB000040939F215093A0212F7033272093A12170
:10DB10003093A221809394212AC89091CE219130F4
:10DB200009F0B7CC813009F0B4CC94E29093CA21CB
:10DB300025E02093C62124E12093C72125E12093ED
:10DB4000C8219093C9211092A1211092A221A1CCA9
:10DB500081E08093CB2188E28093BD21F093CA219C
:10DB60002091992130919A212093A1213093A221D3
:10DB7000209197213091982120939F213093A021CB
:10DB80000C94B76581E08093CB2182E08093BD2126
:10DB9000F093CA2120919D2130919E21A901542FFB
:10DBA00044275295550F507E6091A1217091A2217A
:10DBB000462B572B4093A1215093A22180919F2166
:10DBC00040E050E0582F550F550F36952795369564
:10DBD000279536952795242B352B20939F2130931D
:10DBE000A0210C94B765253030F49B01DB0191979F
:10DBF000519708F4E6C0655071096430710508F06A
:10DC00004FCF109288211092892181E08093872143
:10DC100062ED73E044C88D51853080F520918F21ED
:10DC2000309190212D5031092330310538F569E4C8
:10DC300074E035C881E00E946463A8CC81E08093E1
:10DC4000CB2188E18093BD2187E08093CA21109287
:10DC5000C6211092C7211092C8218093C9218091BA
:10DC60009F219091A021880F991F2091CF21822B75
:10DC700080939F219093A0210C946E65E330C0F4B3
:10DC800020918F2130919021235531092631310582
:10DC900078F467E274E003C88AE08093BD2180E1F4
:10DCA0008093C821F093C921F093CA210C94B765E1
:10DCB0004B3030F520918F21309190212A5031093D
:10DCC00025303105E8F466E174E00C944F6680E09D
:10DCD0000E9464635BCC39E23093BD212093C8215C
:10DCE00020E32093C9212093CA210F97409708F47D
:10DCF00068CB80E00E949862109291210C94AB65F1
:10DD0000943090F480918F21909190210497049702
:10DD100058F4109288211092892181E08093872104
:10DD200063EE73E00C944F6610929421C0E00C9463
:10DD3000576620918F21309190212D33310508F4C1
:10DD4000B1C92E34310508F030CB883009F039CB19
:10DD500089E08093CE2180919F219091A021880F0E
:10DD6000991F80939F219093A0212DCB80918F218B
:10DD700090919021825D9109869708F093C9109245
:10DD8000912182E08093CE210C94AB6580918F210C
:10DD900090919021885A9109889708F083C9109230
:10DDA000912184E18093CE210C94AB6520918F2149
:10DDB00030919021B901615271096131710508F00A
:10DDC0006FCE209388213093892181E08093872131
:10DDD0006BE674E00C944F6681E00E94986281E0EB
:10DDE00080938721109291210C94AB6581E00E9471
:10DDF000986281E0809387219091AC21C0918F211E
:10DE0000D09190210C94A065109387219091AC2122
:10DE10000C94A065809187210E94986210929121B4
:10DE20000C94AB6580E00E9498621092872110925A
:10DE300091210C94AB65893009F0F8C9943209F04E
:10DE40001DCD85E18093AA218091A1219091A221ED
:10DE50008093A8219093A9210C94F365E0E4F9E064
:10DE600081818062818381E08093F0210895E0E4E4
:10DE7000F9E081818F7D81831092F0210895E0E4A3
:10DE8000F9E08FEF9FEF86A397A381818160818363
:10DE90008081846080830895DC01611119C08091C4
:10DEA000FC21811124C08C918093FB2115968C91CB
:10DEB00015978F708093F1219091FB21492F50E0AD
:10DEC000FA013197E033F10560F08091FC2108956B
:10DED0008091FC21882339F38091FC218111F8CFB6
:10DEE000E2CF8827EA5DFE4F8F4F0C94B4F980E0B3
:10DEF000089513968D919C9114979C0136952795C2
:10DF0000369527952093F2218295880F880F807C83
:10DF10008093F32181E08093FC21D7CF12968C91DE
:10DF200012978093EF21843008F4ABC53DEF380F92
:10DF300013964D915C9114972FE080E090E0880F4C
:10DF4000991F40FD8160569547952150C1F7AC015E
:10DF500040785F77440F452F441F550B51954093F0
:10DF6000F221880F8093F321332309F46DC21196B7
:10DF70004D915C91129725E080E090E0880F991F09
:10DF800040FD8160569547952150C1F72091F321BE
:10DF900084FB992790F9922B9093F3218295807FAF
:10DFA0008093F42151C211964D915C91129780E1BA
:10DFB00020E030E0220F331F40FD21605695479549
:10DFC0008150C1F713966D917C91149740E180E0E8
:10DFD00090E0880F991F60FD8160769567954150AC
:10DFE000C1F73093F2212093F3219093F421892FEC
:10DFF00080958093F52181E08093FC2166CF119676
:10E000008D919C9112979C01377036952795369586
:10E010002795369527952093F22113962D913C91C3
:10E020001497A90156954795529542954F704527EB
:10E030005F7045274F718295880F807E842B809377
:10E04000F321822F880F880F880F20FD14C594E0DC
:10E05000892B8093F42181E08093FC2136CF1196A7
:10E060004D915C9112972EE080E090E0880F991F0F
:10E0700040FD8160569547952150C1F713966D91EB
:10E080007C9114974CE020E030E0220F331F60FDBC
:10E090002160769567954150C1F78093F2211092E7
:10E0A000F3211092F4212093F52120952093F6215D
:10E0B00081E08093FC2109CF11962D913C9112971C
:10E0C00084E060E070E0660F771F20FD61603695A8
:10E0D00027958150C1F713964D915C9114972CE0D0
:10E0E00080E090E0880F991F40FD8160569547952C
:10E0F0002150C1F79C0122273F706295607F632BFE
:10E100006093F2218093F32181E08093FC21DDCEA6
:10E110008091EB21882309F4B0C420E02093EB2107
:10E1200011968D919C911297AC0144275073352F15
:10E1300032953F70306E3093F2219F7092958295A8
:10E140008F7089279F7089278093F32113968D9173
:10E150009C91149711963C911197432F4295407FC3
:10E16000392F32953F70342B232B2093F421807F5D
:10E170009F70929582958F7089279F7089278093D1
:10E18000F52113968C918295807F8093F62181E012
:10E190008093FC219ACE13968C918295880F880FDC
:10E1A000807C8093F22181E08093FC218ECE1196B9
:10E1B0004D915C91129788E020E030E0220F331FF0
:10E1C00040FD2160569547958150C1F713966D919A
:10E1D0007C91149748E080E090E0880F991F60FDE3
:10E1E0008160769567954150C1F72093F221809325
:10E1F000F32181E08093FC2168CE11964D915C91D2
:10E2000012972DE080E090E0880F991F40FD81601B
:10E21000569547952150C1F713966D917C911497AF
:10E2200048E020E030E0220F331F60FD216076954A
:10E2300067954150C1F7AC01407E5F715695479597
:10E24000529542954F7045275F7045274093F221C4
:10E25000AC0140955095BA0166277C71972F969531
:10E260009695682F660F660F660F962B9093F32195
:10E270004C7F537056954795569547954093F4219A
:10E2800080958295880F880F807CA9014C7F552747
:10E290005695479556954795842B8093F521C9014E
:10E2A000809590958C7F99279695879596958795DB
:10E2B000922F9295990F990F907C892B8093F6213C
:10E2C00020952295220F220F207C2093F72181E0B8
:10E2D0008093FC21FACD47E02DE730E080E090E02C
:10E2E000880F991F20FD8160369527954150C1F711
:10E2F0009C013695322F22273795279513966D91DD
:10E300007C91149747E080E090E0880F991F60FDB2
:10E310008160769567954150C1F7822B932B282F0A
:10E32000220F21602093F2210024880F991F001CE6
:10E33000880F991F001C892F902D8093F32181E075
:10E340008093FC21C2CD8091EA21882309F497C3F0
:10E3500040E04093EA2113962D913C911497119639
:10E360008C91582F5295507FC901807799279295AB
:10E3700082958F7089279F708927852B842B8093A6
:10E38000F2212295207F2093F32181E08093FC21CC
:10E390009CCD13968D919C91149711962C9120935E
:10E3A000F2219093F3218093F4219C0122273F7066
:10E3B000292F22952F70280F230F807F9927929560
:10E3C00082958F7089279F708927820F8295807F21
:10E3D0008093F52181E08093FC2177CD11964D91BA
:10E3E0005C91129780E120E030E0220F331F40FD66
:10E3F0002160569547958150C1F713966D917C9198
:10E40000149740E180E090E0880F991F60FD8160E3
:10E41000769567954150C1F73093F2212093F3210F
:10E420009093F42190959093F5218093F621809517
:10E430008093F72181E08093FC2147CD13968C9146
:10E44000880F880F8093F22181E08093FC213DCDDD
:10E4500013964D915C9114972BE080E090E0880F2B
:10E46000991F40FD8160569547952150C1F79C0149
:10E470002C7F3770369527953695279536952795B5
:10E480002093F2219C0120953095207C3770002448
:10E49000220F331F001C220F331F001C232F302D8F
:10E4A000982F9295990F907E292B2093F321809598
:10E4B000880F880F8093F42181E08093FC2105CDA3
:10E4C00013964D915C91149720E180E090E0880FC5
:10E4D000991F40FD8160569547952150C1F7909353
:10E4E000F221892F80958093F32181E08093FC2194
:10E4F000ECCC11962D913C911297C9019695879578
:10E500009695879580688093F22113968D919C91C2
:10E5100014972295220F220F207CAC015695479527
:10E5200056954795242B2093F3218295880F880FC9
:10E53000807C8093F42181E08093FC21C6CC1396EB
:10E540008D919C9114979C01220F232F221F330B36
:10E5500031952093F221880F8093F32181E08093FD
:10E56000FC21B3CC8091EB21882309F482C280E0A6
:10E570008093EB2111964D915C9112979A01207E28
:10E58000332736952795329522952F7023273F7094
:10E5900023272068282B2093F22113962D913C915C
:10E5A0001497C901807E99279695879592958295B3
:10E5B0008F7089279F708927440F440F440F842B45
:10E5C0008093F321220F220F220F2093F42181E068
:10E5D0008093FC217ACC11964D915C91129780E149
:10E5E00020E030E0220F331F40FD21605695479513
:10E5F0008150C1F713966D917C91149740E180E0B2
:10E6000090E0880F991F60FD816076956795415075
:10E61000C1F73093F2212093F3219093F42180935A
:10E62000F52181E08093FC2150CC20E030E0119670
:10E630003C91119713968D919C911497822B932B5B
:10E6400020E14EEE57E860E070E056954795215086
:10E6500049F0660F771F40FFF8CF616056954795E8
:10E660002150B9F740E120E030E0220F331F80FD58
:10E670002160969587954150C1F782E08093FB21F8
:10E680007093F2216093F3213093F4218BE880930F
:10E69000F52181E08093FC2118CC8091ED21882325
:10E6A00009F4E5C130E03093ED2113964D915C9172
:10E6B000149711962C91822F8F70282F220F220FE2
:10E6C000CA0180739927929582958F7089279F70D0
:10E6D0008927822B8068832B8093F2214295407F8B
:10E6E0004093F32181E08093FC21EFCB11964D9173
:10E6F0005C91129780E120E030E0220F331F40FD53
:10E700002160569547958150C1F713966D917C9184
:10E71000149740E180E090E0880F991F60FD8160D0
:10E72000769567954150C1F740E44093F22144E06B
:10E730004093F32141E04093F4213093F52120935D
:10E74000F6219093F7218093F8214093FC21BDCBD3
:10E7500011964D915C9112978CE020E030E0220FF1
:10E76000331F40FD2160569547958150C1F71396A0
:10E770006D917C9114974CE080E090E0880F991F98
:10E7800060FD8160769567954150C1F7AC01407F8F
:10E790005F70529542954F7045275F7045274093B3
:10E7A000F221A90144275F708295807F852B809399
:10E7B000F3212093F42181E08093FC2186CB80918A
:10E7C000EE21882309F44CC130E03093EE211396FA
:10E7D0004D915C91149711962C91822F8770282F60
:10E7E000220F220F220FCA018873992796958795C9
:10E7F0009695879596958795822B8068832B809335
:10E80000F2214295440F407E4093F32181E08093B2
:10E81000FC215BCB11964D915C91129780E120E039
:10E8200030E0220F331F40FD2160569547958150FF
:10E83000C1F713966D917C91149740E180E090E0D0
:10E84000880F991F60FD8160769567954150C1F7EB
:10E850003093F2212093F321382F307F292F2295F6
:10E860002F70232B2093F4219C0122273F708827AF
:10E87000907F80959095492F42954F70C901929550
:10E8800082958F7089279F708927842B8093F5212B
:10E8900020953095329522952F7023273F7023279E
:10E8A000207F2093F62181E08093FC210ECB809184
:10E8B000EC21882309F4D8C020E080E08093EC218B
:10E8C00013968C91139786FFCDC090E011963C91E2
:10E8D0003F71330F85FB442740F9342B922B932B48
:10E8E0009093F221880F880F880F8093F32181E0A5
:10E8F0008093FC21EACA13968D919C9114971196EE
:10E900002C911197422F440F440F440F9C01207803
:10E910003370220F232F221F330B3195242B20938A
:10E92000F221282F220F2093F3219C01209530956E
:10E9300020783370220F232F221F330B319511962D
:10E940009C91990F990F990F292B2093F421809571
:10E95000880F8093F52181E08093FC21B6CA13963D
:10E960004D915C91149720E030E0220F331F40FD61
:10E970002160569547959150C1F78FEF8093F22112
:10E9800080EC8093F321C90196958795969587959C
:10E9900080688093F4212295220F220F207C2093FF
:10E9A000F52181E08093FC2190CA11964D915C91F4
:10E9B000129728E080E090E0880F991F40FD816069
:10E9C000569547952150C1F713966D917C911497F8
:10E9D00048E020E030E0220F331F60FD2160769593
:10E9E00067954150C1F74FEB4093F2214FEF4093B1
:10E9F000F32140E84093F421A901569547954068DA
:10EA00004093F521279522272795AC0156954795E8
:10EA1000242B2093F6218795882787958093F721CB
:10EA200081E08093FC2151CA13968D919C9114979B
:10EA3000292F2695269526952093F2219C0136951F
:10EA4000279536952795369527952093F32182951E
:10EA5000880F807E8093F42181E08093FC2135CA69
:10EA600030E4B3CE90E832CF20E480E427CF30E426
:10EA70001ACE88E07DCD90E0EBCA28E04FCB48E08D
:10EA800068CC30E055CACF93DF938091FC21882376
:10EA900061F180910A208F3F69F18091FC218823E8
:10EAA00071F010920920E091FB218E2F90E0FC0183
:10EAB0003197E033F10508F45FC01092FC2180919A
:10EAC000FC21811112C08091D1219091DD21891703
:10EAD00008F058C09091FB21923109F491C18F5FE9
:10EAE0008093D12181E08093FC218091FC21DF91F2
:10EAF000CF91089590910920992379F22091E921ED
:10EB0000222309F41FC18091E7219091E821019609
:10EB10008093E7219093E8214091E5215091E621EF
:10EB20008417950710F31092E7211092E821809145
:10EB3000FB21883009F4FAC68091FB218F3009F45B
:10EB400022C78091FB21883109F450C78091FB21B5
:10EB5000803109F0A2CF822F90E001962091E3212D
:10EB600030E0821793070CF0FDC787E180930A20FD
:10EB700089E28093E42191CF8827EA5AFE4F8F4F94
:10EB80000C94B4F981E08093FC218093DE211092F3
:10EB9000DD211092D121A9CF9091DC218091082014
:10EBA000981709F43FC120910A208091FB218F30F2
:10EBB00009F4F6C08091FB21883109F4F1C08091FD
:10EBC000FB21803109F4ECC08091FB212F3F09F437
:10EBD000F0C1893009F4B4C68091FB21853109F474
:10EBE000AFC6E22FE695E695E695F0E0EE50FE4DD5
:10EBF000808190E030E0209530952770332702C067
:10EC0000959587952A95E2F781709091FB21973031
:10EC100009F4FAC68111DFC1C091DA21D091DB215C
:10EC20008091062090910720C817D90708F4EEC0FC
:10EC3000C091DC21C11105C08091F021882309F425
:10EC4000E6C6CF5FC093DC213ACFC091DC21C11171
:10EC500070C040910A204F3F09F496C19091E42181
:10EC6000491708F052C19091FB21933009F491C6E5
:10EC70009091FB219B3109F4CDC69091FB219E30F0
:10EC800009F405C1E42FE695E695E695F0E0EE502F
:10EC9000FE4D208130E0842F90E080959095877024
:10ECA0009927A90102C0559547958A95E2F740FF3B
:10ECB000D0C68091D621809308202091D52130E0C4
:10ECC0002093062030930720811118C1C091DA21CA
:10ECD000D091DB218091062090910720C817D90799
:10ECE00008F494C080910A208F5F80930A2090E0FE
:10ECF0004091E4212091D22130E0240F311D821770
:10ED0000930784F08FEF80930A208091E9218F5F31
:10ED10008093E9219091E321891709F495C681E058
:10ED2000809309201092DC211092DA211092DB21CD
:10ED3000C6CE80910820C81748F681E08C0F8093DA
:10ED4000DC21BDCE2091E1213091E2214091DF21F3
:10ED50005091E0212417350708F4EFC09091DE218F
:10ED6000911122C19091F1219F3009F435C6909301
:10ED7000DD211092E1211092E2211092DC2110920B
:10ED8000DA211092DB212091FB21822F90E0FC01FF
:10ED90003197E033F10508F421C11092FC217DCEBA
:10EDA0002F3F09F4D8C08091FB218F3009F4E3C5CF
:10EDB0008091FB21883109F4E2C58091FB218031EB
:10EDC00009F4C4C088E08093082088E090E0809334
:10EDD000062090930720E22FE695E695E695F0E071
:10EDE000EE50FE4D808190E030E020953095277008
:10EDF000332702C0959587952A95E2F781700ACF4F
:10EE00009091F4219F609093F42169CE209721F492
:10EE10008091F021811191C52196C093DA21D09380
:10EE2000DB214DCE2091DA213091DB21809106202B
:10EE3000909107202817390709F0B5CE20910A20B4
:10EE40002F5F20930A208091E421281708F4D5C56C
:10EE50008FEF80930A208091FB218F3009F453C6F5
:10EE60008091FB21883109F44EC68091FB218031CD
:10EE700009F449C61092FC2181E080930920809119
:10EE8000F021882309F44ECF0E94376F4BCF4423E3
:10EE900009F462C6413009F496C6423009F45CC6F2
:10EEA000433109F4AEC608F07CC0E42FE695E69540
:10EEB000E695F0E0EE50FE4D808190E0242F30E0AA
:10EEC000209530952770332702C0959587952A9510
:10EED000E2F78170992723E0209308202091D02128
:10EEE000281709F487C6009709F481C62CE830E09A
:10EEF00020930620309307208093D0218091F02129
:10EF000081111BCF0E942E6F18CF8091D2218823B0
:10EF100009F447C08091D421809308202091E921F1
:10EF20009091E321291708F05AC52091D32130E0B0
:10EF30002093062030930720C7CE2F5F3F4F2093AA
:10EF4000E1213093E2218091FC21D1CD273119F0CC
:10EF50002F3209F037CF8091D9218093082020915A
:10EF6000D7213091D8212093062030930720C091DB
:10EF7000DC21C81708F45ECEC091DA21D091DB21E4
:10EF8000209709F049CF44CF8091D9218093082060
:10EF90002091D7213091D82120930620309307204B
:10EFA00093CE8091082090CE1092FC211092DE2109
:10EFB0009CCD893009F49AC58091FB21853109F4F3
:10EFC00095C58091FB21803209F4E7C58091FB2132
:10EFD000873009F421CE80910820C9CF8827EA57CD
:10EFE000FE4F8F4F0C94B4F986E38093D92187E1CB
:10EFF00090E08093D7219093D82188E08093D62108
:10F0000090E19093D5218093D42184E08093D32103
:10F0100081E08093D22198E39093E4218093E321CF
:10F0200088E592E08093E5219093E6218093DF21AB
:10F030009093E02183E390E08093680990936909BD
:10F040002CCD84E38093D92183E390E08093D72172
:10F050009093D8218DE08093D62196E29093D5218C
:10F060008093D4218CE08093D32181E08093D221BE
:10F0700096E19093E4218093E3211092E521109290
:10F08000E62188E592E08093DF219093E02186E3FA
:10F0900090E08093680990936909FFCC83EC80939A
:10F0A000D9218DE290E08093D7219093D82186E0FA
:10F0B0008093E4218FE08093D6219CE29093D52128
:10F0C0008093D4218EE08093D32181E08093D2215C
:10F0D0008093E3211092E5211092E62184E893E0E9
:10F0E0008093DF219093E02183E390E0809368098F
:10F0F00090936909D2CC84E48093D92183E490E091
:10F100008093D7219093D82188E08093D62196E1EF
:10F110009093D5218093D42187E08093D32181E0FF
:10F120008093D22180E38093E42182E08093E321E5
:10F130008BE490E08093E5219093E62181EC92E0CE
:10F140008093DF219093E02183E390E0809368092E
:10F1500090936909A2CC82E88093D9218FE390E053
:10F160008093D7219093D82188E08093D62198E18D
:10F170009093D5218093D42187E08093D32181E09F
:10F180008093D2219CE19093E4218093E32110921B
:10F19000E5211092E62188E592E08093DF219093AB
:10F1A000E02183E390E0809368099093690975CC2E
:10F1B00087E08093D92122E130E02093D72130935A
:10F1C000D82193E19093D62196E09093D521809316
:10F1D000D42182E18093D32181E08093D2218AE0FF
:10F1E0008093E42182E08093E3218DE092E080939C
:10F1F000E5219093E6218093DF219093E02183E342
:10F2000090E0809368099093690947CC89E08093E6
:10F21000D92126E130E02093D7213093D821809363
:10F22000D62196E19093D5218093D42188E08093D4
:10F23000D32181E08093D2219FE09093E4218093B9
:10F24000E3211092E5211092E6218AE491E0809377
:10F25000DF219093E02183E390E08093680990930D
:10F2600069091BCC24E02093D92182E090E08093AF
:10F27000D7219093D8212093082080930620909343
:10F2800007201092D22182E18093E42181E08093D3
:10F29000E3211092E5211092E6218EEE92E0809318
:10F2A000DF219093E02183E390E0809368099093BD
:10F2B0006909F3CB90E19093D92124E130E02093C8
:10F2C000D7213093D82188E08093D6212093D5216F
:10F2D0008093D42186E08093D32181E08093D22152
:10F2E0009093E4218093E32188E592E08093E521E7
:10F2F0009093E6218093DF219093E02186E390E0D4
:10F300008093680990936909C8CB1092D921109213
:10F31000D7211092D82188E08093D62193E490934E
:10F32000D5218093D4218DE18093D32181E08093F6
:10F33000D2219CE09093E42156CF82E88093D9219A
:10F340008FE390E08093D7219093D82188E0809339
:10F35000D62198E19093D5218093D42187E08093A2
:10F36000D32181E08093D2219AE20DCF82E880936D
:10F37000D9218FE390E08093D7219093D82188E022
:10F380008093D62198E19093D5218093D42187E072
:10F390008093D32181E08093D22191E1F4CE88E063
:10F3A0008093D92127E230E02093D7213093D821D0
:10F3B0008093082088E090E08093062090930720B7
:10F3C0001092D22187E08093E42182E08093E321B0
:10F3D0008DE491E08093E5219093E62186EE96E01E
:10F3E0008093DF219093E02181E490E0809368098D
:10F3F0009093690952CB81E28093D92187E991E00A
:10F400008093D7219093D82182E08093E42188E0F3
:10F410008093D62194E39093D5218093D42186E1E3
:10F4200052CE88E28093D9218CE090E08093D7215E
:10F430009093D82187E08093082087E090E0809324
:10F440000620909307201092D22184E28093E42139
:10F4500081E08093E3211092E5211092E62183EA76
:10F4600092E08093DF219093E02186E390E0809307
:10F4700068099093690911CB8091D1218111109273
:10F480000A2087E88093D92183E490E08093D721F4
:10F490009093D82180E18093E42188E08093D62165
:10F4A00098E19093D5218093D42187E08093D32154
:10F4B00081E08093D221C3CE8FE18093D9218DE06A
:10F4C00090E08093D7219093D82188E28093E42123
:10F4D00085E08093D6219AE09093D5218093D42122
:10F4E00082E0F1CD26E02093D92186E090E0809360
:10F4F000D7219093D82120930820809306209093C1
:10F5000007201092D22186E1A1CF88E08093D921F3
:10F5100027E230E02093D7213093D8218093082030
:10F5200088E090E080930620909307201092D221EB
:10F5300081E18093E42183E08093E3218CE291E0F8
:10F540008093E5219093E62186EE96E08093DF217B
:10F550009093E02183E390E0809368099093690998
:10F560009CCA88E08093D92127E230E02093D721FC
:10F570003093D8218093082088E090E08093062083
:10F58000909307201092D2218AE08093E42182E0B8
:10F59000D3CF83E08093D9212EE230E02093D7218E
:10F5A0003093D8218093D6219CE89093D5218093E5
:10F5B000D4218EE28093D32181E08093D22194E103
:10F5C0009093E4218093E3211092E5211092E621AB
:10F5D00083EA92E08093DF219093E0211092D02182
:10F5E00083E090E0809368099093690956CA84E1AA
:10F5F0008093D92124E030E02093D7213093D82183
:10F600008093D62184E08093D52188E08093D42113
:10F6100083E18093D32181E08093D2218AE080939B
:10F62000E42182E08093E3218DE092E08093E52164
:10F630009093E6218093DF219093E02186E390E090
:10F64000809368099093690928CA82E08093D92140
:10F6500026E330E02093D7213093D8218093D62120
:10F660009EE69093D5218093D42189E48093D32181
:10F6700081E08093D2219CE09093E4218093E32168
:10F680001092E5211092E62183EA92E08093DF2137
:10F690009093E02183E390E0809368099093690957
:10F6A000FCC984E48093D92183E490E08093D7213E
:10F6B0009093D82188E08093D62196E19093D5212C
:10F6C0008093D42187E08093D32181E08093D2215D
:10F6D00090E29093E4218093E32181EC92E0809387
:10F6E000E5219093E6218093DF219093E02183E34D
:10F6F00090E08093680990936909CFC988E280936C
:10F70000D9218CE090E08093D7219093D82187E095
:10F710008093082087E090E0809306209093072054
:10F720001092D22185E192CE1092D9211092D72148
:10F730001092D82185E08093D6219AE19093D5212B
:10F740008093D4218AE08093D32181E08093D221D9
:10F750008FE08093E42182E08093E32183EA92E0CA
:10F760008093E5219093E6218093DF219093E0211F
:10F7700086E390E080936809909369098EC98DE0D3
:10F780008093D9212DE030E02093D7213093D821E8
:10F790008093082020930620309307201092D221D6
:10F7A0008093E42181E08093E3211092E52110927F
:10F7B000E62186E395E08093DF219093E02186E3C4
:10F7C00090E0809368099093690967C982E080930B
:10F7D000D9212EE630E02093D7213093D821809391
:10F7E000D6219EE69093D5218093D42189E48093FD
:10F7F000D32181E08093D2219AE03ECF84E38093AD
:10F80000D92183E390E08093D7219093D8218DE094
:10F810008093D62196E29093D5218093D4218CE0D9
:10F820008093D32181E08093D22198E122CC84E49B
:10F830008093D92183E490E08093D7219093D821BD
:10F8400088E08093D62196E19093D5218093D421AE
:10F8500087E08093D32181E08093D22195E2909339
:10F86000E4218093E3211092E5211092E62187E7BD
:10F8700091E08093DF219093E02183E390E08093F7
:10F8800068099093690909C982E88093D921809118
:10F89000D121882309F4A1C181E290E08093D7218E
:10F8A0009093D8211092E42188E08093D62198E1AA
:10F8B0009093D5218093D42187E08093D32181E058
:10F8C0008093D22162CC84E28093D92188E090E0B9
:10F8D0008093D7219093D82182E18093D62188E02C
:10F8E0008093D52199E09093D4218093D3211092D5
:10F8F000D2218091EF21845F8093E4218091D121F6
:10F90000811101C023E02093E32187E791E08093F8
:10F91000E5219093E6218093DF219093E02181E31C
:10F9200090E08093680990936909B7C880E180935B
:10F930000A208FE18093E421B0C80E94376F6CCA1F
:10F9400087E08093082087E090E0809306209093E2
:10F9500007208091FB21893009F4F1C0243009F49B
:10F9600009C1253009F03DC98DE090E08093062063
:10F970009093072036C92F3009F01ACAECCA2730F5
:10F9800009F01BCAE8CA80930A208AE18093E42127
:10F9900084C8403108F088C088E080930820E42FB4
:10F9A000E695E695E695F0E0EE50FE4D808190E01C
:10F9B000242F30E0209530952770332702C095958D
:10F9C00087952A95E2F780FF6CC086E190E08093EE
:10F9D00006209093072092CA8093DD21CAC92FEF99
:10F9E00030E020930620309307206EC987E0809393
:10F9F0000A208FE08093E42150C81092DC211092FD
:10FA0000DA211092DB21D1C891E0892703C90E9435
:10FA10002E6F17C9483048F588E080930820809100
:10FA2000F221682F70E0842F90E080959095877088
:10FA300099279B0102C0359527958A95E2F720FF0B
:10FA400030C088E190E0C3CF1092FC211092E921F0
:10FA500066C98091D421809308202091D32130E081
:10FA600020930620309307202FC9483009F4A2C004
:10FA7000413108F096CA88E0809308208091F321F4
:10FA8000282F30E08FEF840F90E08095909587705D
:10FA90009927A90102C0559547958A95E2F740FD3F
:10FAA000D0CF87E090E093CF403109F479C0453260
:10FAB00008F077CA8FEF840F98E090930820E82F22
:10FAC000E695E695E695F0E0EE50FE4D208130E0BB
:10FAD00090E08095909587709927A90102C055956F
:10FAE00047958A95E2F740FFDCCF6FCF8091D9210F
:10FAF000809308208091D7219091D821809306206F
:10FB00009093072063CA9091E9219F5F9093E92128
:10FB10008091D121882331F026EE36E02093E52133
:10FB20003093E6212091DD21821770F59091E32139
:10FB30009F5F9093E3218F5F8093D1219DC92430F3
:10FB400009F04FC88DE0809308208DE090E080930D
:10FB500006209093072045C883E0809308208EE21A
:10FB600090E035CF8FEF80930A2081E18093E421EC
:10FB70000C944D7584E1809308208DE090E0809393
:10FB80000620909307202DC88091E321981374C913
:10FB90001092FC211092E9216FC910920A2016CA16
:10FBA00088E08093082083E490E08093062090937F
:10FBB0000720A4C9409308208FE390E0809306209B
:10FBC000909307209BC983E08093082089EE90E002
:10FBD000809306209093072091C98FE390E0809353
:10FBE000D7219093D82180E28093E4215DCE2EE24C
:10FBF00030E07EC98DE590E0809306209093072049
:10FC00007DC983E0809308208BEB90E080930620F1
:10FC10009093072073C968E770E080E090E00E944D
:10FC20006F5D682F70E080E090E00E94A3F82AE00A
:10FC300037ED43EA5FE30E942FF90E9475F8462FE3
:10FC400064ED70E280E390E00E9465EE2FEF83ECBC
:10FC500099E0215080409040E1F700C000001092F0
:10FC60008B220895E0E0FAE010A211A289E091E071
:10FC700086A397A364E080E09AE00E943BED61E0F8
:10FC800080E09AE00C9447ED10922009109221092F
:10FC900067E080E099E00E943BED78940895CF9270
:10FCA000DF92EF92FF920F931F93CF9361E08BE06F
:10FCB0000E94705F81508E3F08F459C10E94A0F6E7
:10FCC0004AEA61E08BE00E943C5F60E571E280E31C
:10FCD00090E00E940EEE6B017C01492F55276627AC
:10FCE000772762E08BE00E943C5F8FE39FE1019702
:10FCF000F1F700C00000A7016627772763E08BE0DB
:10FD00000E943C5F8FE39FE10197F1F700C0000084
:10FD100077276F2D5E2D4D2D64E08BE00E943C5FB8
:10FD20008FE39FE10197F1F700C000004C2D65E0E3
:10FD30008BE00E943C5F64E571E280E390E00E940A
:10FD40000EEE6B017C014F2D55276627772766E065
:10FD50008BE00E943C5F8FE39FE10197F1F700C0C9
:10FD60000000A7016627772767E08BE00E943C5FD1
:10FD70008FE39FE10197F1F700C0000077276F2D17
:10FD80005E2D4D2D68E08BE00E943C5F8FE39FE18C
:10FD90000197F1F700C000004C2D69E08BE00E9454
:10FDA0003C5F68E571E280E390E00E940EEE6B013B
:10FDB0007C01492F5527662777276AE08BE00E9450
:10FDC0003C5F8FE39FE10197F1F700C00000A701BE
:10FDD000662777276BE08BE00E943C5F8FE39FE113
:10FDE0000197F1F700C0000077276F2D5E2D4D2D94
:10FDF0006CE08BE00E943C5F8FE39FE10197F1F79D
:10FE000000C000004C2D6DE08BE00E943C5F6CE573
:10FE100071E280E390E00E940EEE6B017C01492FBD
:10FE20005527662777276EE08BE00E943C5F8FE3C3
:10FE30009FE10197F1F700C00000A701662777272F
:10FE40006FE08BE00E943C5F8FE39FE10197F1F749
:10FE500000C0000077276F2D5E2D4D2D60E18BE0F7
:10FE60000E943C5F8FE39FE10197F1F700C0000023
:10FE70004C2D61E18BE00E943C5F60E671E280E323
:10FE800090E00E940EEE6B017C014F2D55276627F6
:10FE9000772762E18BE00E943C5F8FE39FE101974F
:10FEA000F1F700C00000A7016627772763E18BE028
:10FEB0000E943C5F8FE39FE10197F1F700C00000D3
:10FEC00077276F2D5E2D4D2D64E18BE00E943C5F06
:10FED0008FE39FE10197F1F700C000004C2D65E131
:10FEE0008BE00E943C5F64E671E280E390E00E9458
:10FEF0000EEE6B017C01492F55276627772766E1B7
:10FF00008BE00E943C5F8FE39FE10197F1F700C017
:10FF10000000A7016627772767E18BE00E943C5F1E
:10FF20008FE39FE10197F1F700C0000077276F2D65
:10FF30005E2D4D2D68E18BE00E943C5F8FE39FE1D9
:10FF40000197F1F700C000004C2D69E18BE00E94A1
:10FF50003C5F8FE39FE10197F1F700C00000CF9174
:10FF60001F910F91FF90EF90DF90CF90089562E086
:10FF70008BE00E94705FC82E63E08BE00E94705F90
:10FF8000F82E64E08BE00E94705FC82F65E08BE084
:10FF90000E94705F4C2D50E060E070E0742F662787
:10FFA000552744278A019B012F29680179014C2F8D
:10FFB00050E0542F4427482B60E070E09A01AB01D9
:10FFC0002C293D294E295F2960E571E280E390E00C
:10FFD0000E9471EF8FE39FE10197F1F700C00000ED
:10FFE00066E08BE00E94705FC82E67E08BE00E94A5
:10FFF000705FF82E68E08BE00E94705FC82F69E0A8
:020000021000EC
:100000008BE00E94705F4C2D50E060E070E0742F38
:100010006627552744278A019B012F29680179010A
:100020004C2F50E0542F4427482B60E070E09A0199
:10003000AB012C293D294E295F2964E571E280E35B
:1000400090E00E9471EF8FE39FE10197F1F700C00C
:1000500000006AE08BE00E94705FC82E6BE08BE0CE
:100060000E94705FF82E6CE08BE00E94705FC82FDA
:100070006DE08BE00E94705F4C2D50E060E070E01E
:10008000742F6627552744278A019B012F29680171
:1000900079014C2F50E0542F4427482B60E070E04A
:1000A0009A01AB012C293D294E295F2968E571E2AF
:1000B00080E390E00E9471EF8FE39FE10197F1F7F9
:1000C00000C000006EE08BE00E94705FC82E6FE001
:1000D0008BE00E94705FF82E60E18BE00E94705F01
:1000E000C82F61E18BE00E94705F4C2D50E060E012
:1000F00070E0742F6627552744278A019B012F291A
:10010000680179014C2F50E0542F4427482B60E0C0
:1001100070E09A01AB012C293D294E295F296CE53D
:1001200071E280E390E00E9471EF8FE39FE101971D
:10013000F1F700C0000062E18BE00E94705FC82E02
:1001400063E18BE00E94705FF82E64E18BE00E9417
:10015000705FC82F65E18BE00E94705F4C2D50E00E
:1001600060E070E0742F6627552744278A019B01C1
:100170002F29680179014C2F50E0542F4427482B38
:1001800060E070E09A01AB012C293D294E295F29DE
:1001900060E671E280E390E00E9471EF8FE39FE1FF
:1001A0000197F1F700C0000066E18BE00E94705FEC
:1001B000C82E67E18BE00E94705FF82E68E18BE04B
:1001C0000E94705FC82F69E18BE00E94705F4C2D28
:1001D00050E060E070E0742F6627552744278A01BD
:1001E0009B012F29680179014C2F50E0542F44279F
:1001F000482B60E070E09A01AB012C293D294E2983
:100200005F2964E671E280E390E00E9471EF8FE382
:100210009FE10197F1F700C0000040E068E071E263
:1002200080E390E0CF911F910F91FF90EF90DF90CE
:10023000CF900C9465EE4F925F926F927F928F9267
:100240009F92AF92BF92CF92DF92EF92FF9268E2BD
:1002500071E280E390E00E940EEE6B017C0160E3AE
:1002600071E280E390E00E940EEE4B015C0168E3D6
:1002700071E280E390E00E940EEE2B013C0160E40D
:1002800071E280E390E00E940EEEC11420E8D206F5
:10029000E104F206B1F0811420E89206A104B2064E
:1002A00081F0411420E852066104720651F0611594
:1002B00070488105904829F088ED84BF81E08093E3
:1002C0007900FF90EF90DF90CF90BF90AF909F901C
:1002D0008F907F906F905F904F9008952F923F92F4
:1002E0004F925F926F927F928F929F92AF92BF9246
:1002F000CF92DF92EF92FF920F931F93CF93DF93F2
:10030000CDB7DEB72A97CDBFDEBF682E262E498730
:100310002A87FE013196CE01099611928E179F070A
:10032000E1F76BE470E080E090E00E946F5D809305
:100330003A222FEF83EC99E0215080409040E1F782
:1003400000C00000712C69E0362E78E0472EE7E00F
:100350005E2E20E030E0A9016CEF70E280E390E0D7
:100360000E9471EF20E03FEF4FEF5FEF60E070E839
:1003700080E390E00E94C7EF20E030E040E052E0F0
:100380000E94C7EF20E03FEF4FEF54E00E94C7EF1D
:1003900027E030E040E056E20E94C7EF00E02FEF98
:1003A00044E60E94B4F429E640E00E94F8F448E1F3
:1003B000C42E40E2D42EE12CF12C0FE110E02AE013
:1003C00030E04AE050E00E94B8F02FEF3FEF4FEFEF
:1003D00054E00E94C7EF20913A225CE1C52E50E222
:1003E000D52E223008F4FAC00EE110E020EE31E004
:1003F0004AE050E00E94B8F0F6E38F2EF0E29F2E24
:10040000A12CB12CAEE1CA2ED12CB4E6EB2EF12CEE
:1004100000E911E02AE530E04AE050E00E943FF3B5
:100420002BE3822E20E2922E22EC30E04AE050E0D4
:100430000E943FF330E4832E30E2932E2AE231E033
:100440004AE050E00E943FF3772009F4A7C021E082
:10045000721609F4E3C022E0721609F4DAC023E050
:10046000721609F4D1C023E0271570F425E6C22ED8
:1004700020E2D22EE12CF12C0FE110E024EA31E051
:100480004AE050E00E94B8F020E030E0A9010E946C
:10049000C7EF21E03FEF4FEF5FEF0E94C7EF9B01F7
:1004A000AC013058404351096CEF70E280E390E0BA
:1004B0000E9471EF6CEF70E280E390E00E940EEE1C
:1004C0006B017C0168EF70E280E390E00E940EEE29
:1004D000C616D706E806F90669F70E9470F6A895D1
:1004E000AADE8FEF99EF20E0815090402040E1F7A5
:1004F00000C000006CE271E280E390E00E94DFED5A
:10050000882369F3739494E0971510F494E0792E9E
:10051000803309F45BC0813309F44FC0823309F0A2
:1005200068C0E1E0F0E0EC0FFD1FE70DF11D22E0F7
:1005300020830E9424EF8FEF97E823E181509040C1
:100540002040E1F700C000008A81681202CF8B8151
:100550002812FFCE8C8199859813FBCE80E09D8177
:100560002A85921709F48AC0882309F4F2CE80E024
:100570002A96CDBFDEBFDF91CF911F910F91FF90E3
:10058000EF90DF90CF90BF90AF909F908F907F9033
:100590006F905F904F903F902F900895E5E4CE2E9E
:1005A000E0E2DE2EE12CF12C0FE110E02AE931E04F
:1005B0004AE050E00E94B8F067CF81E0E1E0F0E06F
:1005C000EC0FFD1FE70DF11D8083B3CFE1E0F0E0FC
:1005D000EC0FFD1FE70DF11D1082ABCFE12CF12CCC
:1005E0000EE110E02AE931E046E950E00E94B8F05F
:1005F00003CF8333C1F4E1E0F0E0EC0FFD1FE70D22
:10060000F11D83E0808395CF3DE5C32E30E2D32EEC
:10061000C9CF45E5C42E40E2D42EC4CF5DE4C52E3B
:1006200050E2D52EBFCF843349F4E1E0F0E0EC0F87
:10063000FD1FE70DF11D94E090837BCF853349F4D6
:10064000E1E0F0E0EC0FFD1FE70DF11D25E0208358
:1006500070CF863349F4E1E0F0E0EC0FFD1FE70DC9
:10066000F11D86E0808365CF873351F4E1E0F0E04F
:10067000EC0FFD1FE70DF11D50825BCF81E078CFBD
:10068000883341F4E1E0F0E0EC0FFD1FE70DF11DD0
:1006900040824FCF8933C9F4E1E0F0E0EC0FFD1F59
:1006A000E70DF11D30820E9424EF9FEF27E883E1E0
:1006B000915020408040E1F700C000008A818611FF
:1006C00048CE8B81281245CE45CF8534B9F40E949F
:1006D00024EF8FEF97E823E1815090402040E1F72D
:1006E00000C000008A81681242CF8B8128123FCF60
:1006F0008C81298582133BCF81E031CF833409F08F
:1007000018CF712C16CF9DEF88ED08B618BE84BFA8
:100710009093800008BE0E944B5E8091A10A85FFE5
:10072000FCCF8AEA8093A00A1092872208958F92C4
:100730009F92AF92BF92CF92DF92EF92FF929DEF86
:1007400088ED08B618BE84BF9093800008BEE09183
:100750008722F0E0E057FD4D8080912CA12CB12C38
:1007600081149104A104B104D1F0C12CD12C7601E3
:10077000C3948C2D0E946C5E2FEF89EF90E0215086
:1007800080409040E1F700C000002FEFC21AD20A6B
:10079000E20AF20A8C149D04AE04BF0450F7809163
:1007A000A10A85FFFCCF8AEA8093A00A10928722D3
:1007B000FF90EF90DF90CF90BF90AF909F908F9081
:1007C00008959DEF88ED08B618BE84BF9093800011
:1007D00008BE81E00E946C5E2FEF89EF90E021500F
:1007E00080409040E1F700C00000109287220895F9
:1007F000CF92DF92EF92FF929DEF88ED08B618BE80
:1008000084BF9093800008BE8091A10A85FFFCCF31
:100810008AEA8093A00A8FE39FE10197F1F700C075
:10082000000069E08CE00E94705F809334228FE3C7
:100830009FE10197F1F700C000006AE08CE00E94A0
:10084000705F809333228FE39FE10197F1F700C03F
:1008500000006BE08CE00E94705F809332228FE397
:100860009FE10197F1F700C000006CE08CE00E946E
:10087000705F809331228FE39FE10197F1F700C011
:100880000000909134228091A10A85FFFCCF9093C3
:10089000A00A909133228091A10A85FFFCCF90930A
:1008A000A00A909132228091A10A85FFFCCF9093FB
:1008B000A00A909131228091A10A85FFFCCF9093EC
:1008C000A00A1092B0221092B1221092B22210927D
:1008D000B32269E08CE00E94705F4091B022509199
:1008E000B1226091B2227091B322782B4093B02252
:1008F0005093B1226093B2227093B3226AE08CE0ED
:100900000E94705F4091B0225091B1226091B2225A
:100910007091B322682B4093B0225093B122609320
:10092000B2227093B3226BE08CE00E94705F409122
:10093000B0225091B1226091B2227091B322282F3F
:1009400030E0322F2227C901A0E0B0E0842B952BA4
:10095000A62BB72B8093B0229093B122A093B22202
:10096000B093B3226CE08CE00E94705F4091B022A3
:100970005091B1226091B2227091B322482B4093E2
:10098000B0225093B1226093B2227093B32280912F
:10099000B0229091B122A091B222B091B3220196DF
:1009A000A11DB11D0297A105B10518F1C12CD12CD3
:1009B0007601C394C701B6010E946F5D9091A10AB0
:1009C00095FFFCCF8093A00A9FEFC91AD90AE90AC4
:1009D000F90A8091B0229091B122A091B222B091F7
:1009E000B3220196A11DB11DC816D906EA06FB0661
:1009F00008F31092872210926D2293E288ED08B6D8
:100A000018BE84BF909380008091820081FDFCCF4E
:100A100008BEFF90EF90DF90CF90089582E0809322
:100A2000A32281E090E0A0E0B0E08093A622909322
:100A3000A722A093A822B093A922E0918722F0E0F8
:100A4000E357FD4D2081E0918722F0E0E257FD4D14
:100A50004081E0918722F0E0E157FD4D3081E09147
:100A60008722F0E0E057FD4D808190E0A0E0B0E00B
:100A7000B82FAA2799278827A32B822B50E0542F21
:100A8000442760E070E0842B952BA62BB72B809336
:100A90008E2290938F22A0939022B0939122E09186
:100AA0008722F0E0E057FD4D408169E08CE00E9434
:100AB0003C5FE0918722F0E0E157FD4D40816AE024
:100AC0008CE00E943C5FE0918722F0E0E257FD4D10
:100AD00040816BE08CE00E943C5FE0918722F0E077
:100AE000E357FD4D40816CE08CE00E943C5F10922A
:100AF0008722089581ED97E00E94CA5E2FEF83EF71
:100B000091E0215080409040E1F700C000008091CA
:100B1000A10A85FFFCCF8AEA8093A00A84E0809333
:100B2000A32281E08093872208951F93CF93DF93C0
:100B300000D000D0CDB7DEB72FEF83EF91E021508A
:100B400080409040E1F700C000008091A10A85FF3D
:100B5000FCCF8AEA8093A00A0E94A16383D894D82C
:100B600081E08093452210E009C0A895CE0101964E
:100B70000E94AA63811116C080914522813011F430
:100B8000163099F760E080E09AE00E943BED109209
:100B9000872210926D222696CDBFDEBFDF91CF91C6
:100BA0001F91089599818091A10A85FFFCCF9093B0
:100BB000A00A9A812B818091A10A85FFFCCF209306
:100BC000A00A8091A10A85FFFCCF9093A00A9C8186
:100BD0002D818091A10A85FFFCCF2093A00A8091EE
:100BE000A10A85FFFCCF9093A00A9E818091A10A63
:100BF00085FFFCCF9093A00A1F5FBECFCF9383E009
:100C00008093A32281ED97E00E94CA5E2FEF83EFCD
:100C100091E0215080409040E1F700C000008091B9
:100C2000A10A85FFFCCF8AEA8093A00AC1E0C093A5
:100C300087222AD8C0934522CF91089581E08093DE
:100C40006D22E0918722F0E0EF56FD4DE0818E2F7E
:100C500090E0FC013197E930F10508F0089588270C
:100C6000EA54FE4F8F4F0C94B4F98091A10A85FF8E
:100C7000FCCF8FE08093A00A089545CDB9CDCECEAC
:100C800056CDBCCF9EDD2FEF87EA91E62150804004
:100C90009040E1F700C0000088ED84BF81E08093C0
:100CA0007900089527CF41CFCF92DF92EF92FF9244
:100CB000CF936B017C016D5C7F4F8F4F9F4F0E94E4
:100CC0006F5DC82FC701B6016C5C7F4F8F4F9F4F80
:100CD0000E946F5DF82E81ED97E00E94CA5E2FEFB3
:100CE00089EF90E0215080409040E1F700C0000083
:100CF00080E00E94135F40E060E67FE18DE790E0D6
:100D00000E94C25D80E00E94135F40E065E67FE1E3
:100D10008DE790E00E94C25D80E00E94135FC130C9
:100D2000B1F042E061E67FE18DE790E00E94C25DB4
:100D300080E00E94135F4F2D62E67FE18DE790E037
:100D4000CF91FF90EF90DF90CF900C94C25D41E087
:100D500061E67FE18DE790E00E94C25DE9CFAF924E
:100D6000BF92CF92DF92EF92FF920F931F93CF9398
:100D7000DF93C82F64E370E080E090E00E946F5D35
:100D8000D82F63E370E080E090E00E946F5D482F11
:100D90008C2F90E0019724E3289F6001299FD00CBD
:100DA0001124E12CF12C22E1C20E26E0D21EE11C1E
:100DB000F11C2D2F30E0AEE0B1E00E94BDF9C60E6F
:100DC000D71EE81EF91E86E6489FA0011124C40E16
:100DD000D51EE11CF11CC701B6010E946F5DA82E53
:100DE00090E0019726E6289FE001299FD00D11246D
:100DF000BE01655D7E4F80E090E00E946F5D182F20
:100E0000BE01645D7E4F80E090E00E946F5D082F20
:100E1000BE01635D7E4F80E090E00E946F5DB82E62
:100E200096E6A99EB001112468537F4F80E090E0C0
:100E30000E946F5DA82EBE01665D7E4F80E090E04F
:100E40000E946F5D8823D9F02A2D4B2D602F812FB2
:100E500045DA81110BC0DF91CF911F910F91FF9067
:100E6000EF90DF90CF90BF90AF9008952FEF83EC7D
:100E700099E0215080409040E1F700C00000C70198
:100E8000B6010E946F5D809316201092112081E0C0
:100E900080938B22809140228130E9F68093172045
:100EA000DACF8F929F92AF92BF92CF92DF92EF9262
:100EB000FF920F931F93CF93DF93F82E64E370E0BC
:100EC00080E090E00E946F5D082F63E370E080E0B7
:100ED00090E00E946F5D182F66E670E080E090E081
:100EE0000E946F5DD82F67E670E080E090E00E947E
:100EF0006F5DC82F68E670E080E090E00E946F5D53
:100F00008F2D90E001972AE3289F6001299FD00C44
:100F10001124E12CF12C20ECC20E21E0D21EE11CA8
:100F2000F11C202F30E0AEE0B1E00E94BDF9C60E0A
:100F3000D71EE81EF91E26E6129FC0011124C80E16
:100F4000D91EE11CF11C24E3D29FC0011124C80E5C
:100F5000D91EE11CF11C82E6C89FE0011124CC0ED1
:100F6000DD1EE11CF11CC701B6016E5A7B4F8F4F8D
:100F70009F4F0E946F5D882EC701B6016D5A7B4F4F
:100F80008F4F9F4F0E946F5D982EC701B6016C5A1C
:100F90007B4F8F4F9F4F0E946F5DA82EC701B601F8
:100FA0006B5A7B4F8F4F9F4F0E946F5DB82EC701CA
:100FB000B6016A5A7B4F8F4F9F4F0E946F5D082F7B
:100FC000C701B601695A7B4F8F4F9F4F0E946F5DDB
:100FD000182FC701B601685A7B4F8F4F9F4F0E9451
:100FE0006F5DC82FC701B601675A7B4F8F4F9F4F68
:100FF0000E946F5DD82F4C2F682D81E00E94AC605D
:101000004C2F692D82E00E94AC604C2F6A2D83E04A
:101010000E94AC604C2F6B2D84E00E94AC604C2F82
:10102000602F85E00E94AC604C2F612F86E00E940B
:10103000AC60D13099F0D11103C081E080932606D5
:10104000DF91CF911F910F91FF90EF90DF90CF90A4
:10105000BF90AF909F908F900C94DB5FD09325064C
:10106000EFCF8F929F92AF92BF92DF92EF92FF925B
:101070000F931F93CF93DF93082F64E370E080E01A
:1010800090E00E946F5DD82E63E370E080E090E016
:101090000E946F5DF82E66E670E080E090E00E94AE
:1010A0006F5D182F67E670E080E090E00E946F5D52
:1010B000D82F68E670E080E090E00E946F5D69E6FE
:1010C00070E080E090E00E946F5DC82F6AE670E0FB
:1010D00080E090E00E946F5DE82E6BE670E080E0BB
:1010E00090E00E946F5DA02FB0E0119724E330E004
:1010F0000E94CCF94B015C0122E1820E26E0921E97
:10110000A11CB11C2D2D30E0AEE0B1E00E94BDF974
:10111000860E971EA81EB91E2E2D30E0A2E9B1E062
:101120000E94BDF9DC01CB01880D991DAA1DBB1DD4
:1011300046E6F49E90011124820F931FA11DB11D5C
:1011400044E3149F90011124820F931FA11DB11D30
:1011500042E6D49F90011124820F931FA11DB11D5F
:101160002AE3C29FE0011124BC01CD016C0F7D1F59
:10117000811D911D0E946F5D682F70E080E090E0FE
:101180000E94A3F82AE037ED43EA5FE30E942FF9BB
:101190000E9475F8462F64ED70E280E390E00E94B3
:1011A00065EE80E0DF91CF911F910F91FF90EF905E
:1011B000DF90BF90AF909F908F9008952F923F92B5
:1011C0004F925F926F927F928F929F92AF92BF9257
:1011D000CF92DF92EF92FF920F931F93CF93DF9303
:1011E000C82FD62F142F322E813009F43DC3823000
:1011F00009F44BC3833009F459C3843009F40FC197
:10120000853009F420C3E12CF12CC12CD12C86307F
:1012100009F408C3873009F4F3C2883009F4D0C256
:10122000893009F451C28A3009F42CC16C2F8DE049
:101230000E94705F90E0A0E0B0E080931522909350
:101240001622A0931722B0931822C93009F46DC258
:101250004701A12CB12C88159905AA05BB0508F4F6
:10126000D0C02601612C712C481659066A067B06EF
:1012700008F4B2C06C2F8DE00E94705F90E0A0E097
:10128000B0E08093152290931622A0931722B0937A
:101290001822C93009F403C2CA3009F498C1D13008
:1012A00009F440C0D230B1F0D33009F4C9C0DF91A5
:1012B000CF911F910F91FF90EF90DF90CF90BF9053
:1012C000AF909F908F907F906F905F904F903F90E6
:1012D0002F9008958091152290911622A0911722A7
:1012E000B091182288159905AA05BB0500F3AC0139
:1012F000BD01401B51096109710984169506A606B6
:10130000B70630F4481759076A077B0708F4F3C299
:101310008092152290921622A0921722B092182243
:101320004E2D28C04091152250911622609117220F
:1013300070911822441655066606770608F4B7CF52
:10134000400F511D611D711D4093152250931622AF
:10135000609317227093182244155505660577058A
:1013600048F04092152250921622609217227092F5
:1013700018224C2D6C2F8DE00E943C5FC93009F47F
:10138000A6C2CA3009F093CF40911522509116227F
:101390006091172270911822452F562F672F7727BB
:1013A0006BE08DE00E943C5F409115226CE08DE087
:1013B000DF91CF911F910F91FF90EF90DF90CF9031
:1013C000BF90AF909F908F907F906F905F904F9065
:1013D0003F902F900C943C5F4C2D6C2F8DE00E9421
:1013E0003C5F6C2F8DE00E94705F90E0A0E0B0E069
:1013F0008093152290931622A0931722B09318225F
:101400004ECF4E2D6C2F8DE00E943C5F80911522B7
:1014100090911622A0911722B091182222CF69E450
:1014200070E080E090E00E946F5DC82ED12C6AE4ED
:1014300070E080E090E00E946F5DE82EF12CF6CE27
:10144000412F50E0542F4427052E000C660B770BDC
:1014500043294093152250931622609317227093CC
:1014600018226C2F8DE00E943C5FC93009F44CC2F9
:10147000CA3009F01CCF412F6BE08DE00E943C5F29
:10148000432D94CF61E670E080E090E00E946F5DB4
:10149000C82ED12CDC2CCC2462E670E080E090E0F9
:1014A0000E946F5DC82A63E670E080E090E00E94D1
:1014B0006F5DE82EF12CFE2CEE2464E670E080E0F7
:1014C00090E00E946F5DE82A6AE08DE00E94705F04
:1014D00090E0A0E0B0E08093152290931622A093B4
:1014E0001722B09318226BE08DE00E94705F90E0AD
:1014F000982F8827092E000CAA0BBB0B809315226E
:1015000090931622A0931722B09318226CE08DE0DE
:101510000E94705F4091152250911622609117220F
:10152000709118224A015B01882AD501C401809379
:10153000152290931622A0931722B09318224701E8
:10154000A12CB12C88159905AA05BB0508F022C16C
:101550004E2D6AE08DE00E943C5F4F2D6BE08DE0E8
:101560000E943C5F4E2D6CE08DE00E943C5F2601A6
:10157000612C712C8091152290911622A091172236
:10158000B0911822481659066A067B0608F072CEFA
:101590002C2C4C2D6AE08DE00E943C5F4D2D6BE0C1
:1015A0008DE00E943C5F422D6CE08DE00E943C5F2C
:1015B0006AE08DE00E94705F90E0A0E0B0E0809370
:1015C000152290931622A0931722B09318226BE055
:1015D0008DE00E94705F90E0982F8827092E000C04
:1015E000AA0BBB0B8093152290931622A09317226F
:1015F000B09318226CE08DE00E94705F409115223C
:10160000509116226091172270911822482B409316
:1016100015225093162260931722709318223FCE02
:101620004E2D69E08DE00E943C5F4F2D69E08DE01A
:101630000E943C5F4E2D6AE08DE00E943C5F2601D7
:10164000612C712C8091152290911622A091172265
:10165000B0911822481659066A067B0608F00ACE91
:101660002C2C4C2D69E08DE00E943C5F4D2D69E0F3
:101670008DE00E943C5F422D6AE08DE00E943C5F5D
:1016800069E08DE00E94705F90E0A0E0B0E08093A0
:10169000152290931622A0931722B093182269E086
:1016A0008DE00E94705F90E0982F8827092E000C33
:1016B000AA0BBB0B8093152290931622A09317229E
:1016C000B09318226AE097CF6AE570E080E090E07E
:1016D0000E946F5DC82ED12CDC2CCC246BE570E011
:1016E00080E090E00E946F5DC82A6CE570E080E0C9
:1016F00090E00E946F5DE82EF12CFE2CEE246DE54B
:1017000070E080E090E00E946F5DE82A69E08DE083
:101710000E94705F90E0A0E0B0E08093152290936B
:101720001622A0931722B093182269E08DE00E9440
:10173000705F90E0982F8827092E000CAA0BBB0B36
:101740008093152290931622A0931722B09318220B
:101750006AE08DE00E94705F409115225091162240
:1017600060911722709118224A015B01882AD501E5
:10177000C4018093152290931622A0931722B09350
:1017800018224701A12CB12C88159905AA05BB0583
:1017900008F446CF2601612C712C481659066A06BA
:1017A0007B0608F067CD2C2C4C2D6C2F8DE00E9411
:1017B0003C5FC93009F45ACFCA3009F4EFCE11CEDC
:1017C00063E470E080E090E00E946F5DC82ED12C51
:1017D00067E470E080E090E00E946F5DE82EF12CFD
:1017E00068E08DE00E94705F90E0A0E0B0E0809340
:1017F000152290931622A0931722B093182228CD79
:1018000065E570E080E090E00E946F5DC82ED12C0D
:1018100066E570E080E090E00E946F5DE82EF12CBC
:1018200067E0DFCF61E570E080E090E00E946F5DEF
:10183000C82ED12C62E570E080E090E00E946F5DE0
:10184000E82EF12CF3CC6DE470E080E090E00E9493
:101850006F5DC82ED12C6EE470E080E090E00E94B5
:101860006F5DE82EF12CE2CC6DE370E080E090E05B
:101870000E946F5DC82ED12C6EE370E080E090E096
:101880000E946F5DE82EF12CD1CC61E470E080E025
:1018900090E00E946F5DC82ED12C62E470E080E081
:1018A00090E00E946F5DE82EF12CC0CC65E470E002
:1018B00080E090E00E946F5DC82ED12C66E470E05D
:1018C00080E090E00E946F5DE82EF12CAFCC40915B
:1018D0001522509116226091172270911822452FDF
:1018E000562F672F772769E08DE00E943C5F40917B
:1018F00015226AE05CCD4093152250931622609326
:1019000017227093182236CD412F69E08DE00E9496
:101910003C5F432D6AE04BCD8F929F92AF92BF9276
:10192000CF92DF92EF92FF920F931F93CF93DF93AB
:10193000F82E64E370E080E090E00E946F5D082F75
:1019400063E370E080E090E00E946F5DA82E66E6A1
:1019500070E080E090E00E946F5DB82E67E670E076
:1019600080E090E00E946F5DD82F68E670E080E034
:1019700090E00E946F5D69E670E080E090E00E9478
:101980006F5DC82F6AE670E080E090E00E946F5DB6
:10199000182F6BE670E080E090E00E946F5D6CE6CF
:1019A00070E080E090E00E946F5D882E6DE670E050
:1019B00080E090E00E946F5D982E6EE670E080E01F
:1019C00090E00E946F5DAF2DB0E0119723E530E00D
:1019D0000E94CCF96B017C0120ECC20E21E0D21EEA
:1019E000E11CF11C202F30E0AEE0B1E00E94BDF917
:1019F000C60ED71EE81EF91E212F30E0A2E9B1E085
:101A00000E94BDF9C60ED71EE81EF91E282D30E033
:101A1000A4E3B0E00E94BDF9C60ED71EE81EF91E71
:101A2000292D30E0A7E3B0E00E94BDF9C60ED71E15
:101A3000E81EF91E36E6A39EC0011124C80ED91E69
:101A4000E11CF11C44E3B49EC0011124C80ED91E50
:101A5000E11CF11C52E6D59FC0011124C80ED91E0D
:101A6000E11CF11C8AE3C89FE0011124CC0EDD1EAD
:101A7000E11CF11CC701B6016A597B4F8F4F9F4F84
:101A80000E946F5D80931422C701B60169597B4F94
:101A90008F4F9F4F0E946F5D80931322C701B60145
:101AA00068597B4F8F4F9F4F0E946F5D809312222A
:101AB000C701B60161597B4F8F4F9F4F0E946F5DE9
:101AC00080931122C701B6016F587B4F8F4F9F4FF4
:101AD0000E946F5D80931022C701B60160597B4F51
:101AE0008F4F9F4F0E946F5D80930F22682F8DE074
:101AF0000E94705F90E080930D2290930E2280915F
:101B00001422813081F0823009F47CC1DF91CF91C1
:101B10001F910F91FF90EF90DF90CF90BF90AF900B
:101B20009F908F90089580911322823009F46DC0A8
:101B3000833009F488C0813009F4B6C010920C22B9
:101B400090911222992309F4E3C24601570192E5CC
:101B5000890E94E0991EA11CB11C80E0C0E0DBE17D
:101B60002AC0482FC8279C01225031092230310554
:101B700008F4A9C08630910509F4A5C08531910506
:101B800009F4A1C08B31910509F49DC08091132205
:101B9000823009F474C0833009F47FC0813009F4C5
:101BA00075C080910C228F5F80930C22909112223D
:101BB000891708F0DBC0A5019401280F311D411DD4
:101BC000511DCA01B9010E946F5D90E080930D2202
:101BD00090930E2220911122213019F640910C226F
:101BE00050E02091102230E0285F3F4F421753070A
:101BF00009F0B7CF60910F228DE00E94705F90E0F6
:101C000080930D2290930E22ACCF8091B10885FF76
:101C1000FCCF82E08093B00810920C2280911222B7
:101C2000811193CFC0E08091B10885FFFCCFC093B4
:101C3000B0088091B10885FFFCCF83E08093B008A5
:101C40008091142260CF8091B10985FFFCCF82E0A2
:101C50008093B00910920C2280911222811175CFCD
:101C6000C0E08091B10985FFFCCFC093B00980919D
:101C7000B10985FFFCCF83E08093B009BEC080919D
:101C8000B10885FFFCCF4093B0088BCF8091A108AD
:101C900085FFFCCF4093A00884CF8091B10985FFD8
:101CA000FCCF4093B0097DCF8091A10885FFFCCF88
:101CB00082E08093A00810920C2280911222811160
:101CC00044CFC0E067C0209113222230C1F02330FE
:101CD00049F12130D1F180589F4F80930D2290938C
:101CE0000E222230C1F0233049F1213009F059CFC2
:101CF0009091A10895FFFCCF8093A00852CF20912E
:101D0000B10825FFFCCFD093B00880589F4F809337
:101D10000D2290930E229091B10895FFFCCF8093F5
:101D2000B0083FCF2091B10925FFFCCFD093B00977
:101D300080589F4F80930D2290930E229091B1096D
:101D400095FFFCCF8093B0092CCF2091A10825FFEF
:101D5000FCCFD093A00880589F4F80930D22909382
:101D60000E229091A10895FFC3CFC6CF8EEF8C0FA6
:101D7000823000F1C630F1F0C531E1F0CB31D1F065
:101D800080911322823009F44ECF833009F469CF59
:101D9000813059F58091A10885FFFCCFC093A00840
:101DA0008091A10885FFFCCF83E08093A0088091FB
:101DB0001422A9CE80911322823009F4C7C0833047
:101DC00009F4ADC0813009F493C0D0E0C058DF4FB2
:101DD000C0930D22D0930E22823009F4C5C0833007
:101DE00009F4ABC0813009F491C0823009F421CFED
:101DF000833009F43CCF813099F2809114228230F3
:101E000009F084CE3FE1C30E34E0D31EE11CF11C87
:101E10000E949F5F8FE79EE30197F1F700C00000EB
:101E200088ED0E94AA5F89ED0E94AA5F809113222B
:101E30000E94AA5F10920B2210920C228091122213
:101E4000882309F456C160E0C0E020C0C827209173
:101E50000B22AC01425051094230510508F48DC0AB
:101E60008630910509F489C08531910509F485C052
:101E70004B9709F482C02F5F20930B226F5F609312
:101E80000C2280911222681708F082C0862F90E001
:101E9000A0E0B0E0C396A11DB11DBC01CD016C0D49
:101EA0007D1D8E1D9F1D0E946F5D90E080930D2211
:101EB00090930E222091112260910C22213031F654
:101EC000462F50E02091102230E0285F3F4F42170C
:101ED000530709F0BBCF60910F228DE00E94705F25
:101EE00090E080930D2290930E2260910C22AECF51
:101EF0008091A10885FFFCCF8BE18093A008D0E002
:101F0000C058DF4FC0930D22D0930E228091A108BC
:101F100085FD44CF8091A10885FFF8CF3FCF809108
:101F2000B10985FFFCCF8BE18093B009D0E0C058A8
:101F3000DF4FC0930D22D0930E228091B10985FD11
:101F400094CE8091B10985FFF8CF8FCE8091B108F2
:101F500085FFFCCF8BE18093B008D0E0C058DF4F05
:101F6000C0930D22D0930E228091B10885FD5FCEE3
:101F70008091B10885FFF8CF5ACE2E5F20930B22B7
:101F80006F5F60930C2280911222681708F47ECF55
:101F9000DEEFDC0FD23008F46AC0C63009F467C047
:101FA000C53109F464C0CB3109F461C080910B22C2
:101FB0008D5F0E94AA5F82E00E94AA5F10920C22AD
:101FC00080911222882309F490C060E020C09A0119
:101FD000225031092230310508F47EC046305105C7
:101FE00009F47AC04531510509F476C04B315105E9
:101FF00009F472C0842F0E94AA5F60910C226F5F67
:1020000060930C2280911222681708F042C0862F3C
:1020100090E0A0E0B0E0C396A11DB11DBC01CD01D0
:102020006C0D7D1D8E1D9F1D0E946F5D482F50E021
:1020300040930D2250930E2290911122913039F647
:1020400020910C2230E08091102290E00896281711
:10205000390709F0BCCF60910F228DE00E94705FBC
:10206000482F50E040930D2250930E22B0CF809124
:102070000B2291E0980F90930B228C5F0E94AA5F35
:1020800082E00E94AA5F10920C228091122281119C
:102090009CCFD23030F0C63021F0C53111F0CB31B9
:1020A00021F58BE10E94AA5F80E88C0F0E94AA5F55
:1020B00083E00E94AA5F81E00E949F5FDF91CF9141
:1020C0001F910F91FF90EF90DF90CF90BF90AF9056
:1020D0009F908F900C94DB5F8BE10E94AA5F8091B0
:1020E0000D2280580E94AA5F88CF8C2F0E94AA5F81
:1020F000DFCF83E00E94AA5F82E00E94AA5F109275
:102100000C2280911222C0E0882379F3DEEF5DCFAC
:10211000C0E038CE9F92AF92BF92CF92DF92EF9203
:10212000FF920F931F93CF93DF93F82E64E370E039
:1021300080E090E00E946F5D982E63E370E080E0A5
:1021400090E00E946F5D082F66E670E080E090E00E
:102150000E946F5D182F67E670E080E090E00E94BB
:102160006F5DD82F68E670E080E090E00E946F5DC0
:1021700069E670E080E090E00E946F5DC82F6AE63B
:1021800070E080E090E00E946F5DA82E6BE670E04A
:1021900080E090E00E946F5D6CE670E080E090E08F
:1021A0000E946F5DB82E6DE670E080E090E00E94C6
:1021B0006F5DAF2DB0E0119727E330E00E94CCF9BE
:1021C0006B017C0120ECC20E21E0D21EE11CF11C4F
:1021D000292D30E0AEE0B1E00E94BDF9C60ED71E59
:1021E000E81EF91E2A2D30E0A2E9B1E00E94BDF9F7
:1021F000C60ED71EE81EF91E2B2D30E0A4E3B0E07A
:102200000E94BDF9C60ED71EE81EF91E26E6029FE3
:10221000C0011124C80ED91EE11CF11C24E3129F39
:10222000C0011124C80ED91EE11CF11C22E6D29F68
:10223000C0011124C80ED91EE11CF11C8AE3C89FFD
:10224000E0011124CC0EDD1EE11CF11CC701B6011A
:102250006E5A7B4F8F4F9F4F0E946F5D80930A2273
:10226000C701B6016D5A7B4F8F4F9F4F0E946F5D24
:1022700080930922C701B6016C5A7B4F8F4F9F4F45
:102280000E946F5D80930822C701B6016B5A7B4F95
:102290008F4F9F4F0E946F5D80930722C701B60149
:1022A0006A5A7B4F8F4F9F4F0E946F5D082F20917E
:1022B00007224091082260910A22809109220E94FF
:1022C000DE88DF91CF911F910F91FF90EF90DF900B
:1022D000CF90BF90AF909F9008958F929F92AF92B2
:1022E000BF92CF92DF92EF92FF920F931F93CF9303
:1022F000DF93C82F64E370E080E090E00E946F5DA0
:10230000F82E63E370E080E090E00E946F5DA82EFD
:1023100066E670E080E090E00E946F5DB82E67E6B0
:1023200070E080E090E00E946F5D082F68E670E04A
:1023300080E090E00E946F5D69E670E080E090E0F0
:102340000E946F5D182F6AE670E080E090E00E94C6
:102350006F5D882E6BE670E080E090E00E946F5D1C
:102360006CE670E080E090E00E946F5D982E6DE674
:1023700070E080E090E00E946F5DD82F6EE670E024
:1023800080E090E00E946F5D482F2F2D30E0AEE09E
:10239000B1E00E94BDF96B017C01282D30E0A2E97B
:1023A000B1E00E94BDF9C60ED71EE81EF91E20EC52
:1023B000C20E21E0D21EE11CF11C292D30E0A4E365
:1023C000B0E00E94BDF9C60ED71EE81EF91E242FEC
:1023D00030E0A3E5B0E00E94BDF9C60ED71EE81EAE
:1023E000F91E26E6A29EC0011124C80ED91EE11CCA
:1023F000F11C24E3B29EC0011124C80ED91EE11CB9
:10240000F11C22E6029FC0011124C80ED91EE11C56
:10241000F11C2AE3129FC0011124C80ED91EE11C31
:10242000F11C2C2F30E021503109C901330FAA0BC8
:10243000BB0B9C01AD012D0F311D411D511DA7E3AB
:10244000B0E00E94D2F9C60ED71EE81EF91EC701E1
:10245000B6016E5A7B4F8F4F9F4F0E946F5DC82F02
:10246000C701B6016D5A7B4F8F4F9F4F0E946F5D22
:10247000182FC701B6016C5A7B4F8F4F9F4F0E9498
:102480006F5DD82FC701B6016B5A7B4F8F4F9F4F9F
:102490000E946F5DD230B9F1D33019F121E030E004
:1024A000C13019F1C23091F1C330F1F5829FA00122
:1024B000839F500D112440938C2250938D22113014
:1024C00009F450C010926022DF91CF911F910F91BB
:1024D000FF90EF90DF90CF90BF90AF909F908F9044
:1024E000089520E13EE0C130E9F6829FA001839F7C
:1024F000500D11244093812250938222113021F1FA
:1025000010926222E1CF2CE330E0CACF829FA0017B
:10251000839F500D11244093AC225093AD22113073
:10252000D1F010926122D0CFC43071F6829FA00109
:10253000839F500D11244093AE225093AF2211304F
:10254000C1F010925F22C0CF1093622210926922D4
:1025500010926A22B9CF10936122109267221092D2
:102560006822B2CF109360221092652210926622E8
:10257000ABCF10935F221092632210926422A4CFFB
:102580004F925F926F927F928F929F92AF92BF9283
:10259000CF92DF92EF92FF920F931F93CF93DF932F
:1025A000F82E64E370E080E090E00E946F5DD82E2A
:1025B00063E370E080E090E00E946F5DA82E66E625
:1025C00070E080E090E00E946F5DB82E67E670E0FA
:1025D00080E090E00E946F5D082F68E670E080E088
:1025E00090E00E946F5D69E670E080E090E00E94FC
:1025F0006F5D182F6AE670E080E090E00E946F5DEA
:10260000E82E6BE670E080E090E00E946F5D6CE683
:1026100070E080E090E00E946F5D882E6DE670E0D3
:1026200080E090E00E946F5DD82F6EE670E080E061
:1026300090E00E946F5D982E6FE670E080E090E081
:102640000E946F5DC82F60E770E080E090E00E941C
:102650006F5D482FAF2DB0E0119725E330E00E9469
:10266000CCF92B013C0120EC420E21E0521E611CF2
:10267000711C2D2D30E0AEE0B1E00E94BDF9460E98
:10268000571E681E791E2E2D30E0A2E9B1E00E948F
:10269000BDF973016201C60ED71EE81EF91E282D72
:1026A00030E0A4E3B0E00E94BDF9C60ED71EE81EDC
:1026B000F91E292D30E0A3E5B0E00E94BDF9C60E59
:1026C000D71EE81EF91E242F30E0A6E3B0E00E94DA
:1026D000BDF9C60ED71EE81EF91E26E6A29EC00151
:1026E0001124C80ED91EE11CF11C24E3B29EC001C6
:1026F0001124C80ED91EE11CF11C22E6029FC00164
:102700001124C80ED91EE11CF11C2AE3129FC0013E
:102710001124C80ED91EE11CF11C8C2F90E0A0E002
:10272000B0E09C01AD012D0F311D411D511DA7E3EE
:10273000B0E00E94D2F9C60ED71EE81EF91EC701EE
:10274000B6016D5A7B4F8F4F9F4F0E946F5D8093F4
:102750000622C701B6016E5A7B4F8F4F9F4F0E94D2
:102760006F5D8093052290915D22913009F494C0B1
:1027700090915C22913009F48FC090915B2291304E
:1027800009F48AC090915A22913009F485C0909141
:102790005922913009F480C090915822913009F467
:1027A0007BC090915722913009F476C090915622C7
:1027B000913009F471C090915522913009F46CC0A8
:1027C00090915422913009F467C090915322913036
:1027D00009F462C090915222913009F45DC0909149
:1027E0005122913009F458C090915022913009F44F
:1027F00053C090914F22913009F44EC090914E22D7
:10280000913009F449C090910622292F913039F571
:10281000813039F441E06DE08CE00E943C5F8091B2
:102820000522811107C040E06DE08CE00E943C5F12
:1028300080910522823051F46DE08CE00E94705F3F
:10284000811192C410925D2280910522833009F497
:10285000A6C290910622843009F4FCC1292F92303F
:10286000B1F580910522813039F441E06EE08CE0D1
:102870000E943C5F80910522882309F47BC182304D
:1028800009F4B4C2833009F497C2909106228430CF
:1028900009F4E6C1292F1BC0843089F0DF91CF9164
:1028A0001F910F91FF90EF90DF90CF90BF90AF906E
:1028B0009F908F907F906F905F904F900895909130
:1028C0000622292F913009F4C5C1923099F2933034
:1028D00009F434C1943009F41CC1953009F404C1E1
:1028E000963009F4ECC0973009F4D4C0983009F45C
:1028F000BCC0993009F4A4C09A3009F48CC09B3054
:1029000009F474C09C3009F45CC09D3009F444C0E3
:102910009E3069F19F30B9F0203109F0BFCF80912E
:102920000522813009F4F3C1882309F41BC18230E8
:1029300009F402C2833009F4F2C1843009F0AECF49
:1029400010924E22ABCF80910522813009F41FC234
:10295000882309F41FC1823009F40EC2833009F4C0
:10296000FEC1843009F4D0C120910622D5CF8091D8
:102970000522813009F445C2882309F41BC1823045
:1029800009F41AC3833009F477C390910622843086
:1029900009F4AEC1292FBECF80910522813009F400
:1029A000ADC2882309F4FEC0823009F452C38330DB
:1029B00009F442C390910622843009F493C1292F6F
:1029C000A7CF80910522813009F43BC2882309F406
:1029D00009C1823009F4CDC2833009F45AC3909101
:1029E0000622843009F478C1292F8FCF80910522E7
:1029F000813009F496C2882309F4ECC0823009F4CE
:102A000008C3833009F4F8C290910622843009F497
:102A10005DC1292F77CF80910522813009F4E4C26E
:102A2000882309F4CFC0823009F470C2833009F4DE
:102A300018C290910622843009F442C1292F5FCF39
:102A400080910522813009F431C2882309F4FAC04B
:102A5000823009F42BC3833009F4A1C2909106227D
:102A6000843009F427C1292F47CF80910522813076
:102A700009F4EFC1882309F4DDC0823009F426C2CD
:102A8000833009F42EC290910622843009F40CC1DF
:102A9000292F2FCF80910522813009F40FC288237E
:102AA00009F4C0C0823009F4F6C1833009F4E6C1EC
:102AB00090910622843009F4F1C0292F17CF80911C
:102AC0000522813009F4D0C2882309F4A3C08230E2
:102AD00009F4F7C2833009F47AC290910622843057
:102AE00009F4D6C0292FFFCE80910522813009F448
:102AF0009BC2882309F486C0823009F427C2833040
:102B000009F417C290910622843009F4BBC0292F22
:102B1000E7CE80910522813009F423C2882309F48D
:102B200069C0823009F430C2833009F47DC19091CC
:102B30000622843009F4A0C0292FCFCE809105222F
:102B4000813009F404C18823E9F0823009F461C1BD
:102B5000833009F43EC190910622843009F486C086
:102B6000292FB8CE40E06FE18CE00E943C5F80915D
:102B70000522DDCE40E06EE08CE00E943C5F80915B
:102B800005227DCE40E06FE08CE00E943C5F8091AA
:102B90000522DBCF40E06EE18CE00E943C5F80913B
:102BA0000522D9CE40E06CE18CE00E943C5F809130
:102BB0000522FACE40E06DE18CE00E943C5F8091FE
:102BC0000522DDCE40E069E18CE00E943C5F80910F
:102BD000052229CF40E06AE18CE00E943C5F8091B1
:102BE00005220CCF40E06BE18CE00E943C5F8091BD
:102BF0000522EFCE40E060E18CE00E943C5F8091D6
:102C000005228FCF40E061E18CE00E943C5F809123
:102C1000052272CF40E065E18CE00E943C5F80912C
:102C2000052255CF40E066E18CE00E943C5F809138
:102C3000052238CF40E067E18CE00E943C5F809144
:102C400005221BCF40E068E18CE00E943C5F809150
:102C50000522FECE10925D22292F923009F037CE48
:102C600010925C22292F933009F034CE10925B220F
:102C7000292F943009F031CE10925A22292F953005
:102C800009F02ECE10925922292F963009F02BCE22
:102C900010925822292F973009F028CE10925722EF
:102CA000292F983009F025CE10925622292F9930DD
:102CB00009F022CE10925522292F9A3009F01FCE0A
:102CC00010925422292F9B3009F01CCE10925322CF
:102CD000292F9C3009F019CE10925222292F9D30B5
:102CE00009F016CE10925122292F9E3009F012CEF3
:102CF00010925022292F9F3009F00ECE10924F22B1
:102D0000903109F0CBCD1CCE90910622F7CF41E057
:102D10006FE18CE00E943C5F8091052205CE6FE15F
:102D20008CE00E94705F813009F436C281E08093AC
:102D30004E228091052201CE6FE18CE00E94705FEF
:102D40008111CAC110924E2280910522F3CD41E03B
:102D50006FE08CE00E943C5F80910522F4CE6EE132
:102D60008CE00E94705F813009F41BC281E0809387
:102D70004F2280910522F5CD6EE18CE00E94705FBC
:102D80008111FEC110924F2280910522E7CD41E0D2
:102D90006EE18CE00E943C5F80910522D9CD6DE010
:102DA0008CE00E94705F813009F400C281E0809362
:102DB0005D22809105224DCD6EE08CE00E94705F17
:102DC000813009F411C281E080935C228091052258
:102DD0005CCD6FE08CE00E94705F813009F4EBC144
:102DE00081E080935B2280910522B5CE6EE08CE07D
:102DF0000E94705F8111BEC110925C2280910522F9
:102E000041CD41E06DE18CE00E943C5F8091052264
:102E1000B3CD6FE08CE00E94705F811169C11092A8
:102E20005B228091052294CE60E18CE00E94705F6D
:102E3000813009F4C5C181E080935A228091052236
:102E400076CE41E06BE18CE00E943C5F80910522F0
:102E5000BDCD41E067E18CE00E943C5F809105229E
:102E600009CE69E18CE00E94705F813009F4DAC11B
:102E700081E08093542280910522DBCD66E18CE0D5
:102E80000E94705F813009F4D2C181E080935722A3
:102E9000809105220DCE66E18CE00E94705F811169
:102EA00051C11092572280910522FFCD41E068E187
:102EB0008CE00E943C5F80910522C7CD41E066E135
:102EC0008CE00E943C5F80910522E9CD67E18CE0B7
:102ED0000E94705F81113CC11092562280910522A0
:102EE000CFCD67E18CE00E94705F813009F486C12C
:102EF00081E08093562280910522C5CD41E06CE1AE
:102F00008CE00E943C5F809105224BCD69E18CE012
:102F10000E94705F8111F8C01092542280910522A6
:102F200085CD41E06AE18CE00E943C5F8091052202
:102F300062CD61E18CE00E94705F813009F459C17B
:102F400081E08093592280910522DCCD61E18CE003
:102F50000E94705F8111D2C0109259228091052287
:102F6000CECD41E060E18CE00E943C5F8091052283
:102F7000D5CD6BE18CE00E94705F8111EFC01092A3
:102F800052228091052228CD60E18CE00E94705F82
:102F90008111A8C010925A2280910522C5CD68E106
:102FA0008CE00E94705F813009F42DC181E0809334
:102FB00055228091052252CD6DE18CE00E94705F18
:102FC0008111A8C01092502280910522DBCC65E1CE
:102FD0008CE00E94705F813009F41AC181E0809317
:102FE00058228091052279CD41E069E18CE00E9470
:102FF0003C5F8091052214CD6AE18CE00E94705FF5
:10300000813009F4E7C081E080935322809105224A
:10301000FBCC6AE18CE00E94705F811187C0109246
:10302000532280910522EDCC41E061E18CE00E94C9
:103030003C5F809105225DCD6CE18CE00E94705F69
:10304000813009F4CCC081E0809351228091052227
:10305000B1CC6CE18CE00E94705F811161C0109274
:10306000512280910522A3CC41E065E18CE00E94D1
:103070003C5F8091052228CD6DE18CE00E94705F5D
:10308000813009F4CAC081E08093502280910522EA
:103090007CCC6BE18CE00E94705F813009F495C0BC
:1030A00081E0809352228091052299CC68E18CE0E6
:1030B0000E94705F811140C01092552280910522BC
:1030C000CACC65E18CE00E94705F81115FC01092F4
:1030D000582280910522FECC81E080934E2280917F
:1030E000052228CC81E080935A22809105221CCDB4
:1030F00081E080935B22809105222ACD81E080933C
:10310000592280910522FBCC81E08093542280914A
:1031100005228CCC81E0809350228091052232CC14
:1031200081E0809351228091052241CC81E08093FF
:1031300053228091052265CC81E0809355228091B5
:10314000052289CC81E08093572280910522ADCC65
:1031500081E0809356228091052292CC81E0809379
:1031600052228091052238CC81E080935D228091AB
:1031700005226CCB81E080935C228091052282CB7A
:1031800081E080934F2280910522E8CB81E08093FB
:103190005822809105229ECC10924E2280910522C9
:1031A000CCCB10924F2280910522DBCB10925D2276
:1031B000809105224ECB10925B2280910522CBCCD0
:1031C00010925A2280910522B2CC10925222809104
:1031D000052205CC109253228091052215CC109225
:1031E000512280910522E6CB10925C22809105222B
:1031F0004CCB109259228091052284CC10925622F9
:103200008091052240CC109255228091052226CC37
:10321000109258228091052260CC10925022809109
:103220000522B3CB109254228091052202CC109239
:103230005722809105223CCC2F923F924F925F9271
:103240006F927F928F929F92AF92BF92CF92DF92B6
:10325000EF92FF920F931F93CF93DF9300D000D094
:10326000CDB7DEB7B82E64E370E080E090E00E9456
:103270006F5D882E63E370E080E090E00E946F5DF8
:10328000C82E66E670E080E090E00E946F5DD82E68
:1032900067E670E080E090E00E946F5DE82E68E6EF
:1032A00070E080E090E00E946F5D69E670E080E091
:1032B00090E00E946F5D082F6AE670E080E090E089
:1032C0000E946F5D682E6BE670E080E090E00E94E7
:1032D0006F5D6CE670E080E090E00E946F5D782E9C
:1032E0006DE670E080E090E00E946F5DF82E6EE683
:1032F00070E080E090E00E946F5D982E6FE670E0D5
:1033000080E090E00E946F5D182F60E770E080E041
:1033100090E00E946F5DA82E61E770E080E090E091
:103320000E946F5D482F22E3B21609F406C1AB2D4F
:10333000B0E0119724E630E00E94CCF91B012C018B
:103340002FED220E25E0321E411C511C282D30E0AD
:10335000AEE0B1E00E94BDF9260E371E481E591E90
:10336000262D30E0A2E9B1E00E94BDF9260E371EFD
:10337000481E591E272D30E0A4E3B0E00E94BDF99D
:1033800032012101460E571E681E791E292D30E09C
:10339000A3E5B0E00E94BDF9460E571E681E791ED7
:1033A0002A2D30E0A6E3B0E00E94BDF953014201AE
:1033B000860E971EA81EB91E242F30E0A5E3B0E0AC
:1033C0000E94BDF9860E971EA81EB91E26E6C29E53
:1033D000C0011124880E991EA11CB11C24E3D29EA9
:1033E000C0011124880E991EA11CB11C22E6E29E88
:1033F000C0011124880E991EA11CB11C2AE3029F52
:10340000C0011124880E991EA11CB11C812F90E0CF
:10341000A0E0B0E09C01AD012F0D311D411D511DFB
:10342000A7E3B0E00E94D2F9860E971EA81EB91E2F
:103430000E943F6F7501640184E3C80ED11CE11C3A
:10344000F11C98E5890E911CA11CB11C0BC026E053
:10345000C20ED11CE11CF11C8C149D04AE04BF04EF
:1034600009F455C0C701B6010E946F5D882379F346
:10347000C701B6010E946F5D8983C701B6016E5F07
:103480007F4F8F4F9F4F0E946F5D082F10E0C70145
:10349000B6016F5F7F4F8F4F9F4F0E946F5D182B5C
:1034A0000A831B83C701B6016C5F7F4F8F4F9F4F0D
:1034B0000E946F5D082F10E0C701B6016D5F7F4F5E
:1034C0008F4F9F4F0E946F5D182B0C831D83C70188
:1034D000B6016B5F7F4F8F4F9F4F0E946F5D8E8352
:1034E0000E94327E61E0CE0101960E944C6FA89549
:1034F0002FEF87E893E1215080409040E1F700C032
:10350000000060E080E09AE00E943BEDA0CF2696AC
:10351000CDBFDEBFDF91CF911F910F91FF90EF9054
:10352000DF90CF90BF90AF909F908F907F906F90E3
:103530005F904F903F902F9008958DE0882E8FE1FF
:10354000982E8DE7A82EB12C73CF3F924F925F92A9
:103550006F927F928F929F92AF92BF92CF92DF92A3
:10356000EF92FF920F931F93CF93DF93782E64E334
:1035700070E080E090E00E946F5D882E63E370E071
:1035800080E090E00E946F5DF82E66E670E080E0DB
:1035900090E00E946F5D082F67E670E080E090E0A9
:1035A0000E946F5D182F68E670E080E090E00E9456
:1035B0006F5D69E670E080E090E00E946F5DD82F5B
:1035C0006AE670E080E090E00E946F5D982E6BE606
:1035D00070E080E090E00E946F5D6CE670E080E05B
:1035E00090E00E946F5DA82E6DE670E080E090E0B4
:1035F0000E946F5D382E6EE670E080E090E00E94E1
:103600006F5DB82E6FE670E080E090E00E946F5D25
:10361000C82F60E770E080E090E00E946F5DC82EE8
:1036200061E770E080E090E00E946F5DD82E62E775
:1036300070E080E090E00E946F5DE82E63E770E04C
:1036400080E090E00E946F5D482FA72DB0E01197B9
:1036500028E330E00E94CCF92B013C012FED420E13
:1036600025E0521E611C711C282D30E0AEE0B1E057
:103670000E94BDF9460E571E681E791E292D30E0A6
:10368000A2E9B1E00E94BDF9460E571E681E791EE0
:103690002A2D30E0A4E3B0E00E94BDF9460E571E8B
:1036A000681E791E2B2D30E0A3E5B0E00E94BDF925
:1036B000460E571E681E791E2C2D30E0A6E3B0E0A2
:1036C0000E94BDF9460E571E681E791E2D2D30E052
:1036D000A5E3B0E00E94BDF9460E571E681E791E94
:1036E0002E2D30E0A4E6B0E00E94BDF9460E571E34
:1036F000681E791E242F30E0ACE3B0E00E94BDF9D3
:10370000DC01CB01840D951DA61DB71D46E6F49E78
:10371000900111246C017D01C20ED31EE11CF11C2D
:1037200024E3029FC0011124C80ED91EE11CF11C24
:1037300042E6149FC0011124C80ED91EE11CF11CE1
:103740002AE3D29FC0011124C80ED91EE11CF11C2E
:103750008C2F90E0A0E0B0E09C01AD01230D311D65
:10376000411D511DA7E3B0E00E94D2F9C60ED71E3D
:10377000E81EF91EC701B6016C5C7F4F8F4F9F4F4B
:103780000E946F5D80930422C701B6016D5C7F4F7C
:103790008F4F9F4F0E946F5D8093032282E00E94B3
:1037A0009F5F8FE79EE30197F1F700C0000087ED70
:1037B0000E94AA5F87ED0E94AA5F809104220E9466
:1037C000AA5F809103220E94AA5F81E00E949F5F0E
:1037D000DF91CF911F910F91FF90EF90DF90CF90ED
:1037E000BF90AF909F908F907F906F905F904F9021
:1037F0003F900C94DB5F2F923F924F925F926F92BB
:103800007F928F929F92AF92BF92CF92DF92EF9270
:10381000FF920F931F93CF93DF9300D0CDB7DEB706
:10382000282E64E370E080E090E00E946F5DF82E47
:1038300063E370E080E090E00E946F5DB82E66E682
:1038400070E080E090E00E946F5D082F67E670E016
:1038500080E090E00E946F5D182F68E670E080E0E5
:1038600090E00E946F5D69E670E080E090E00E9469
:103870006F5D8B836AE670E080E090E00E946F5D90
:10388000382E6BE670E080E090E00E946F5D6CE6A1
:1038900070E080E090E00E946F5D582E6DE670E071
:1038A00080E090E00E946F5D482E6EE670E080E060
:1038B00090E00E946F5D682E6FE670E080E090E01F
:1038C0000E946F5D8A8360E770E080E090E00E9474
:1038D0006F5D782E61E770E080E090E00E946F5DA0
:1038E000882E62E770E080E090E00E946F5D982E85
:1038F00063E770E080E090E00E946F5DA82E64E7CF
:1039000070E080E090E00E946F5D898365E770E081
:1039100080E090E00E946F5D482F2F2D30E0AEE0F8
:10392000B1E00E94BDF96B017C01232D30E0A2E9DA
:10393000B1E00E94BDF9C60ED71EE81EF91E2FED9C
:10394000C20E25E0D21EE11CF11C252D30E0A4E3BF
:10395000B0E00E94BDF9C60ED71EE81EF91E262D46
:1039600030E0A3E5B0E00E94BDF9C60ED71EE81E08
:10397000F91E272D30E0A6E3B0E00E94BDF9C60E87
:10398000D71EE81EF91E282D30E0A5E3B0E00E9406
:10399000BDF9C60ED71EE81EF91E292D30E0A4E69B
:1039A000B0E00E94BDF9C60ED71EE81EF91E2A2DF2
:1039B00030E0ACE3B0E00E94BDF9C60ED71EE81EB1
:1039C000F91E242F30E0A4EEB3E00E94BDF9C60E2C
:1039D000D71EE81EF91E36E6B39EC0011124C80E9C
:1039E000D91EE11CF11C64E3069FC0011124C80E1E
:1039F000D91EE11CF11C22E6129FC0011124C80E41
:103A0000D91EE11CF11C6B813AE3639FC0011124B4
:103A1000C80ED91EE11CF11C2A81822F90E0A0E083
:103A2000B0E09C01AD01240D311D411D511DA7E3E6
:103A3000B0E00E94D2F9C60ED71EE81EF91E222D54
:103A400030E021503109C901330FAA0BBB0B9C0197
:103A5000AD016981260F311D411D511DA8E3B0E064
:103A60000E94D2F9C60ED71EE81EF91EC701B60184
:103A70006B5C7F4F8F4F9F4F0E946F5D8983C701A3
:103A8000B6016D5C7F4F8F4F9F4F0E946F5D8A83A1
:103A9000C701B6016C5C7F4F8F4F9F4F0E946F5DD7
:103AA000482F6A8189812396CDBFDEBFDF91CF91F8
:103AB0001F910F91FF90EF90DF90CF90BF90AF904C
:103AC0009F908F907F906F905F904F903F902F903E
:103AD0000C9447EFCF93DF93D82FC62F682F8C2FEE
:103AE0000E94705F8130A1F041E06D2F8C2F0E9409
:103AF0003C5F2FEF83EC99E0215080409040E1F74C
:103B000000C0000081E080931720DF91CF910895DD
:103B100040E06D2F8C2F0E943C5FEBCFAC019C01ED
:103B2000329522952F7023273F702327A7E4B3E017
:103B30000E94BDF996958795969587959695879558
:103B4000882359F060EF78ED869F9001879F300DB4
:103B5000969F300D1124420F531F9A0136952795D9
:103B60003695279536952795A5ECB0E20E94BDF9CC
:103B7000929582958F7089279F708927009759F0B9
:103B800068E17CEF869F9001879F300D969F300DF6
:103B90001124420F531F9A01369527953695279584
:103BA000ABE7B4E10E94BDF996958795882329F08B
:103BB00024E6829F4019510911249A01ADECBCEC16
:103BC0000E94BDF9969587959695879596958795C8
:103BD000805D0895AC019C01329522952F702327BA
:103BE0003F702327A7E4B3E00E94BDF9969587951F
:103BF0009695879596958795882359F060EF78ED8F
:103C0000869F9001879F300D969F300D1124420FA3
:103C1000531F9A0136952795369527953695279502
:103C2000A5ECB0E20E94BDF9929582958F7089272C
:103C30009F708927009759F068E17CEF869F90017B
:103C4000879F300D969F300D1124420F531F9A010C
:103C50003695279536952795ABE7B4E10E94BDF9D7
:103C600096958795882329F024E6829F401951096B
:103C700011249A01ADECBCEC0E94BDF99695879594
:103C80009695879596958795882329F02AE0829FB7
:103C900040195109112480E3840F08952F923F9217
:103CA0004F925F926F927F928F929F92AF92BF924C
:103CB000CF92DF92EF92FF920F931F93CF93DF93F8
:103CC000CDB7DEB7C655D109CDBFDEBF67968FAF82
:103CD0006797082F10E00150110986E6809F500178
:103CE000819FB00C1124B50163537F4F80E090E0B9
:103CF0000E946F5DF82E63E370E080E090E00E9428
:103D00006F5D682EB50166537F4F80E090E00E94A2
:103D10006F5D882EB50165537F4F80E090E00E9473
:103D20006F5D982EB50164537F4F80E090E00E9454
:103D30006F5DB82E6BE470E080E090E00E946F5DF4
:103D400025968FAF25970E9470F620E03FEF4FEF4A
:103D50005FEF60E070E880E390E00E94C7EF2B2DFA
:103D600030E040E050E052604829892C912C982C9A
:103D70008824A12CB12C282939294A295B290E94A1
:103D8000C7EF27E030E040E056E20E94C7EF2D96F3
:103D90006CAF7DAF8EAF9FAF2D97812C912C5401CE
:103DA00010161106DCF4712C26E6729EB001112467
:103DB00063537F4F80E090E00E946F5D282F30E0DA
:103DC000AEE0B1E00E94BDF9860E971EA81EB91E96
:103DD0007394872D90E08017910734F336E6639E45
:103DE000C001112488539F4FA5019401280F391F4A
:103DF000411D511D29962CAF3DAF4EAF5FAF2997A6
:103E00004F2D50E024964EAF5FAF2497452B09F419
:103E100005C1A1E0B0E066961FAE669765961FAE3D
:103E2000659764961FAE649751E05BAFCE01C39671
:103E30001C01FE01F196EBABFCAB11972EE031E0DB
:103E40000E94CCF929964CAC5DAC6EAC7FAC299746
:103E5000460E571E681E791E8E010F5F1F4FF80118
:103E60001192E215F305E1F7C301B2016F577F4FDD
:103E70008F4F9F4F0E946F5DF82EC301B2016E57A6
:103E80007F4F8F4F9F4F0E946F5D6F2D70E0762F99
:103E90006627682B2596FFAD259780E090E0F230ED
:103EA00009F40AC10E94A1F82AE939E949E15FE36E
:103EB0000E940DF80E9475F86B017C016EAF7FAF18
:103EC000C301B2016D577F4F8F4F9F4F0E946F5DAF
:103ED000B82EC301B2016C577F4F8F4F9F4F0E9486
:103EE0006F5D6B2D70E0762F6627682B80E090E089
:103EF0000E94A1F829E23CE54FE05FE30E940DF843
:103F00000E9475F86DAB7EAB8FAB98AF8DA99EA963
:103F100022968EAF9FAF2297C301B20169577F4FA0
:103F20008F4F9F4F0E946F5DB82EC301B20168573B
:103F30007F4F8F4F9F4F0E946F5D6B2D70E0762FEC
:103F40006627682B80E090E00E94A1F829E23CE51A
:103F50004FE05FE30E940DF80E9475F84B015C0191
:103F60006CAF7DAFC301B2016B577F4F8F4F9F4F37
:103F70000E946F5D89AFC301B2016A577F4F8F4FB7
:103F80009F4F0E946F5D99AD692F70E0762F662775
:103F9000682B80E090E00E94A1F82AE939E949E124
:103FA0005FE30E940DF80E9475F869AF7AAF6C0D5F
:103FB0007D1D6132734030F0E0E2F3E0EC19FD0961
:103FC000E9AFFAAF2DA93EA9820E931E31EE8316FA
:103FD00031E0930640F040EE51E08DA99EA9481BC8
:103FE000590B4CAF5DAFC301B2016D5F7F4F8F4F77
:103FF0009F4F0E946F5D813009F497C1863009F4AC
:10400000FEC0FBADFF5FFBAFAF2FB0E024962EAD3F
:104010003FAD24972A173B070CF00FCF20E030E08C
:1040200040E051E22D966CAD7DAD8EAD9FAD2D97EC
:104030000E94C7EF20E030E0A9010E94C7EF21E015
:104040003FEF4FEF5FEF0E94C7EF9B01AC0130588D
:10405000404351096CEF70E280E390E00E9471EF01
:104060006CEF70E280E390E00E940EEE4B015C0189
:1040700068EF70E280E390E00E940EEE86169706ED
:10408000A806B90669F710921720CA5ADF4FCDBFAC
:10409000DEBFDF91CF911F910F91FF90EF90DF90E6
:1040A000CF90BF90AF909F908F907F906F905F90D8
:1040B0004F903F902F9008950E94A1F829E23CE58F
:1040C0004FE05FE30E940DF80E9475F86DAB7EAB88
:1040D0008FAB98AF2DA93EA92EAF3FAFC301B20160
:1040E0006D577F4F8F4F9F4F0E946F5DF82EC3011A
:1040F000B2016C577F4F8F4F9F4F0E946F5D6F2DA6
:1041000070E0762F6627682B80E090E00E94A1F88F
:104110002AE939E949E15FE30E940DF80E9475F848
:104120004B015C0122966EAF7FAF2297C301B201B3
:1041300069577F4F8F4F9F4F0E946F5DF82EC301CD
:10414000B20168577F4F8F4F9F4F0E946F5D6F2D59
:1041500070E0762F6627682B80E090E00E94A1F83F
:104160002AE939E949E15FE30E940DF80E9475F8F8
:104170006B017C016CAF7DAFC301B2016B577F4F08
:104180008F4F9F4F0E946F5D89AFC301B2016A5785
:104190007F4F8F4F9F4F0E946F5D39AD632F70E04F
:1041A000762F6627682B80E090E00E94A1F829E234
:1041B0003CE54FE05FE30E940DF80E9475F869AF9F
:1041C0007AAF4DA95EA9640F751F613E714040F042
:1041D00020EE31E04DA95EA9241B350B29AF3AAF83
:1041E000C80CD91C51E2C51653E0D50608F4FBCE25
:1041F00080E293E0881999098CAF9DAFF4CEC3019A
:10420000B20163587F4F8F4F9F4F0E946F5DF82E12
:10421000C301B20164587F4F8F4F9F4F0E946F5D63
:10422000E82EF110C5C27301620135E0C30ED11C46
:10423000E11CF11CC701B6010E946F5D882311F0DB
:10424000F8018083FFEFCF1ADF0AEF0AFF0A0F5F42
:104250001F4F2016310671F7C301B20163597F4F1A
:104260008F4F9F4F0E946F5D2F968FAF2F97C30187
:10427000B20162597F4F8F4F9F4F0E946F5D6096D2
:104280008FAF6097C301B20161597F4F8F4F9F4F2E
:104290000E946F5D2E968FAF2E97C301B2016059B9
:1042A0007F4F8F4F9F4F0E946F5D61968FAF6197D9
:1042B000C301B2016F587F4F8F4F9F4F0E946F5DB8
:1042C00062968FAF6297C301B2016E587F4F8F4FD6
:1042D0009F4F0E946F5D63968FAF639720E030E041
:1042E00040E053E02D966CAD7DAD8EAD9FAD2D972A
:1042F0000E94C7EF6B017C01C301B20160587F4F80
:104300008F4F9F4F0E946F5D9FEF980F953008F081
:10431000C6C0823009F0CDC164966FAD6497662344
:1043200009F440C308E010E0C3C06BAD67968FADE1
:1043300067970E94705F813009F485C28111F0C2D5
:104340007301620125E0C20ED11CE11CF11CC70102
:10435000B6010E946F5D882311F0F8018083FFEFA2
:10436000CF1ADF0AEF0AFF0A0F5F1F4F2016310630
:1043700071F7C301B20163597F4F8F4F9F4F0E9466
:104380006F5D2F968FAF2F97C301B20162597F4F98
:104390008F4F9F4F0E946F5D60968FAF6097C301F4
:1043A000B20161597F4F8F4F9F4F0E946F5D2E96D4
:1043B0008FAF2E97C301B20160597F4F8F4F9F4F30
:1043C0000E946F5D61968FAF6197C301B2016F5814
:1043D0007F4F8F4F9F4F0E946F5D62968FAF6297A6
:1043E000C301B2016E587F4F8F4F9F4F0E946F5D88
:1043F00063968FAF6397C82ED12CE12CF12C689473
:10440000F2F861962FAD6197E22A62963FAD62970E
:10441000832F90E0982F8827A0E0B0E0C82AD92AFF
:10442000EA2AFB2A3BAD832F90E0A0E0B0E09C019C
:10443000AD0153602D966CAD7DAD8EAD9FAD2D97CA
:104440000E94C7EFA70196010E94C7EF2E960FADFD
:104450002E9760962FAD60972F964FAD2F970E94A5
:10446000F8F46DAB7EAB8FAB98AFC301B20160586F
:104470007F4F8F4F9F4F0E946F5D9FEF980F95303A
:1044800008F0E3C0823009F051C164964FAD6497E3
:10449000442309F4BCC2A8E0CA2ED12CDFC081E0BD
:1044A0009EEF980F933008F43DCF865E082F10E002
:1044B0002E963FAD2E97832F90E0A0E0B0E0B46041
:1044C000AC01BD012F96EFAD2F976E2B6096FFAD1F
:1044D00060978F2F90E0982F8827A0E0B0E09A0196
:1044E000AB01282B392B4A2B5B2BC701B6010E944D
:1044F000C7EF29E030E040E05FE10E94C7EF20E134
:1045000030E040E05EE00E94C7EF2EAD3FAD229567
:104510003295307F3227207F32276901E12CF12C40
:10452000460157015FE0880C991CAA1CBB1C5A95D8
:10453000D1F722962EAD3FAD229722953295307F4E
:104540003227207F32276901E12CF12C6894F6F89C
:10455000A50194012C293D294E295F290E94C7EF0E
:1045600029AD3AAD4EAD5FAD240F351F2295329582
:10457000307F3227207F32276901E12CF12C460160
:104580005701AFE0880C991CAA1CBB1CAA95D1F757
:104590002CAD3DAD2296EEADFFAD22972E0F3F1F05
:1045A00022953295307F3227207F32276901E12C16
:1045B000F12C6894F6F8A50194012C293D294E2987
:1045C0005F290E94C7EF6396FFAD6397CF2ED12C72
:1045D000E12CF12C6894F2F84601570161962FAD59
:1045E0006197A22A62964FAD6297242F30E0322F56
:1045F00022276901E12CF12CA50194012C293D29E8
:104600004E295F290E94C7EF2CAD3DAD3695279509
:104610002296EEADFFAD22972E0F3F1F49AD5AAD4A
:1046200056954795EEADFFAD4E0F5F1FFE013196DB
:104630006F01E12CF6E0FF2E0E94B8F02D966CAFD2
:104640007DAF8EAF9FAF2D97DCCC81E09EEF980FB2
:10465000933008F420CF865EC82ED12CC301B2015E
:104660006A567F4F8F4F9F4F0E946F5D81111DC013
:10467000A12CB12C9E012F5F3F4F4901ECACFDAC4A
:1046800009AD1AAD22962EAD3FAD22974EAD5FAD6E
:104690006DA97EA98FA998AD0E94BAF12D966CAF35
:1046A0007DAF8EAF9FAF2D97ACCCA12CBB24B39424
:1046B000E1CF833009F07BC265969FAD659791117C
:1046C00031CE28E030E040E055E0C701B6010E945D
:1046D000C7EF2CE932E540E051E00E94C7EF2CE142
:1046E00038E048E057E00E94C7EF2CE134E340E0B7
:1046F00058E00E94C7EF18E0E12E12E5F12E00E02D
:1047000010E028E030E040E050E00E9428F76B0124
:104710007C0166961FAE6697E1E06596EFAF659700
:1047200064961FAE649708E010E0C2CE833009F0B3
:10473000FCC165966FAD65976111ADCE28E030E0A4
:1047400040E055E06DA97EA98FA998AD0E94C7EF02
:104750002CE932E540E051E00E94C7EF2CE138E05F
:1047600048E057E00E94C7EF2CE134E340E058E016
:104770000E94C7EF18E0E12E12E5F12E00E010E0F4
:1047800028E030E040E050E00E9428F76DAB7EABBF
:104790008FAB98AF66961FAE669781E065968FAF38
:1047A000659764961FAE6497A8E0CA2ED12C56CFA9
:1047B0006F2D8DE00E94705F482F50E029E0F216C7
:1047C00009F469C13AE0F31609F47CC1409301226F
:1047D000509302229A013695279536952795ABE797
:1047E000B4E10E94BDF98C01169507956CE9600350
:1047F00090011124240F351FADECBCEC0E94BDF9D3
:104800009C01369527953695279536952795942FB3
:104810008CE9809F900D1124EAE02E9F90191124BD
:10482000F1E0EF1609F42DC142E0E41609F42DC1C0
:1048300053E0E51211CD005D0983205D2A83905D70
:104840009B831C8209CD7301620197E3C90ED11CC1
:10485000E11CF11CC701B6010E946F5D882311F0B5
:10486000F8018083FFEFCF1ADF0AEF0AFF0A0F5F1C
:104870001F4F2016310671F7C301B2016A587F4FEE
:104880008F4F9F4F0E946F5D2F968FAF2F97C30161
:10489000B20169587F4F8F4F9F4F0E946F5D6096A6
:1048A0008FAF6097C301B20168587F4F8F4F9F4F02
:1048B0000E946F5D2E968FAF2E97C301B20167588D
:1048C0007F4F8F4F9F4F0E946F5D61968FAF6197B3
:1048D000C301B20166587F4F8F4F9F4F0E946F5D9B
:1048E00062968FAF6297C301B20165587F4F8F4FB9
:1048F0009F4F0E946F5D63968FAF63976396EFAD96
:104900006397CE2ED12CE12CF12C6894F2F86196AD
:10491000FFAD6197EF2A62962FAD6297822F79CD16
:10492000833009F0DEC04AE249837301620155E039
:10493000C50ED11CE11CF11C8E010E5F1F4FC7017B
:10494000B6010E946F5D882311F0F8018083FFEFAC
:10495000CF1ADF0AEF0AFF0A0F5F1F4F2BA93CA9EE
:104960002017310761F7CC24CA94DC2CEC2C54E0DE
:10497000F52E3FEF63963FAF63974FEF62964FAFD1
:1049800062975FEF61965FAF619760EF2E966FAFB2
:104990002E9780EF60968FAF609790EF2F969FAF26
:1049A0002F9740CD28E030E040E055E0C701B60148
:1049B0000E94C7EF2CE83BE240E051E00E94C7EFC5
:1049C00027E136E048E057E00E94C7EF27E138E2F0
:1049D00040E058E00E94C7EF18EFE12E1AE2F12EF6
:1049E00000E010E028E030E040E050E00E9428F7CE
:1049F0006B017C0166961FAE669765961FAE659744
:104A000081E064968FAF649708E010E051CD28E014
